:020000040000FA
:100000000C945D070C948E070C948E070C948E074D
:100010000C948E070C948E070C948E070C948E070C
:100020000C948E070C948E070C948E070C948E07FC
:100030000C948E070C9461870C948E070C948E0799
:100040000C948E070C948E070C948E070C948E07DC
:100050000C948E070C948E070C948E070C9440859C
:100060000C948E070C94517E0C94277E0C948E0772
:100070000C948E070C948E070C948E070C948E07AC
:100080000C948E070C948E070C948E070C948E079C
:100090000C948E070C948E070C948E070C94D889C0
:1000A0000C948E070C948E070C948E070C948E077C
:1000B0000C948E070C948E070C948E070C948E076C
:1000C0000C948E070C948E070C948E070C948E075C
:1000D0000C948E070C948E070C94F17D0C94C77DC4
:1000E0000C948E070C9442130C9403140C94C327A5
:1000F0000C9490080C94A1170C9406740C9425741D
:100100000C944B120C9495110C9479080C944E732A
:100110000C94FE720C94DC080C94BA0D0C94DB72F7
:100120000C947A110C9405080C949B730C940E1586
:100130000C94E88E0C9447740C94C8130C94AC7215
:100140000C94D5150C94F5740C942B740C94AE741B
:100150000C9456080C94AE720C949F740C94C87452
:100160000C94AA720C940F7D0C94C0150C943374EB
:100170000C9471080C94256B0C9475080C941D96C6
:100180000C9446740C9493080C9469080C943617DC
:100190000C944B740C9489080C9418170C94441408
:1001A0000C9466080C942F740C94AB720C94931EF0
:1001B0000C94BB710C9495070C9479960C940412D2
:1001C0000C94AD720C94EA720C9423130C94BF0837
:1001D0000C9465150C9468200C9421740C946C1389
:1001E0000C94E6180C940C730C941B740C946C19FE
:1001F0000C94C1740C94C40D0C9470170C941B08CF
:100200000C94E2130C9418740C9441190C94B507D7
:100210000C9439740C945A080C9489890C940C74BD
:100220000C9435080C94BF110C9487150C945B1436
:100230000C941A110C9410740C943D740C941312B9
:100240000C9416190C9464080C941F080C94400824
:100250000C9414740C9441744E414E494E495459B7
:10026000494E46CDCCCC3D0AD7233C17B7D1387781
:10027000CC2B329595E6241FB14F0A000020410097
:1002800000C84200401C4620BCBE4CCA1B0E5AAEE1
:10029000C59D7400407A10F35A00A0724E180900F0
:1002A00010A5D4E80000E87648170000E40B5402DB
:1002B0000000CA9A3B000000E1F505000080969816
:1002C00000000040420F000000A086010000001066
:1002D0002700000000E803000000006400000000A8
:1002E000000A00000000000100000000002C76D889
:1002F00088DC674F0823DFC1DFAE59E1B1B796E56F
:10030000E3E453C63AE651997696E8E6C28426EBD2
:10031000898C9B62ED407C6FFCEFBC9C9F40F2BAE5
:10032000A56FA5F490055A2AF75C936B6CF9676D7D
:10033000C11BFCE0E40D47FEF520E6B500D0ED90D2
:100340002E0300943577050080841E080000204E9F
:100350000A000000C80C333333330F986E12831138
:1003600041EF8D2114893BE65516CFFEE6DB18D10F
:10037000844B381BF77C1D901DA4BBE424203284E1
:10038000725E228100C9F124ECA1E53D27436F6E26
:1003900074656E742D547970653A20746578742F85
:1003A00068746D6C0D0A0D0A3C68313E4550494336
:1003B000204641494C3C2F68313E00485454502F50
:1003C000312E302034303020426164205265717506
:1003D0006573740D0A004163636573732D436F6E1B
:1003E00074726F6C2D416C6C6F772D4F72696769F9
:1003F0006E3A202A0D0A436F6E74656E742D54791F
:1004000070653A20005365727665723A20576562CE
:100410006475696E6F2F312E370D0A0048545450A1
:100420002F312E3020323030204F4B0D0A00436FD9
:100430006E6E656374696F6E3A20636C6F73650DE1
:100440000A436F6E74656E742D547970653A20613D
:1004500070706C69636174696F6E2F782D77777730
:100460002D666F726D2D75726C656E636F64656459
:1004700000506F7374206661696C65640055706C20
:100480006F6164204661696C65643A2000234E6F99
:100490002073656E736F7220666F722074656D7065
:1004A00020262068756D696469747921004E6F207B
:1004B00053656E736F72210020666F722074656DD4
:1004C0007020262068756D69646974792100235352
:1004D000656E736F72204572726F72200053656E85
:1004E000736F72204572726F7221002357726F6EA4
:1004F000672073656E736F7220666F722074656D0E
:100500007020262068756D696469747921005772BE
:100510006F6E672053656E736F7221004320483DF4
:1005200000543D00202020202020202020202020BA
:1005300020202020002020202020202020202020DB
:1005400020202020200020202020202020202020CB
:1005500020202020202000202020202020202020BB
:1005600020202020202000202020202020202020AB
:100570002020202020200054696D657374616D7007
:100580002075706C6F6164206661696C65640053EE
:10059000657474696E6720636C6F636B2074696D3A
:1005A0006500236572726F72202D20004950206112
:1005B0006464726573733A2000496E76616C696495
:1005C00020534D2073746570732070657220616EC6
:1005D000676C653D00534D207374657073207065C2
:1005E0007220616E676C653D003C703E54696D65BC
:1005F0003A20003C2F68333E0A003C62723E42546F
:10060000206E616D653D003C62723E506174683DD4
:10061000003C68333E53797374656D3A20566572B9
:1006200073696F6E3D00506172616D6574657273C0
:1006300020726573657420646F6E6521002F6F658D
:100640002F736D6C69676874706F2F73332F00613F
:100650006E676C6520646972656374696F6E3A20B9
:100660000043757272656E7420534D2069732023A8
:1006700000534D3A5461626C652073746570732049
:1006800070657220616E676C653D00534D3A506F26
:100690006C6172697A65722073746570732070651D
:1006A0007220616E676C653D002344485450494E8A
:1006B0003D00234448543D00236E65743D424C4543
:1006C00000236E65743D5769466900236E65743D6D
:1006D0004254002366747020757365726E616D6597
:1006E0003A003A0023486F7374207365727665721E
:1006F00020495020616E6420506F72743A00235478
:10070000696D65207365727665722049503A0023E1
:1007100052656C617920646576696365733A00237C
:1007200052656C617920737461747573206C6162B9
:10073000656C733A20002352656C61792073746193
:100740007465733A002352656C61792070696E7329
:100750003A00234E6F2E206F6620636F6E74726FA7
:100760006C2072656C6179733D00234E6F2E206F93
:10077000662072656C6179733D0046696E64696ECE
:10078000672057694669204950004E45543D426CE8
:100790007565746F6F7468204C45004E45543D423A
:1007A0006C7565746F6F7468004E45543D576946AB
:1007B00069005344206F70656E206661696C004E5D
:1007C0006577206461746120636F6C6C6563746924
:1007D0006F6E207374617274656400437572726524
:1007E0006E742073657474696E67733A005379731D
:1007F00074656D20726573657420617420002344F4
:100800005320546865726D6F6D6574657220636105
:100810006C6962726174656420666F72202300499E
:100820006E76616C696420616E676C6520666F72BC
:1008300020002073746570732070657220616E678C
:100840006C653D0020737465707320706572206163
:100850006E676C653D005461626C65205365742061
:100860003000235475726E7461626C652053657438
:10087000203000506F6C6172697A65722053657424
:1008800020300023506F6C6172697A657220536565
:10089000742030005461626C652053657420300010
:1008A000235475726E7461626C65205365742030D8
:1008B00000506F6C6172697A6572205365742030E4
:1008C0000023506F6C6172697A65722053657420E1
:1008D0003000576946692049503A00234C6F6767DA
:1008E0006572204E616D653A20004C4F4747455276
:1008F0000056455253494F4E005265626F6F7469FE
:100900006E672E2E2E005245424F4F540053657293
:1009100076657220506F72742075706461746564BE
:100920000053504F52543D0049502075706461741B
:100930006564005349503D002354696D652053653B
:100940007276657220495020757064617465640028
:10095000545349503D004352454C4159004448547A
:1009600050494E3D0074696D6520696E74657276FC
:10097000616C3D0054494D455354414D503D005428
:10098000494D455354414D5000237765627365725C
:1009900076657220626567696E7300536574746969
:1009A0006E672049500053657474696E6720446512
:1009B00076696365204950202E2E2E00506F6C61A1
:1009C00072697A65722053657420300023506F6C11
:1009D0006172697A657220536574203000546573C2
:1009E00074204C616D70732F46616E730065727276
:1009F0006F72206F70656E696E672066696C653A0C
:100A000020004C616D70204D6F746F72002354692B
:100A10006D65202020202020446174652020202046
:100A2000205365636F6E647320506F6C6172697AD6
:100A30006572205461626C652054286F43292048F8
:100A4000282529202000696E69742E20646F6E6548
:100A50002E00534420696E69742E206661696C65AE
:100A6000642100696E69742E206661696C65642179
:100A7000002323204F452057656C636F6D6520234D
:100A80002300496E697469616C697A696E672053E5
:100A90004420636172642E2E2E0075706C6F616449
:100AA00020627920465450206661696C656421009B
:100AB00075706C6F616420627920465450204F4BF2
:100AC000210053797374656D207374617274696E5B
:100AD000672E2E2E003C703E4C616D7020616E645E
:100AE000204D6F746F722044726976657273205363
:100AF0007461747573EFBC9A3C2F703E003C2164A6
:100B00006F63747970652068746D6C3E3C68746DB9
:100B10006C3E3C686561643E3C6D65746120636851
:100B200061727365743D227574662D38223E3C7483
:100B300069746C653E4F6E6C696E65206578706592
:100B400072696D656E74202D20506F6C6172697AC8
:100B50006174696F6E2065666665637473206F6685
:100B6000206C696768743C2F7469746C653E3C2F17
:100B7000686561643E3C626F64793E3C68313E4F1B
:100B80006E6C696E65206578706572696D656E74EE
:100B9000202D20506F6C6172697A6174696F6E20CC
:100BA00065666665637473206F66206C6967687438
:100BB0003C2F68313E003C68343E436F7079726967
:100BC000676874284329323032302D323032322E69
:100BD00050726F662E205945554E47205961752039
:100BE0005975656E3C2F68343E3C2F626F64793EC8
:100BF0003C2F68746D6C3E003C68313E43616E6E04
:100C00006F74206765742073656E736F72207265F0
:100C10006164696E6773213C2F68313E007C3C3E05
:100C20005E2B3D3F2F5B5D3B2C2A225C00000020A9
:100C3000002300260029002C002F003200000100B4
:100C40000003010601090100000A0B02090C0D0E48
:100C5000080703040100000000000000000000007D
:100C60000000000000000000000000000000000084
:100C70000000001211100000000000000000000041
:100C80000000000000000000000000000053797325
:100C900074656D20726573746172746564210020DF
:100CA00053797374656D20726573746172746564D1
:100CB00021004E6574776F726B206D61696E74618F
:100CC000696E656420617420002323436F6D6D613C
:100CD0006E64400000002200250028002B002E003A
:100CE0003100340002010000050108010B01000081
:100CF0002100240027002A002D00300033000101CC
:100D00000000040107010A01010210202008081058
:100D1000204010204080020102010804020101026B
:100D20000408102040808040201008040201800444
:100D3000020180402010080402010804020101029F
:100D4000040810204080010204081020408005059E
:100D50000505070508080808020202020A0A080831
:100D6000040404040101010101010101030303035F
:100D700003030303040707070C0C0C0C0C0C0C0CEE
:100D80000202020206060606060606060B0B0B0BFF
:100D90000B0B0B0B417070656E64206D6561732EDB
:100DA000200053696E676C65206D6561732E2000AD
:100DB00053617665206D65617375726520746F3A55
:100DC0000020202020202020202020202020202043
:100DD00020000000010001001010020001000100CD
:100DE000B000000016000000280000001000000005
:100DF00020000000010001000000000000000000D1
:100E000000000000000000000000000000000000E2
:100E100000000000FF000000FFFF0000FFFF0000D7
:100E2000FFFF0000CFBF0000C7BF0000C3BF00002E
:100E3000C1BF0000C0BF000000000000C0BF000034
:100E4000C1BF0000C3BF0000C7BF0000CFBF00008C
:100E5000FFFF0000FFFF0000000000000000000096
:100E60000000000000000000000000000000000082
:100E70000000000000000000000000000000000072
:100E80000000000000000000000000000000000062
:100E90000000000000000000557365722D61676559
:100EA0006E743A202A0D0A446973616C6C6F773A4C
:100EB000202F0D0A000079961D9611241FBECFEF3A
:100EC000D1E2DEBFCDBF00E00CBF19E0A0E0B2E090
:100ED000E0E4F3E601E00BBF02C007900D92AE3CE8
:100EE000B107D9F725E1AEECB9E001C01D92A135FB
:100EF000B207E1F717E0CCE5D7E000E006C02197A4
:100F00000109802FFE010E94A7AECB35D10780E0FA
:100F10000807A9F70E9430990C948EB10C94000038
:100F20008EBD0DB407FEFDCF0895DC015996ED91FD
:100F3000FC913097B9F083899489A589B689428557
:100F4000538564857585841B950BA60BB70B81159E
:100F500020E89207A105B10538F08FEF9FE7A0E0E8
:100F6000B0E0089590E080E00895CF93DF931F9262
:100F7000CDB7DEB76983DC01ED91FC910280F3818E
:100F8000E02D41E050E0BE016F5F7F4F19950F905B
:100F9000DF91CF910895FC0120812EBD9B0121504E
:100FA000310941F051810DB407FEFDCF4EB55EBD54
:100FB0004193F5CF61507109860F971F0DB407FE5D
:100FC000FDCF2EB5FC0120830895E091480CF091EF
:100FD000490C90818091470C8095892380830895E6
:100FE0008EBD00000DB407FEFDCF8EB5089590E0D4
:100FF00020914A0C233339F40C96982F990F990FAE
:10100000990F80E008954896F8CFCF93DF931F9211
:10101000CDB7DEB76983DC01ED91FC910280F381ED
:10102000E02D41E050E0BE016F5F7F4F19950F90BA
:10103000DF91CF910895FC01818D928D0895CF931A
:10104000DF931F92CDB7DEB76983DC01ED91FC9190
:101050000280F381E02D41E050E0BE016F5F7F4FE1
:1010600019950F90DF91CF910895FC019485FB01B4
:101070008485981303C081E0983008F080E00895DB
:10108000CF93DF931F92CDB7DEB76983DC01ED917B
:10109000FC910280F381E02D41E050E0BE016F5FE2
:1010A0007F4F19950F90DF91CF910895FC017687BE
:1010B00065870895DC01ED91FC91068CF78DE02D9C
:1010C000199591E089270895862F089581E0862754
:1010D000089521E0FC018485883008F020E0822F0B
:1010E0000895FC01848595850895FC01848995897E
:1010F000089522E134E0FC0131832083FB01408923
:10110000518962897389FC014283538364837583A7
:101110000895DC01ED91FC91048CF58DE02D19947E
:1011200090E080E00895FC01818D928D009711F090
:101130000C948A8C089561E0FC0184810C94877E74
:10114000CF93DF93EC018FEF8EBD2FEF8F819885CA
:10115000AC014F5F5F4F58874F838130924028F436
:101160000DB407FEFDCF2EBDF1CF0DB407FEFDCFB0
:10117000CE010E949B081E82DF91CF910895CF93EC
:10118000DF93EC01E98DFA8D309749F481E090E02E
:101190009B838A8390E080E0DF91CF910895138252
:1011A0001282898D9A8D0E94598DE98DFA8D228146
:1011B0003381232B59F7F0CFCF92DF92EF92FF923A
:1011C0000F931F93CF93DF93CDB7DEB7AF970FB6D3
:1011D000F894DEBF0FBECDBF7C016A0102E114E0CE
:1011E0001A8309831C861B8688EE93E0A0E0B0E09A
:1011F0008D879E87AF87B88B8CE993E09A87898724
:10120000188F0F8B198E1A8E1B8E1C8E88E089A367
:101210001BA70AA71CA61DA61EA61FA68091190E15
:1012200090911A0EA0911B0EB0911C0E8EA39FA33D
:10123000A8A7B9A78B839C83AD83BE8318861F8222
:10124000AE01465D5F4FCE0101960E94E082813083
:101250009105B1F4D701ED91FC910488F589E02D59
:101260001DA30CA38CA59DA5AEA5BFA58EA39FA372
:10127000A8A7B9A7A601BE016C5D7F4FC70119954C
:10128000AF960FB6F894DEBF0FBECDBFDF91CF9102
:101290001F910F91FF90EF90DF90CF9008959F9254
:1012A000AF92BF92CF92DF92EF92FF920F931F9374
:1012B000CF93DF935C017B018B01D0E0C0E0F801AC
:1012C00091908F016501CC0EDD1EC6010E94EBAC32
:1012D000981621F0692DC6010E94F3AC2196C23305
:1012E000F1E0DF0761F7C701DF91CF911F910F9107
:1012F000FF90EF90DF90CF90BF90AF909F900895B8
:10130000FF920F931F93CF93DF93F82ECAEADBE08F
:101310008E0161E0D80112968C910E94EA7E609164
:10132000690BF80182810E94877E64EF71E080E0A2
:1013300090E00E94407F0E5F1F4FFBE0003B1F07C5
:1013400041F7FF2009F447C060916B0B8A810E942E
:10135000877E68EE73E080E090E00E94407F6091BD
:101360006B0B8C810E94877E68EE73E080E090E0DA
:101370000E94407F6091690B8A810E94877E68EE9F
:1013800073E080E090E00E94407F22968BE0CE3AAE
:10139000D807D1F668EE73E080E090E00E94407FCD
:1013A000C1EDD2E00CEA1BE0E991F991D8018C91F2
:1013B0000E5F1F4FEE0FFF1FE759F44F60810E9431
:1013C000877E68EC70E080E090E00E94407FB2E0B1
:1013D000C73DDB0749F7DF91CF911F910F91FF9038
:1013E000089581E08093EF028091F002882341F01C
:1013F00088E08093491160E08EE391E10C941E89AE
:1014000008958091F0028823F9F08091EF028823FB
:10141000D9F081E00E944B898BE39FE10197F1F7BE
:1014200060E080E00E945C8967E675E08EE391E110
:101430000E94977D61E080E00E945C8967E575E02D
:101440008EE391E10C94977D08950F931F93CF93B2
:10145000DF932091F002222309F45CC02091EF0277
:10146000222309F457C0EA018C016F3F7F4FF1F44A
:1014700061E080E00E945C89B8018EE391E10E9406
:10148000757D66E475E08EE391E10E94977D61E0F1
:10149000F80184810E945C89BE01DD0F880B990BE5
:1014A000DF91CF911F910F910C94407F0E940F828A
:1014B000AB01BC0180919B0A90919C0AA0919D0A6E
:1014C000B0919E0A8C599F4FAF4FBF4F841795071D
:1014D000A607B707F8F461E080E00E945C89B801D4
:1014E0008EE391E10E94757D65E375E08EE391E105
:1014F0000E94977D61E0F80184810E945C890E94CE
:101500000F8260939B0A70939C0A80939D0A90932C
:101510009E0AC2CFDF91CF911F910F910895CF9373
:10152000DF93EC010E948A8C882311F01D8281E0F8
:10153000DF91CF9108953F924F925F926F927F9289
:101540008F929F92AF92BF92CF92DF92EF92FF92D3
:101550000F931F93CF93DF93CDB7DEB72C970FB6C2
:10156000F894DEBF0FBECDBF5C01DC015B968D90B1
:101570009C905C9716964D905D906D907C9019971D
:10158000411451046104710409F468C0BFEF4B1A9F
:101590005B0A6B0A7B0A312CF40181859285A38555
:1015A000B4859C01AD012F5F3F4F4F4F5F4F29879F
:1015B0003A874B875C87730162011D821E821F82FE
:1015C0001886F40181859285A385B4852D813E819D
:1015D0004F815885281739074A075B0708F056C01E
:1015E00089859A85AB85BC858C159D05AE05BF05A3
:1015F00050F482E0C82ED12CE12CF12C92E0492E3F
:10160000512C612C712C9E012F5F3F4FB701A60119
:10161000C4010E949E8B8823C9F189819A81AB8184
:10162000BC81892B8A2B8B2B09F1260137019FEF77
:10163000491A590A690A790A2D813E814F815885D4
:101640002F5F3F4F4F4F5F4F2D833E834F83588710
:101650003FEFC31AD30AE30AF30AB3CFF401408081
:101660005180628073803324339496CFC414D504A0
:10167000E604F70409F70FEF1FEF2FEF3FE0B70184
:10168000A601C4010E94FC8A811119C080E02C9639
:101690000FB6F894DEBF0FBECDBFDF91CF911F9183
:1016A0000F91FF90EF90DF90CF90BF90AF909F9001
:1016B0008F907F906F905F904F903F900895F501CD
:1016C0004681578160857185411551056105710518
:1016D00039F097018601C4010E94FC8A8823B1F287
:1016E000D5011696CD92DD92ED92FC92199733209A
:1016F00051F0D701C6010196A11DB11DF4018083EF
:101700009183A283B383F5018789908DA18DB28DDA
:10171000892B8A2B8B2B39F4C78AD08EE18EF28EDF
:1017200084818068848381E0B2CF8FEF0E9490072C
:101730008EB508958F929F92AF92BF92FF920F93B2
:101740001F93CF93DF93EC01F62E49015A018E814E
:10175000882319F0CE010E94A00860E08C810E94CD
:10176000877E8CE291E00E94C5828F2D80640E946A
:10177000900708E110E0D501C401002E04C0B69521
:10178000A795979587950A94D2F70E9490070850DD
:101790001109083F8FEF180771F785E9FF2021F045
:1017A00088E0F8120DC087E80E94900710E00E94C0
:1017B000950B8A8787FF06C01F3F21F01F5FF7CF79
:1017C0008FEFF2CFDF91CF911F910F91FF90BF90DC
:1017D000AF909F908F900895AF92BF92CF92DF927B
:1017E000EF92FF920F931F93CF93DF93EC01690168
:1017F000C801820F931F8130924050F58E8188235B
:1018000079F088819981AA81BB8184179507A60701
:10181000B70731F48F819885C816D90608F042C001
:10182000488359836A837B838B85833039F089E0D1
:10183000440F551F661F771F8A95D1F79A01AB0198
:1018400061E1CE010E949A0B882389F083E08D83A9
:10185000CE010E949B0880E0DF91CF911F910F91F4
:10186000FF90EF90DF90CF90BF90AF9008950E94CF
:101870000F825B010E94950B8A878F3F69F40E945B
:101880000F826A197B096D327140A0F38FE08D835E
:10189000CE010E949B08DCCF8E3FB1F418861F82D8
:1018A00081E08E838FEF8EBD2FEF8F8198858C1511
:1018B0009D0560F40DB407FEFDCF2EBD8F81988588
:1018C000019698878F83F1CF8DE0E1CFC801019712
:1018D000F7012FEFAF014E195F094817590738F488
:1018E0000DB407FEFDCF3EB531932EBDF3CF0DB441
:1018F00007FEFDCF2EB5E80EF91EF70120838F817C
:101900009885080F191F18870F838985882319F078
:101910000115124030F08E81882319F0CE010E940B
:10192000A00881E099CF0F931F93CF93DF93EC0131
:10193000890182E1411551056105710599F08B8599
:10194000833039F089E0440F551F661F771F8A9551
:10195000D1F79A01AB0168E1CE010E949A0B88236E
:1019600019F084E08D8338C08EEF8EBDF801C80178
:101970009E5F0DB407FEFDCF20812EBD0DB407FE86
:10198000FDCF21812EBD3296E817F90791F70DB4EE
:1019900007FEFDCF8FEF0E9490078FEF0E94900708
:1019A0000E94950B8A878F71853089F488E592E0D3
:1019B0000E94C5828823A9F020E030E0A9016DE0F3
:1019C000CE010E949A0B882371F084E1CBCF81E194
:1019D0008D83CE010E949B08CE010E949B0880E06F
:1019E0000AC085E1BFCF0E94950B8111EECFCE01D9
:1019F0000E949B0881E0DF91CF911F910F91089584
:101A0000FC01DB0112968D919C9113979383828345
:101A100084E793E09183808314968C911497848358
:101A200015968C911597858316964D915D916D91C4
:101A30007C91199746835783608771871A964D91D9
:101A40005D916D917C911D9742875387648775875F
:101A50001E964D915D916D917C9151974687578768
:101A6000608B718B52968C915297828B53964D91CD
:101A70005D916D917C915697438B548B658B768BE2
:101A800057964D915D916D917C915A97478B508FF0
:101A9000618F728F5B968D919C91948F838F089547
:101AA000DC015996ED91FC91309721F081E0958110
:101AB000911101C080E00895CF93DF93EC01898DEF
:101AC0009A8D009741F00E948F0A898D9A8D0E940D
:101AD00066AF1A8E198EDF91CF910895EF92FF9223
:101AE0000F931F93CF93DF93EC017B018A011B823D
:101AF0001A8288EE93E0A0E0B0E08C839D83AE83F1
:101B0000BF8384EF93E0998388838DE190E00E9406
:101B1000CAAE9A8F898F009779F02DE1F701DC0129
:101B200001900D922A95E1F74CE050E0B801CE010A
:101B30000C960E9435B1188EDF91CF911F910F91B5
:101B4000FF90EF900895CF93DF931F92CDB7DEB74C
:101B500041E050E0BE016F5F7F4F0E94658F0197AB
:101B600031F4898190E00F90DF91CF9108958FEF4C
:101B70009FEFF9CFFC01818D928D009711F00C94AD
:101B8000A30D8FEF9FEF08950F931F93CF93DF93D4
:101B9000EC01898D9A8D10E000E0009799F00E9489
:101BA000A30D8C010F3F100769F0898D9A8DFC0100
:101BB00042855385648575854150510961097109D4
:101BC0000E94C58CC801DF91CF911F910F9108959C
:101BD000E091480CF091490C80819091470C892B41
:101BE00080830895AF92BF92CF92DF92EF92FF92DF
:101BF0000F931F93CF93DF9300D01F92CDB7DEB723
:101C00008C016B017A0180914A0C8333E9F45B010A
:101C10006801C40ED51EC016D106A9F10E94E507C1
:101C20008FE00E94F007812F0E94F007802F0E9412
:101C3000F0070F5F1F4F80E00E94F007F5018193CE
:101C40005F010E94E80DE7CF843369F50E94E50744
:101C500019830A838F2D8F778B83EC8264E070E089
:101C6000CE0101960E94CB07A70170E060E0C6019B
:101C70000E9405B1E114F10421F0B701C6010E94F0
:101C8000CB070E94E80DC7010F900F900F900F90A7
:101C9000DF91CF911F910F91FF90EF90DF90CF9048
:101CA000BF90AF9008950E94E5070F3F110509F01E
:101CB00030F419820A831B8263E070E0D1CF17FDF4
:101CC0000BC019820A8333E0169507953A95E1F720
:101CD000007E08600B83F0CFC80126E096958795BB
:101CE0002A95E1F7807E19830A830115104C18F4B8
:101CF00080618B83E1CF8861FCCFCF93DF931F920C
:101D0000CDB7DEB720914B0C30E0322F2227260FC3
:101D1000371F90E0982F882741E050E0BE016F5FA9
:101D20007F4F820F931F0E94F20D89810F90DF91E8
:101D3000CF910895AF92BF92CF92DF92EF92FF9230
:101D40000F931F93CF93DF9300D000D01F921F9269
:101D5000CDB7DEB78C017B016A0180914A0C8333D9
:101D6000E1F45801A40EB51EA016B10609F46FC027
:101D70000E94E50780EF0E94F007812F0E94F00784
:101D8000802F0E94F0070F5F1F4FF70181917F01A5
:101D90000E94F0070E94E80DE7CF5B01A40EB51E7C
:101DA0008433C1F40E94E50719830A838D2D80686E
:101DB0008B83CC8264E070E0CE0101960E94CB0759
:101DC000AE14BF0409F441C0F70181917F010E9464
:101DD000F007F6CF0E94E5070F3F110509F028F440
:101DE00019820A8384E08B830CC017FD17C0198207
:101DF0000A8333E0169507953A95E1F7007E0C606B
:101E00000B8386E0C816D104A0F5F701DE01149615
:101E1000EA15FB0599F081918D93FACFC80126E070
:101E2000969587952A95E1F7807E19830A83011597
:101E3000104C10F48461D7CF8C61D5CFB6016D5FA3
:101E40007F4FCE0101960E94CB070E94E80DC6018C
:101E500028960FB6F894DEBF0FBECDBFDF91CF91AD
:101E60001F910F91FF90EF90DF90CF90BF90AF90B8
:101E7000089563E070E0CE0101960E94CB07F70160
:101E800081917F010E94F007AE14BF04C1F7DDCF3E
:101E9000CF93DF931F92CDB7DEB741E050E0BE0194
:101EA0006F5F7F4F90E080E00E94F20D89810F907C
:101EB000DF91CF910895CF93DF93C4E1D0E00E94EA
:101EC000480F882361F061E070E080E090E00E94BC
:101ED000407F2197A1F780E0DF91CF91089581E0C5
:101EE000FBCFCF93DF931F92CDB7DEB7898341E05D
:101EF00050E0BE016F5F7F4F90E080E00E949A0E3D
:101F00000F90DF91CF91089563E070E00C947D0E07
:101F1000DA01E0914B0CF0E0FE2FEE27E60FF71F01
:101F200090E0982F8827A901BD018E0F9F1F0C9468
:101F30009A0ECF93DF931F921F92CDB7DEB77983AE
:101F40006A8322E030E0AE014F5F5F4F60E170E0F6
:101F50000E94880F0F900F90DF91CF910895CF933B
:101F6000DF931F921F92CDB7DEB779836A8322E099
:101F700030E0AE014F5F5F4F64E070E00E94880F79
:101F80000F900F90DF91CF910895CF93DF931F9221
:101F9000CDB7DEB720914B0C30E0322F2227260F31
:101FA000371F90E0982F8827498341E050E0BE0119
:101FB0006F5F7F4F820F931F0E949A0E0F90DF91E9
:101FC000CF910895CF93C82F462F61E070E00E9413
:101FD000C50F61E070E08C2F0E947D0E8111F9CF5A
:101FE000CF910895DA01E0914B0CF0E0FE2FEE273F
:101FF000E60FF71F90E0982F8827A901BD018E0FEB
:102000009F1F0C94F20D6F927F929F92AF92BF929E
:10201000CF92DF92EF92FF920F931F93CF93DF93B4
:102020001F921F92CDB7DEB7982E8B013A0169013E
:1020300022E030E0AE014F5F5F4F64E270E00E944B
:10204000F20FE980FA80FE24EF24FE24E00EF11E58
:102050009701377040914A0C092D10E0C8014333B5
:1020600009F04CC00896982F8827990F990F990F5F
:10207000820F931F473309F446C0A9014C0D5D1D23
:102080004130584008F43FC060E078E05B01A21A9C
:10209000B30AA501B3010E949A0EA6014A195B0971
:1020A000B3016A0D7B1D80914A0C833349F5085FAB
:1020B0001F4F000F000F000F80E0902F0E949A0E1C
:1020C000EC0CFD1CF982EA8222E030E0AE014F5FA9
:1020D0005F4F64E270E0892D0E94880F0F900F908F
:1020E000DF91CF911F910F91FF90EF90DF90CF90F4
:1020F000BF90AF909F907F906F9008954096B3CF20
:10210000005F1F4FD6CFA601B301D8CFEF92FF9249
:102110001F93CF93DF931F921F92CDB7DEB7182F77
:1021200022E030E0AE014F5F5F4F60E270E00E945E
:10213000F20FE980FA80FE24EF24FE2422E030E052
:10214000AE014F5F5F4F60E270E0812F0E94F20F9F
:1021500089819A81982789279827E816F90689F4B2
:1021600087E0189FF0011124E350F44FF582E482D8
:10217000C7010F900F90DF91CF911F91FF90EF90CB
:1021800008957C01DBCFFF920F931F93CF93DF93D2
:102190001F921F92CDB7DEB7F82E22E030E0AE01DD
:1021A0004F5F5F4F66E270E00E94F20F09811A8173
:1021B00010270127102722E030E0AE014F5F5F4F6C
:1021C00066E270E08F2D0E94F20F89819A81982734
:1021D000892798270817190749F4C8010F900F900D
:1021E000DF91CF911F910F91FF9008958C01E3CF64
:1021F00044E050E0BC018FE090E00C949A0E08950A
:102200001F93CF93DF93182F80E591E00E943176E2
:10221000812F0E948610EC01812F0E94840F87314C
:1022200021F08C3111F0D0E0C0E0CE01DF91CF91F0
:102230001F910895FC018485883010F40C940011DE
:1022400090E080E00895CF92DF92EF92FF921F938B
:10225000CF93DF93182F7B01EA014130584010F0F3
:10226000C0E0D8E080E591E00E943176812F0E94A5
:1022700086106C01812F0E94840F873111F08C3100
:1022800021F5CC16DD0670F380E591E00E943176F1
:102290009E01A70170E060E0812F0E94031060E2C0
:1022A00070E0812F0E94E20F62E070E0812F0E94B7
:1022B0007D0E84FD0DC0812F0E94840F8823B9F00C
:1022C00080E591E00E943176EFCFD0E0C0E0DCCF36
:1022D00040E162E070E0812F0E94C50FCE01DF91E6
:1022E000CF911F91FF90EF90DF90CF900895D0E0B5
:1022F000C0E0F4CF0F931F93CF93DF938C01EA01DB
:10230000FC018485883048F40E942311892B39F41C
:1023100081E090E0F80193838283D0E0C0E0CE01B9
:10232000DF91CF911F910F910895CF92DF92EF929D
:10233000FF920F931F93CF93DF938B017A016C0170
:1023400029EBC20ED11CF6014081EC012A964423F0
:1023500049F050E0BC0167567F4FCE010E947A11D0
:10236000F6011082A701B801CE01DF91CF911F9134
:102370000F91FF90EF90DF90CF900C947A11CF9354
:10238000DF93EC01C754DF4FE88121E02E0F288353
:10239000E80FF92FF11DE756FF4F6083203249F413
:1023A000BC0167567F4F40E250E00A960E947A11C6
:1023B000188281E090E0DF91CF9108951F93CF9331
:1023C000DF931F92CDB7DEB7182F80E591E00E9412
:1023D0003176812F0E94F70727E0129FF001112428
:1023E000E350F44F22813381377041E050E0BE0169
:1023F0006F5F7F4F820F931F0E94F20D89810F90B4
:10240000DF91CF911F910895FC01808D883040F4B9
:10241000218D328D232B21F00E94DE1190E0089552
:102420008FEF9FEF0895CF93DF93FC012485283031
:1024300028F08FEF9FEFDF91CF910895EC0101908D
:10244000F081E02D0084F185E02D1995892B89F329
:102450008C850E94DE1190E0EECF1F93CF93DF9327
:10246000182F87E0189FE0011124C350D44F8881B2
:102470009981009761F480E591E00E943176812F87
:102480000E94C3102E81821B910999838883DF915A
:10249000CF911F910895FC018485883010F40C942D
:1024A0002D1290E080E008954F925F927F928F927C
:1024B0009F92AF92BF92CF92DF92EF92FF920F93D3
:1024C0001F93CF93DF931F921F92CDB7DEB7782E65
:1024D0006B014A01A82EB12C27E0829FC001112474
:1024E000FC01E350F44F7F010081118180E591E010
:1024F0000E9431760815190554F4872D0E94C310E7
:10250000F70126818C01021B11091183008301153B
:10251000110519F5872D0E94840F843159F0882305
:1025200049F001E010E08C3111F410E000E0119569
:1025300001951109C8010F900F90DF91CF911F9164
:102540000F91FF90EF90DF90CF90BF90AF909F9052
:102550008F907F905F904F900895801691060CF4B5
:10256000840187E08A9DF0018B9DF00D1124E350DA
:10257000F44FE280F380C114D10451F12701F7E058
:102580005F22872D0E94F707840D951D20914A0C2C
:10259000273309F453C09801240D351D21303840EC
:1025A00008F44CC020E038E0490184189508A401E3
:1025B000B6010E94F20D2601480C591C6801C8188A
:1025C000D908872D0E94F707A601B2010E94F20DDB
:1025D000E00EF11E87E08A9DF0018B9DF00D112425
:1025E000E350F44FF382E28220813181201B310BD2
:1025F000318320838681800F912F911D8A3F910521
:1026000010F4232BF1F487E08A9DF0018B9DF00DEF
:102610001124E350F44F1682F982EA8222E030E07E
:10262000AE014F5F5F4F68E270E0872D0E94880F18
:1026300060E470E0872D0E94E20F7CCFA801B60114
:10264000C5CF868377CFCF93DF93FC01218D328D69
:102650002115310529F48FEF9FEFDF91CF91089578
:10266000EC01808D4217530708F0A9010E94541213
:102670001816190684F7298D3A8D281B390B3A8FC5
:10268000298FEBCF0F931F93CF93DF931F92CDB77B
:10269000DEB7FC01218D328D232B41F48FEF9FEFAC
:1026A0000F90DF91CF911F910F9108958C0141E020
:1026B00050E0BE016F5F7F4FFC01808D0E9454127D
:1026C000181619065CF7F801818D928D0197928F8B
:1026D000818F898190E0E4CF0F931F93CF93DF9395
:1026E00000D000D01F921F92CDB7DEB78C01D80169
:1026F00059964D915C915A974115510551F0ED91C4
:10270000FC91048CF58DE02D70E060E0C801199516
:10271000EECFF801808D0E942D12892BB1F148E097
:1027200050E0BE016F5F7F4FD80158968C910E9498
:10273000541218161906F4F4D801509684E0FE01DC
:10274000319601900D928A95E1F78D8190E0982F56
:1027500088272E81820F911DF801958B848B8F81A4
:10276000282F30E0322F22278885820F932F911D4A
:10277000928F818F28960FB6F894DEBF0FBECDBF23
:10278000DF91CF911F910F91089590E080E0F2CFFB
:10279000CF93DF931F92CDB7DEB741E050E0BE018B
:1027A0006F5F7F4FFC0184850E9454121816190632
:1027B00034F4898190E00F90DF91CF9108958FEFED
:1027C0009FEFF9CFFC018485883010F40C945412EB
:1027D00090E080E00895CF93C82F80E591E00E94BB
:1027E000317668E070E08C2FCF910C94E20FCF939C
:1027F000C82F80E591E00E94317660E170E08C2F77
:10280000CF910C94E20FCF92DF92EF92FF920F9351
:102810001F93CF93DF9300D000D0CDB7DEB78C01EC
:102820006B017A01FC01808D883010F40E94F7134F
:1028300082E194E09A838983F60182819381A48165
:10284000B5818B839C83AD83BE83B701CE01019696
:102850000E94B178F801808F8830A0F4F586E48674
:10286000128E118E81E026960FB6F894DEBF0FBE51
:10287000CDBFDF91CF911F910F91FF90EF90DF902F
:10288000CF90089580E0EFCFCF93DF93EC01888D58
:10289000883020F40E94F71388E0888FDF91CF9171
:1028A0000895CF93C82F80E591E00E9431768C2F58
:1028B000CF910C94840FEF92FF920F931F93CF93BD
:1028C000DF937C0180914A0CD4E0833309F0D8E097
:1028D00005E31CE0C0E0F801219131918F01F7017F
:1028E000848195812817390729F0CF5FDC13F3CF56
:1028F00080E006C08C2F0E9451148431B1F781E032
:10290000DF91CF911F910F91FF90EF9008959F92CB
:10291000AF92BF92CF92DF92EF92FF920F931F93ED
:10292000CF93DF93EC017B0180914A0C811121C090
:102930001B821A8288EE93E0A0E0B0E08C839D8336
:10294000AE83BF8386EC93E09983888388E08C878D
:1029500088EE93E09E878D87CE01DF91CF911F9106
:102960000F91FF90EF90DF90CF90BF90AF909F902E
:10297000089534E0932E833311F028E0922E85E3FE
:10298000C82E8CE0D82E10E098E0B92EA12CD601EC
:102990002D913D916D01F7018481958128173907AB
:1029A00091F4812F0E945114082F873111F08C313E
:1029B00039F5812F0E942D12892B59F50C3119F40C
:1029C000812F0E94EB131F5F9112E1CFA11008C06D
:1029D000D701ED91FC910084F185E02DC701199597
:1029E0001B821A8288EE93E0A0E0B0E08C839D8386
:1029F000AE83BF8386EC93E099838883BC86A8CF9F
:102A0000843149F08111DFCFF601329711821082B3
:102A1000DACFB12ED8CFAA24A394D5CF8F929F928C
:102A2000AF92BF92CF92DF92EF92FF920F931F93DC
:102A3000CF93DF93CDB7DEB72F970FB6F894DEBFF5
:102A40000FBECDBF5C014B017A0180914A0C8823F7
:102A5000C9F104E0833309F008E0B501CE01019625
:102A60000E94871485E3C82E8CE0D82E10E0F60172
:102A7000219131916F01F5018481958128173907E2
:102A800051F4812F0E945114873129F4A701B40118
:102A9000812F0E9423111F5F0113E9CFC7012F96D9
:102AA0000FB6F894DEBF0FBECDBFDF91CF911F915F
:102AB0000F91FF90EF90DF90CF90BF90AF909F90DD
:102AC0008F900895F12CE12CE9CFCF93DF93EC01A7
:102AD0008C858830D0F40E945114843189F0882389
:102AE00079F0883169F021E08C3159F4E881F9817D
:102AF0000084F185E02DCE01199521E0892B09F4A0
:102B000020E0822FDF91CF91089580E0FBCFCF921C
:102B1000DF92EF92FF92CF93DF93EC018C858830A8
:102B200068F40E94EB130E940F826B017C018C857C
:102B30000E945114811109C088E08C87DF91CF91E8
:102B4000FF90EF90DF90CF90089561E070E080E01B
:102B500090E00E94407F0E940F82AB01BC014C19A3
:102B60005D096E097F098D859E85B0E0A0E048175C
:102B700059076A077B07D8F28C850E94F713DCCFD0
:102B8000CF93DF93EC018C85883060F40E94511460
:102B9000873111F08C3131F48C850E940011811540
:102BA000984088F3DF91CF910895CF92DF92EF9212
:102BB000FF920F931F93CF93DF93CDB7DEB7AF97FD
:102BC0000FB6F894DEBF0FBECDBF8C016B017A014A
:102BD00082E194E09A8389831B821C821D821E827B
:102BE0001C861B8648EE53E060E070E04D875E87F0
:102BF0006F87788B2CE933E03A872987988F8F8B02
:102C0000198E1A8E1B8E1C8E28E029A39BA78AA7DB
:102C10001CA61DA61EA61FA6D8011C968C91883046
:102C200060F40E945114882321F0F80184850E94E9
:102C3000EB1388E0D8011C968C938091190E90912B
:102C40001A0EA0911B0EB0911C0E8EA39FA3A8A7D5
:102C5000B9A78B839C83AD83BE8318861F82AE0188
:102C6000465D5F4FB601CE0101960E94E08200975B
:102C7000C1F0D801ED91FC910684F785E02D82E149
:102C800094E09DA38CA38CA59DA5AEA5BFA58EA306
:102C90009FA3A8A7B9A7A701BE016C5D7F4FC8017C
:102CA0001995AF960FB6F894DEBF0FBECDBFDF917A
:102CB000CF911F910F91FF90EF90DF90CF900895EB
:102CC0008F929F92AF92BF92CF92DF92EF92FF923C
:102CD0000F931F93CF93DF9300D000D000D01F92AB
:102CE000CDB7DEB790914A0C911115C018E0812F35
:102CF0002A960FB6F894DEBF0FBECDBFDF91CF91FD
:102D00001F910F91FF90EF90DF90CF90BF90AF9009
:102D10009F908F90089528E0F22E933311F494E061
:102D2000F92E6B01082F80E591E00E9431769E011B
:102D30002F5F3F4F5901490110E0812F0E94840FFE
:102D4000F40181934F018823C1F01F5FF112F5CF89
:102D5000F12CF50191915F019D3149F0983139F0E5
:102D60009A51923020F0F3941F11F3CFBFCF60E15E
:102D700070E08F2D0E94E20F1F2DE12EF12CF70144
:102D8000EE0FFF1FEB5CF34F1182108283EE93E096
:102D90000197F1F7402F70E060E0812F0E94C50F8E
:102DA0004FEF62E070E0812F0E94C50FB601CD2881
:102DB00089F4809190029091910201968115F0EC36
:102DC0009F0798F1909391028093900260919002F6
:102DD00070919102812F0E94AF0F61E070E0812F0E
:102DE0000E94E20F27E02E9DC0012F9D900D11241F
:102DF0009C012350344F7901F9011182108222E0A5
:102E000030E0AE01475F5F4F68E270E0812F0E94C3
:102E1000F20F89859A85982789279827F701938348
:102E2000828316821582148262CF80E090ECCACF32
:102E30000F931F93CF93DF93EC018B01888D883024
:102E400010F40E94F713B80182E00E946016888F88
:102E5000883050F41D870C871A8E198E81E0DF911F
:102E6000CF911F910F91089580E0F9CF9F92AF927B
:102E7000BF92CF92DF92EF92FF920F931F93CF9367
:102E8000DF938C015B01942EE52EFC01C688D78868
:102E9000F08C80E591E00E9431768F2D0E948610A3
:102EA000C92DDE2D8C179D0708F4EC019E01A501AC
:102EB000B6018F2D0E940310F801868997898C0F27
:102EC0009D1F978B868BCE01DF91CF911F910F9124
:102ED000FF90EF90DF90CF90BF90AF909F900895BC
:102EE000CF93FC01C08D80E591E00E94317660E2D5
:102EF00070E08C2F0E94E20F62E070E08C2F0E9445
:102F00007D0E84FD16C062E070E08C2F0E947D0E65
:102F100083FF0AC048E162E070E08C2F0E94C50F79
:102F200080E090E0CF91089580E591E00E943176B5
:102F3000E3CF40E162E070E08C2F0E94C50F81E09A
:102F4000F0CFFF920F931F93CF93DF93EB01FC0120
:102F5000178A168A2A81211109C02B81211106C0E6
:102F60002C81211103C02D81222301F1411551052E
:102F7000E9F08A01FC01F08C80E591E00E94317655
:102F8000AE014E5F5F4F24E030E06CE070E08F2DCB
:102F90000E94880FB8018F2D0E94990F81E090E068
:102FA000DF91CF911F910F91FF90089580E0F7CFAF
:102FB0007F928F929F92AF92BF92CF92DF92EF92C9
:102FC000FF920F931F93CF93DF93CDB7DEB7A697F2
:102FD0000FB6F894DEBF0FBECDBF8C01762E942EB7
:102FE000852E20E2A22ECE0101967C01DC01EA2D85
:102FF0001D92EA95E9F76801F3E4CF0ED11C82E156
:1030000094E09AA389A38FEF8BA38CA38DA38EA3A7
:1030100043E450E0BE016F5D7F4FC6010E94A117DF
:10302000019609F4BFC081E089838A8386E0B82EC7
:10303000BB821C82D80114966D917D918D919C91DB
:1030400017970E94AFAE6D837E838F8398878986A2
:103050009A8680E890E09C878B874CE150E0B7012E
:10306000C6010E943617FE0137968AE1DF011D92E4
:103070008A95E9F74801B8E08B0E911CF401D7015D
:1030800001900D92BA94E1F740E150E0B701C6011A
:103090000E943617F7011192AA94E9F796E0A92E3B
:1030A000B12C40E250E0B701C6010E943617F1E0B2
:1030B000AF1AB108B1F783E6898392E89A8393E562
:1030C0009B838C8385E38D8381E08E837F829DE368
:1030D000988797E099878A8786E0F401DE011B963E
:1030E00001900D928A95E1F78CE0898B8A8B64E1DF
:1030F00074E0CE0143960E9420B1D8011B966C91DA
:10310000CE0149960E947677F8016485CE014B96F0
:103110000E947677D8011D966C91CE014D960E9443
:1031200076774EE150E0B701C6010E943617B3E052
:103130007B121EC082E3898384E08A83F80196852E
:103140009B8397859C8390899D8391899E8396E339
:103150009F838887828D8987838D8A87848D8B87DB
:10316000858D8C874CE050E0B701C6010E94361770
:1031700087E3898386E08A8391E09B8393E09C8345
:103180008D838FE08E838AE38F838BE388878FEF35
:10319000898749E050E0B701C6010E943617C60191
:1031A0000E947017A6960FB6F894DEBF0FBECDBF73
:1031B000DF91CF911F910F91FF90EF90DF90CF9013
:1031C000BF90AF909F908F907F9008950F931F9323
:1031D000CF938C01FC016481758181E20E946016AD
:1031E000C82F8830F8F480E591E00E9431768C2F6A
:1031F0000E94840F833131F08C2FCF911F910F915A
:103200000C94EB1362E070E08C2F0E94E20FF80147
:1032100084819581EC2FF0E0EE0FFF1FEB5CF34F04
:1032200091838083CF911F910F9108950F931F93E6
:10323000CF93DF931F921F92CDB7DEB7FC01248599
:103240002830E0F48C0180E591E00E94317622E0A4
:1032500030E0AE014F5F5F4F60E170E0F8018485C0
:103260000E94F20F89819A819827892798270F90C9
:103270000F90DF91CF911F910F91089590E080E022
:10328000F6CF0F931F93CF93DF931F921F92CDB76B
:10329000DEB7FC0124852830E0F48C0180E591E064
:1032A0000E94317622E030E0AE014F5F5F4F64E074
:1032B00070E0F80184850E94F20F89819A81982735
:1032C000892798270F900F90DF91CF911F910F9131
:1032D000089590E080E0F6CFCF92DF92EF92FF92D8
:1032E0001F93CF93DF93EC017B016A018C858830BB
:1032F00048F40E945114882319F08C850E94EB1326
:1033000088E08C87F70182819381A481B581009741
:10331000A105B10551F490E080E0DF91CF911F91BC
:10332000FF90EF90DF90CF9008958F3F9F4FAF4F6A
:10333000BF4F89F370E060E081E20E946016182FB1
:103340008C87883040F780E591E00E943176A701B4
:103350004E5F5F4F24E030E06CE070E0812F0E9410
:10336000880FB601812F0E94990F64E070E0812FD1
:103370000E94E20F0E940F826B017C018C850E94EB
:103380005114873111F18C3101F1882321F20E940F
:103390000F82AB01BC014C195D096E097F098D8557
:1033A0009E85B0E0A0E084179507A607B70738F020
:1033B00061E070E080E090E00E94407FDFCF8C858C
:1033C0000E94F71388E08C87A6CF81E090E0A5CF1C
:1033D000CF93DF93EC0182E194E0998388831A8292
:1033E0001B821C821D8280E591E00E943176BE0125
:1033F0006E5F7F4F44E050E08FE090E00E94F20D5E
:10340000CE01DF91CF9108954F925F926F927F929C
:103410008F929F92AF92BF92CF92DF92EF92FF92E4
:103420000F931F93CF93DF93EC01181619061CF42A
:103430004C0104972CF0C1E0D0E063E0862E912C83
:103440008E01000F111F7E01EE0CFF1CEE0CFF1C05
:103450008C169D060CF4B3C097012C5B3D4F5901AF
:10346000F90180819181A281B381970121523D4F61
:103470006901181619061A061B063CF50E94AF854D
:10348000F601408051806280738064197509860955
:103490009709F50140805180628073804616570677
:1034A0006806790658F410821182128213820E94F3
:1034B000AF85F601608371838283938321960E5FCB
:1034C0001F4FF4E0EF0EF11CC3CF980129523D4F7E
:1034D0003901F90180819181980121533D4F5901B2
:1034E000F9012081318182179307C1F0880F991F5C
:1034F000FC01E759F44F6081F801E655F44F8081F3
:103500000E94877EF30180819181F5019183808300
:103510006CE271E080E090E00E94407FF6018081E3
:103520009181A281B381181619061A061B0634F67A
:103530000E94AF85F6012081318142815381621B57
:10354000730B840B950BF701E154FD4F2081318102
:1035500042815381261737074807590708F0AECF35
:10356000F601108211821282138298012C5A3D4F6B
:103570006901F90180819181F501208131818217F2
:10358000930709F49BCF880F991FFC01E759F44F6B
:103590006081F801E655F44F80810E94877EF60134
:1035A00080819181F50191838083F30191838083F0
:1035B0006CE271E080E090E00E94407F7FCFDF917D
:1035C000CF911F910F91FF90EF90DF90CF90BF9020
:1035D000AF909F908F907F906F905F904F900895E5
:1035E000CF93DF93FC0124813581232B69F0EC011B
:1035F000BC0185E29DE00E94837DBE0188E89CE0DD
:10360000DF91CF910C94837DDF91CF910895CF937B
:10361000DF93FC0124813581232B69F0EC01BC018F
:1036200085E29DE00E94757DBE0188E89CE0DF9107
:10363000CF910C94757DDF91CF9108958F929F92D9
:10364000AF92BF92CF92DF92EF92FF920F931F93B0
:10365000CF93DF938C01862F0B30110509F09FC0AB
:103660009091C710992309F0F89462E10E94737F4A
:10367000EC018091C710882309F07894209701F11C
:1036800080E090ECA9E7B4EC8093BA109093BB1063
:10369000A093BC10B093BD108093BE109093BF1048
:1036A000A093C010B093C110CE3F8FEFD80709F49C
:1036B000A9C0CF3FDC0709F462C0CCEFDFEF30C117
:1036C000C091C210E090C3106E2D70E090E080E0D9
:1036D0000E94CEAB2DEC3CEC4CEC5DE30E942DAC9B
:1036E0004B015C016C2F70E090E080E00E94CEAB5B
:1036F0009B01AC01C501B4010E9475AD6093BA1085
:103700007093BB108093BC109093BD10D091C410E7
:10371000F090C5106D2F6F7770E090E080E00E9410
:10372000CEAB4B015C016F2D70E090E080E00E9419
:10373000CEAB2DEC3CEC4CEC5DE30E942DAC9B0140
:10374000AC01C501B4010E9475ADD7FD26C06093E0
:10375000BE107093BF108093C0109093C110CE0D17
:10376000CD0FCF0D81E090E02091C610C21302C0B2
:1037700090E080E0892B09F493C0CFEFDFEFCE011A
:10378000DF91CF911F910F91FF90EF90DF90CF903D
:10379000BF90AF909F908F9008959058D8CFCFEF63
:1037A000DFEF0631110509F0BBC09091C7109923D6
:1037B00009F0F89461E00E94737FEC018091C710DA
:1037C000882309F07894209701F180E090ECA9E734
:1037D000B4EC8093BA109093BB10A093BC10B0933C
:1037E000BD108093BE109093BF10A093C010B093F3
:1037F000C110CF3FDC0719F2209709F451C022967F
:1038000009F05BCFCEEFDFEF8BC0C091C310D0913A
:10381000C2106091C2107091C31076276727762777
:1038200090E080E00E94CCAB2DEC3CEC4CEC5DE3F6
:103830000E942DAC6093BA107093BB108093BC10A3
:103840009093BD10E090C510F090C4106F2D6F776D
:10385000762F6E2D90E080E00E94CCAB2DEC3CECFE
:103860004CEC5DE30E942DACF7FC18C06093BE10D9
:103870007093BF108093C0109093C1108C2F8D0F48
:103880008E0D8F0DC1E0D0E09091C610891302C05B
:10389000D0E0C0E0D195C195D109ABCF9058E6CF2B
:1038A000C090BA10D090BB10E090BC10F090BD104A
:1038B00020E030E048EC52E4C701B6010E9489AE36
:1038C000D0E0C0E0181614F4CBEFDFEF20E030E0DA
:1038D000A901C701B6010E94C7AB87FF02C0CAEFAA
:1038E000DFEFC090BE10D090BF10E090C010F090FD
:1038F000C11020E030E048EC52ECC701B6010E9454
:10390000C7AB87FF02C0C9EFDFEF20E030E040EF38
:1039100052E4C701B6010E9489AE18160CF483C0A8
:103920000C30110509F02BCF81E08093830C8CE5DE
:103930008093850C1092840C1092860C60E082ECCF
:103940009DE00E94F57481E00E942E880E941B7FFA
:103950006B017C0180917D0C811168C081E08093B6
:103960007D0C80937C0C9FEF90937B0C10927A0CD3
:1039700094E09093790C8093580C8091580C886B4C
:103980008093580C8091570C813009F028C1109217
:10399000570C0E941B7F6B017C018091580C809317
:1039A000BB0080917F0C9091800CA091810CB09114
:1039B000820C892B8A2B8B2BA1F00E941B7F0091FC
:1039C0007F0C1091800C2091810C3091820C6C192D
:1039D0007D098E099F09061717072807390708F47C
:1039E00046C08091BC0083FDD8CF85EC8093BC009D
:1039F0000E941B7F6B017C0180917D0C813009F45A
:103A0000F0C080917A0C853008F00DC180917A0C5D
:103A1000A9E5BCE0E2EBFBE090E0981769F12D919D
:103A200021939F5FFACFC8EFDFEF7ACF80917F0CB1
:103A30009091800CA091810CB091820C892B8A2BE3
:103A40008B2B09F487CF0E941B7F00917F0C109174
:103A5000800C2091810C3091820C6C197D098E09AB
:103A60009F09061717072807390708F073CF8091B9
:103A70007E0C0E940D8880E01092460C8093450CCD
:103A8000082F10E0CEEFDFEF882309F478CECDEFDA
:103A9000DFEF053011050CF472CECEE8DAE082ECEF
:103AA0009DE00E94AE7488872196CE018E589A4080
:103AB00080179107A4F3C091960A0091970A602F8E
:103AC00070E090E080E00E94CEAB2DEC3CEC4CEC42
:103AD0005DE30E942DAC6B017C016C2F70E090E0E7
:103AE00080E00E94CEAB9B01AC01C701B6010E94F1
:103AF00075AD6B017C01C0928E0AD0928F0AE09264
:103B0000900AF092910AD091980A1091990A6D2F1B
:103B10006F7770E090E080E00E94CEAB4B015C01DB
:103B2000612F70E090E080E00E94CEAB2DEC3CEC89
:103B30004CEC5DE30E942DAC9B01AC01C501B401CE
:103B40000E9475ADD7FD71C06093920A7093930A7D
:103B50008093940A9093950AC00FCD0FC10F809166
:103B60009A0AC8130ACE20E030E048EC52E4C701BC
:103B7000B6010E9489AED0E0C0E0181614F4CBEF75
:103B8000DFEF20E030E040EA50E4C701B6010E94D8
:103B9000C7AB87FF02C0CAEFDFEFC090920AD09098
:103BA000930AE090940AF090950A20E030E040EF0C
:103BB00051ECC701B6010E94C7AB87FF02C0C9EF35
:103BC000DFEF20E030E040EF52E4C701B6010E9491
:103BD00089AE18160CF0D3CDC8EFDFEFD0CD85EE4F
:103BE00005CF80917F0C9091800CA091810CB091B9
:103BF000820C892B8A2B8B2B09F4FECE0E941B7F13
:103C000000917F0C1091800C2091810C3091820CDE
:103C10006C197D098E099F090617170728073907B0
:103C200008F0EACE24CF85E0F3CE90588DCFCF9325
:103C3000DF93FB0122813381DC0113963C932E93A9
:103C40001297448155816681778114964D935D93D7
:103C50006D937C931797408551856285738518967F
:103C60004D935D936D937C931B971C96EF012C965F
:103C70009C01275E3F4F49914D93A217B307D9F797
:103C8000218D328DFC01328F218FDF91CF910895EC
:103C90000F931F93CF93DF938C01EB01FE0164918F
:103CA0002196662349F0D801ED91FC910190F081B5
:103CB000E02DC8011995F2CFDF91CF911F910F919F
:103CC0000895EF92FF920F931F93CF93DF93EC0130
:103CD0007B018A016CE174E00E94481E65E074E09B
:103CE000CE010E94481E66ED73E0CE010E94481E80
:103CF000B701CE010E946D7D67E779E0CE010E9499
:103D00006D7D0115110521F0B801CE010E946D7D78
:103D100067E779E0CE01DF91CF911F910F91FF907E
:103D2000EF900C946D7DCF93DF93EC016BEB73E020
:103D30000E94481E65E074E0CE010E94481E6DE8B6
:103D400073E0CE01DF91CF910C94481ECF93DF93A7
:103D5000EC01FB01248135810E94687CCE01DF915A
:103D6000CF910895EF92FF920F931F93CF93DF931C
:103D700000D000D0CDB7DEB78C017B016DE174E0DF
:103D80000E94537C8AE0E816F1042CF462ED76E0A0
:103D9000C8010E942E7BB701CE0101960E94A17935
:103DA000BE016F5F7F4FC8010E94387BCE01019634
:103DB0000E94B47BC80126960FB6F894DEBF0FBEF2
:103DC000CDBFDF91CF911F910F91FF90EF9008959C
:103DD0002F923F924F925F926F927F928F929F921B
:103DE000AF92BF92CF92DF92EF92FF920F931F9309
:103DF000CF93DF93CDB7DEB7C258D1090FB6F89491
:103E0000DEBF0FBECDBF6C015B0188EE482E83E0A4
:103E1000582E612C712C04EF13E09BE5892E912C18
:103E20008C0E9D1E8CE0880E911C1B019FEF291AA1
:103E3000390AD6015996ED90FC90F70185818230C0
:103E400008F493C082859385A485B5858F719927E1
:103E5000AA27BB27892B8A2B8B2B09F086C040E22F
:103E600050E0BE016F5F7F4FC7010E94658F8032B7
:103E700009F07BC08981882309F477C0853E79F3F6
:103E80008E3269F38C8583FDEACF22961FAE1EAE7B
:103E9000229784E793E09FAF8EAF24961FAE2497BE
:103EA000BE016F5F7F4FE0E080E04EE2DB019D915D
:103EB000BD019032A1F0883049F426E730E02C0FA4
:103EC0003D1F2E0F311DD9014C93EF5F26E730E0E7
:103ED0002C0F3D1F2E0F311DD9019C93EF5F8F5F7B
:103EE0008B3021F786E790E08C0F9D1F8E0F911D80
:103EF000FC011082D60159966D917C9121E0AE01B2
:103F00004A585F4FCE01CE960E946C90882369F18B
:103F1000BE01625C7F4FCE0181960E94000DAE0112
:103F20004A585F4FBE016F5D7F4FCE01855A9F4F4C
:103F30000E946E0DCE01855A9F4F0E94500D88231E
:103F400009F4ACC0F12CFA141B042CF569E0CE0185
:103F500001960E941F7CCE0101960E94071BCE0194
:103F600001960E94B47BF394EECF6F961FAE1EAE07
:103F70006F97A3964CAE5DAE6EAE7FAEA3976D9677
:103F80001FAF0EAF6D97E6961FAE1EAEE697A896D2
:103F90001FAEA897CFCFB401CE0101960E94537CEB
:103FA000CE0101960E94071BCE0101960E94B47BB0
:103FB000E696EEADFFADE697309709F447C08581F0
:103FC000823008F443C068E674E0CE0101960E9496
:103FD000537CCE0101960E94F01ACE0101960E94F8
:103FE000B47B6F968EAD9FAD6F979C838B83A396AA
:103FF0008CAD9DADAEADBFADA3978D839E83AF83DA
:10400000B887A7968CAD9DADAEADBFADA79789879C
:104010009A87AB87BC871A8309838DE0F401DE01A0
:104020001D9601900D928A95E1F7E6968EAD9FADB3
:10403000E6979B8F8A8FB101CE0101960E94E81E00
:10404000CE01855A9F4F0E945C0DF3CE6BE174E068
:10405000CE0101960E94537CCE0101960E94071B5F
:10406000CE0101960E94B47BE696EEADFFADE697D9
:1040700040E050E0BA01309721F0438954896589C6
:104080007689CE0101960E94CD79CE0101960E94DB
:10409000F01ACE0101960E94B47BD2CFCE57DF4FEB
:1040A0000FB6F894DEBF0FBECDBFDF91CF911F9149
:1040B0000F91FF90EF90DF90CF90BF90AF909F90C7
:1040C0008F907F906F905F904F903F902F900895CA
:1040D000CF92DF92EF92FF920F931F93CF93DF93D4
:1040E000CDB7DEB7C455D1090FB6F894DEBF0FBE09
:1040F000CDBF65965FAF4EAF65972091DB0B3091DA
:10410000DC0B2F5F3F4F3093DC0B2093DB0B2091B8
:10411000F80B2111C1C08B016C0181E08093F80B79
:104120001092DC0B1092DB0B6DE174E0CE01895B29
:104130009F4F0E94537C6DE174E0CE01835B9F4FE3
:104140000E94537C50E040E06EE174E0C6010E94A2
:10415000611E0130110509F08EC06DE174E082E549
:104160009FE00E9497796DE174E08EE29FE00E94EB
:1041700097796596EEADFFAD65978081882309F448
:1041800074C000E210E09E012F5F3F4F40E250E01C
:10419000BE016F5D7F4FCE018D5A9F4F0E94787692
:1041A000049739F3BE016F5D7F4FCE018F5B9F4F48
:1041B0000E94537CBE016F5B7F4FCE01895B9F4F96
:1041C0000E947B7BCE018F5B9F4F0E94B47BBE0120
:1041D0006F5F7F4FCE018F5B9F4F0E94537CBE016C
:1041E0006F5B7F4FCE01835B9F4F0E947B7BCE0135
:1041F0008F5B9F4F0E94B47B2D968EAD9FAD2D9708
:104200000297029730F467E374E08EE29FE00E9429
:104210009779BE01695B7F4F82E59FE00E94387B02
:1042200063968EAD9FAD6397892B09F4A2CF63E4AB
:1042300076E0CE018F5B9F4F0E94537CBE01635B93
:104240007F4FCE018F5B9F4F0E94CF7A60E476E074
:104250000E94B97ABC0182E59FE00E94387BCE01C2
:104260008F5B9F4F0E94B47B84CF62E57FE08EE23C
:104270009FE00E94387B1092F80BCE01835B9F4F2A
:104280000E94B47BCE01895B9F4F0E94B47B0FB626
:10429000F894DEBF0FBECDBFCC5ADF4F0FB6F894F7
:1042A000DEBF0FBECDBFDF91CF911F910F91FF9069
:1042B000EF90DF90CF9008950F931F93CF93DF93EC
:1042C00000D000D0CDB7DEB720916D0B2223A9F02E
:1042D0008C0168EC77E0CE0101960E94537CB80116
:1042E000CE0101960E94CF7ABC0185E29DE00E943A
:1042F000837DCE0101960E94B47B26960FB6F8947A
:10430000DEBF0FBECDBFDF91CF911F910F910895FA
:104310000F931F93CF93DF93CDB7DEB72C970FB6D4
:10432000F894DEBF0FBECDBF8C010E945987BC013F
:10433000C8010E94B21E0E945187BC01CE0107969F
:104340000E94B21E60E077E0CE0101960E94537C8D
:10435000BE01695F7F4FCE0101960E94CF7ABC01FA
:10436000C8010E94387BCE0101960E94B47BCE0129
:1043700007960E94B47B60E476E0C8010E942E7B21
:104380000E944987BC01CE0101960E94B21EBE0167
:104390006F5F7F4FC8010E94387BCE0101960E945B
:1043A000B47B6EE374E0C8010E942E7B0E944187BB
:1043B000BC01CE0101960E94B21EBE016F5F7F4F0D
:1043C000C8010E94387BCE0101960E94B47B6EE347
:1043D00074E0C8010E942E7B0E943787BC01CE0189
:1043E00001960E94B21EBE016F5F7F4FC8010E94FE
:1043F000387BCE0101960E94B47BC8012C960FB683
:10440000F894DEBF0FBECDBFDF91CF911F910F910A
:1044100008950F931F93CF93DF93CDB7DEB72C97FB
:104420000FB6F894DEBF0FBECDBF8C010E94598736
:10443000BC01C8010E94B21E0E945187BC01CE017E
:1044400007960E94B21E60E077E0CE0101960E94BE
:10445000537CBE01695F7F4FCE0101960E94CF7AE7
:10446000BC01C8010E94387BCE0101960E94B47B3A
:10447000CE0107960E94B47B0E94AF850E943E86C3
:104480006091D20B70E0CE0107960E94B21E60E0F0
:1044900077E0CE0101960E94537CBE01695F7F4F99
:1044A000CE0101960E94CF7ABC01C8010E94387BE0
:1044B000CE0101960E94B47BCE0107960E94B47B88
:1044C00060E476E0C8010E942E7B0E944987BC010F
:1044D000CE0101960E94B21EBE016F5F7F4FC801E0
:1044E0000E94387BCE0101960E94B47B6EE374E09B
:1044F000C8010E942E7B0E944187BC01CE0101961B
:104500000E94B21EBE016F5F7F4FC8010E94387BC0
:10451000CE0101960E94B47B6EE374E0C8010E9454
:104520002E7B0E943787BC01CE0101960E94B21EED
:10453000BE016F5F7F4FC8010E94387BCE0101969C
:104540000E94B47BC8012C960FB6F894DEBF0FBE54
:10455000CDBFDF91CF911F910F910895CF92DF9240
:10456000EF92FF920F931F93CF93DF9300D000D071
:10457000CDB7DEB77C01FB01848195818A01081BE0
:10458000190B101611069CF0C7010E94387CC70158
:1045900026960FB6F894DEBF0FBECDBFDF91CF9148
:1045A0001F910F91FF90EF90DF90CF900895CE0173
:1045B00001960E944A7CCC24C394D12C60E476E01E
:1045C000CE0101960E942E7BFFEFCF1ADF0A0C1559
:1045D0001D05A4F7BE016F5F7F4FC7010E94387CA5
:1045E000CE0101960E94B47BD2CFDF92EF92FF9270
:1045F0000F931F93CF93DF93CDB7DEB762970FB6BC
:10460000F894DEBF0FBECDBF8C0110929F0A6DE102
:1046100074E0CE010D960E94537CFF24F39485E252
:104620009DE00E940C7320919F0A181619067CF5D4
:1046300021112DC085E29DE00E94EA728A3009F0C6
:104640007EC089899A89892B09F481C0F0929F0ADA
:1046500060E474E0CE0101960E94537CBE01635F6A
:104660007F4FCE0101960E94CF7ABC01CE01079602
:104670000E944A7CCE0107960E945C21CE010796DB
:104680000E94B47BCE0101960E94B47B60C0F12CE5
:10469000E12CDD24D394222309F460C089899A890E
:1046A000019709F045C06FED74E0CE0107960E94B6
:1046B000537CBE01695F7F4FCE010D960E949E7AAA
:1046C000F12C811115C060E574E0CE0101960E94C5
:1046D000537CBE016F5F7F4FCE010D960E949E7A84
:1046E000FF24F3948111F12CCE0101960E94B47B3A
:1046F000CE0107960E94B47BFF20A1F050E040E07D
:10470000BE01635F7F4FCE0101960E94A61EBE01CF
:104710006F5F7F4F85EF9EE00E947B7BCE0101960D
:104720000E94B47B64E170E080E090E00E94407FF2
:10473000BE01635F7F4FC8010E94387C8EC08D3000
:1047400009F47FCF682FCE010D960E940C7B6AE0A2
:1047500070E080E090E00E94407F61CF88E89CE0BC
:104760000E940C731816190614F588E89CE00E9444
:10477000EA728A30A9F08D3099F090919F0A9111D8
:104780000FC0682FCE010D960E940C7B8FEFE81AA8
:10479000F80A65E070E080E090E00E94407FDECFA4
:1047A00089899A89892BA9F3D0929F0AF2CF64E173
:1047B00070E080E090E00E94407FEF2809F43FC065
:1047C00089899A89892BD9F180916D0B882389F188
:1047D00068EC77E0CE0101960E94537CBE016F5FCA
:1047E0007F4FCE010D960E949E7AF82ECE01019643
:1047F0000E94B47BF1101DC069E474E0CE01019603
:104800000E94537CCE0101960E94071BCE010196A7
:104810000E94B47BBE01635F7F4FCE0101960E9470
:104820004A7CCE0101960E94F01ACE0101960E94A8
:10483000B47B64E170E080E090E00E94407F898971
:104840009A8920919F0A21112BCF009709F028CF38
:104850006DE174E0C8010E94537CCE010D960E9468
:10486000B47BC80162960FB6F894DEBF0FBECDBF11
:10487000DF91CF911F910F91FF90EF90DF900895FE
:104880000F931F93CF93DF93CDB7DEB72C970FB65F
:10489000F894DEBF0FBECDBF2C893D89FE01749612
:1048A000AAEABBE090E080E032962817390734F09E
:1048B000408151814D935D930196F6CFCE5BDE4FE3
:1048C00088819981C254D140281739070CF01CC245
:1048D000DC01AA0FBB1FA655B44F880F991FFC011E
:1048E000E855F44F8081918101968D939C938C8D36
:1048F0009D8D90936A0B8093690B8E8D9F8D909305
:104900006C0B80936B0BAD968FADAD97BE01645968
:104910007F4F8F3209F001C2CE0107960E94537C6F
:1049200062E574E0CE0101960E94537CBE01695F8E
:104930007F4FCE0101960E94CF7ABC0186EE90E1B6
:104940000E94647BCE0101960E94B47BCE01079643
:104950000E94B47B66EE70E1CE0101960E944A7C13
:10496000CE0101960E94F01ACE0101960E94B47BFE
:1049700068E674E0CE0101960E94537CBE016F5F31
:104980007F4F86EE90E10E947E7A182FCE0101962D
:104990000E94B47B4091EA105091EB10112309F46E
:1049A000C3C1BA016250710986EE90E10E946D7A2E
:1049B000682FCE0101960E941F7CBE016F5F7F4F62
:1049C00088EC90E10E947B7BCE0101960E94B47B33
:1049D00068EB7FE0CE0107960E94537C6AE674E0A4
:1049E000CE0101960E94537CBE01695F7F4FCE01CC
:1049F00001960E94CF7ABC0180EE90E10E94647B18
:104A0000CE0101960E94B47BCE0107960E94B47B32
:104A100024968FAD24971F928F9323968FAD239763
:104A20001F928F9322968FAD22971F928F9321967C
:104A30008FAD21971F928F9380E794E09F938F9380
:104A40008AE99BE09F938F930E945EB1CE52DF4F25
:104A500088819981C25DD04090938D0280938C02B1
:104A6000BE016C527F4FCE0101960E94537CBE0165
:104A70006F5F7F4F8AED90E10E947B7BCE010196B4
:104A80000E94B47BBE0161527F4FCE0101960E940D
:104A9000537CBE016F5F7F4F84ED90E10E947B7B72
:104AA000CE0101960E94B47B4091D8105091D9104C
:104AB0004250510964ED70E1CE0101960E94A61E9C
:104AC000CE0101960E94057A6C5960939702CE013F
:104AD00001960E94B47BCC5EDE4F688179818A8129
:104AE0009B81C451D1400E94CEAB0FB6F894DEBF7B
:104AF0000FBECDBF9B01AC010E948EAE882389F012
:104B00008CE390E0A0E0B0E0CC5EDE4F8883998338
:104B1000AA83BB83C451D140CD5EDE4F1882C351FE
:104B2000D140CD5EDE4F8881C351D140882399F0BA
:104B3000CC5EDE4F88819981AA81BB81C451D1406E
:104B400080936E0290936F02A0937002B0937102F3
:104B500081E08093500CC85EDE4F688179818A8144
:104B60009B81C851D1409B01AC010E948EAE88232D
:104B700061F080E090E0A0E7B2E4C85EDE4F888399
:104B80009983AA83BB83C851D140C45EDE4F68813C
:104B90007981CC51D140072E000C880B990B0E94D3
:104BA000CEAB9B01AC010E948EAE882341F082E027
:104BB00090E0C45EDE4F99838883CC51D140CE5BB8
:104BC000DE4F68817981C254D140072E000C880BDA
:104BD000990B0E94CEAB9B01AC010E948EAE882344
:104BE00041F083E090E0CE5BDE4F99838883C2542E
:104BF000D140C45CDE4F08811981CC53D140B8014B
:104C0000012E000C880B990B0E94CEAB9B01AC01CE
:104C10000E948EAE811103C01016110644F080E58B
:104C200090E0C45CDE4F99838883CC53D140C45C50
:104C3000DE4F88819981CC53D14090933F0280937D
:104C40003E0288E2FE01E551FF4FAEE6BBE0019077
:104C50000D928A95E1F7CE5CDE4F88819981AA8119
:104C6000BB81C253D1408093290290932A02A09322
:104C70002B02B0932C02CA5CDE4F88819981AA81F5
:104C8000BB81C653D1408093250290932602A09306
:104C90002702B0932802C65CDE4F88819981CA53EF
:104CA000D14090935D0280935C02CC5BDE4F6881C3
:104CB0007981C454D140072E000C880B990B0E94B7
:104CC000CEAB9B01AC010E948EAE882341F088E3FD
:104CD00090E0CC5BDE4F99838883C454D140CC5B99
:104CE000DE4F88819981C454D14090938F02809384
:104CF0008E022C960FB6F894DEBF0FBECDBFDF91AB
:104D0000CF911F910F9108958091AE0B9091AF0BB1
:104D10009093B10B8093B00BEACDCE0107960E9421
:104D2000537C67E574E0FECD4150510966EE70E1B9
:104D3000CE0101960E94A61EBE016F5F7F4F88ECD8
:104D400090E10E947B7BCE0101960E94B47B66EECF
:104D500070E1CE0101960E944A7C68E674E0CE01C3
:104D600001960E94B97ABC0186EE90E10E94647BB4
:104D70002BCEDF92EF92FF920F931F93CF93DF938F
:104D8000CDB7DEB762970FB6F894DEBF0FBECDBFCA
:104D90002091F002222379F12091EF02222359F190
:104DA0007A018C016F3F7F4FA1F560E080E00E94A7
:104DB0005C89D12CB8018EE391E10E94757D64E29B
:104DC00075E08EE391E10E94977DF801848160E0B7
:104DD0008D0D0E945C890E940F826093530C70932A
:104DE000540C8093550C9093560CB701FF0C880B14
:104DF000990B0E94407F62960FB6F894DEBF0FBEFB
:104E0000CDBFDF91CF911F910F91FF90EF90DF9079
:104E1000089560E080E00E945C890E940F8228EE85
:104E200033E040E050E00E9411ADCA01B90120E832
:104E300031E541E050E00E9433ADAB01BC0120E020
:104E4000CE0101960E94F27BBE016F5F7F4FCE01C3
:104E500007960E944A7C62EB78E0CE0107960E949A
:104E6000B97ABC01CE010D960E944A7CCE0107960C
:104E70000E94B47BCE0101960E94B47BBE01635FA9
:104E80007F4F8EE391E10E94757DD98860E08D2D82
:104E90000E945C89CE010D960E94B47B8BCFCF938C
:104EA000DF9300D000D0CDB7DEB70E94010ACE015B
:104EB00001960E9488214AE050E06FEF7FEFCE011B
:104EC00001960E94B926CE0101960E94B47B61E052
:104ED00080E00E945C89CE0101960E94E8196EE391
:104EE00071E1CE0101960E940F7D6CE774E08EE3C4
:104EF00091E10E946D7D0E940F826093E50B70939B
:104F0000E60B8093E70B9093E80B26960FB6F89488
:104F1000DEBF0FBECDBFDF91CF9108950F931F93DA
:104F2000CF93DF9300D000D0CDB7DEB78C01CE0198
:104F300001960E9488214AE050E06FEF7FEFCE019A
:104F400001960E94B926CE0101960E94B47BB80159
:104F5000CE0101960E944A7C4AE050E06FEF7FEF5D
:104F6000CE0101960E94250ACE0101960E94B47BD3
:104F700026960FB6F894DEBF0FBECDBFDF91CF915E
:104F80001F910F910895EF92FF920F931F93CF936C
:104F9000DF9300D01F92CDB7DEB78C017B01FB0100
:104FA00084858830A8F082E194E0F80191838083C1
:104FB0001282138214821582C8010F900F900F90F5
:104FC0000F90DF91CF911F910F91FF90EF90089577
:104FD00080E591E00E94317624E030E0AE014F5F41
:104FE0005F4F6CE070E0F70184850E94F20FBE0114
:104FF0006F5F7F4FC8010E94BB7DDECF3F924F9213
:105000005F926F927F928F929F92AF92BF92CF9258
:10501000DF92EF92FF920F931F93CF93DF93CDB761
:10502000DEB7EA970FB6F894DEBF0FBECDBF7C01A6
:105030002A013B0169010E940F824B015C0187013B
:105040000D5B1F4FC8010E946C13181619069CF0C7
:105050000E940F82681979098A099B09461657062A
:105060006806790608F466C162E370E080E090E0CB
:105070000E94407FE7CF42E250E0BE016F5F7F4F6A
:10508000C8010E94231389818230D1F0312C832DF5
:10509000EA960FB6F894DEBF0FBECDBFDF91CF9179
:1050A0001F910F91FF90EF90DF90CF90BF90AF9046
:1050B0009F908F907F906F905F904F903F9008955A
:1050C000F801848995898334910501F76D817E818A
:1050D0008F8198850E94AFAE4B015C01F601808202
:1050E0009182A282B38246E050E0B701685F7F4FB1
:1050F000CE014D960E94DDB0892B41F6F7018081EB
:105100009181A281B38188169906AA06BB0608F48C
:10511000BDCF84819581A681B78188159905AA059F
:10512000BB0508F4B3CF89899A89AB89BC89868786
:105130009787A08BB18B4EEC50E070E060E0C80127
:105140000E942313312CC701829698AB8FA7F701D9
:10515000B696FAABE9AB08969CAB8BAB67019AE1CC
:10516000C90ED11CBD96FEABEDABC701429698AF00
:105170008FABFD97FAAFE9AF4701FEE18F0E911CAF
:10518000F801818D928D181619060CF080CFC80198
:105190000E9442138333910509F4B2C014F58130A3
:1051A000910509F464C044F4892B51F3C8010E94AD
:1051B0004213AC01552775C08330910509F462C0D4
:1051C0000697A1F7C8010E944213B82E44E050E0B0
:1051D000B401C8010E942313EB2DE450FF0BAF0173
:1051E00060C08A33910509F45FC084F58533910569
:1051F000B1F1C697D9F6C8010E9442135C01B6010D
:10520000CE0189960E94BB7D8BA59CA5ADA5BEA5B0
:10521000892B8A2B8B2BB1F0EDA9FEA94080518000
:1052200062807380B601CE0183960E94BB7D8DA102
:105230009EA1AFA1B8A5A501481659066A067B062E
:1052400009F0B8CF44E050E0B60118C08B339105A7
:1052500009F440C08F3F910509F492CFA7CFC80150
:105260000E944213C8010E944213382E89CFC80100
:105270000E94421344E050E06FA978ADC8010E943B
:1052800023137ECFC8010E944213B82E44E050E0A1
:1052900069AD7AADC8010E9423138B2D8450990B00
:1052A000AC0170E060E0EACFC8010E94421344E024
:1052B00050E069A97AA9C8010E942313F70166A1E9
:1052C00077A180A591A50E94AFAE66A377A380A722
:1052D00091A756CFC8010E94421344E050E06BA949
:1052E0007CA9C8010E942313F70162A573A584A5B8
:1052F00095A50E94AFAE62A773A784A795A740CFDC
:10530000C8010E94421344E050E06FA578A9C8018B
:105310000E942313F70162A173A184A195A10E94A9
:10532000AFAE62A373A384A395A366A777A780AB50
:1053300091AB26CF33243A94AACE2F923F924F922C
:105340005F926F927F928F929F92AF92BF92CF9215
:10535000DF92EF92FF920F931F93CF93DF9300D0D2
:1053600000D0CDB7DEB78C010E9432A32FEC37E01E
:1053700040E050E00E9433ADDC01CB010196A11D5D
:10538000B11DF80184839583A683B78380839183BD
:10539000A283B3835801F3E4AF0EB11CC5010E9490
:1053A000441464E470E0C5010E941817882309F4CE
:1053B00045C10E940F822B013C01480182E4880E06
:1053C000911C48EEC42E43E0D42EE12CF12C52E087
:1053D000252E1E821D82D4018C918330B1F1811162
:1053E00066C0F80184819581A681B7810196A11DCF
:1053F000B11D84839583A683B7830E940F826419AD
:10540000750986099709A70196010E9411ADA901A6
:1054100061E0C8010E94D81781E0D4018C938D818E
:105420009E810197C1F20E940F8264197509860955
:105430009709D801D6962D913D914D915C91D997C0
:10544000261737074807590720F6C5010E9444145C
:10545000F80184819581A681B7810196A11DB11DB6
:1054600084839583A683B7830E940F82F801FE96FA
:1054700060837183828393838D819E8126960FB68C
:10548000F894DEBF0FBECDBFDF91CF911F910F917A
:10549000FF90EF90DF90CF90BF90AF909F908F9054
:1054A0007F906F905F904F903F902F900895843041
:1054B000F1F4F80184819581A681B7810196A11D3F
:1054C000B11D84839583A683B7830E940F826419DC
:1054D000750986099709A70196010E9411ADA901D6
:1054E00063E0C8010E94D817D4012C9298CF813074
:1054F00051F5F80142AD53AD64AD75AD9E012F5F1E
:105500003F4FC8010E94FE27382EF2E08F1390C053
:1055100089819A81AB81BC81F80184839583A683BC
:10552000B7830E940F826419750986099709A7013C
:1055300096010E9411ADA90163E0C8010E94D8172D
:10554000D4013C926CCF823009F069CFF80142ADB2
:1055500053AD64AD75AD9E012F5F3F4FC8010E94F2
:10556000FE27382EF5E08F135DC0E3E0D401EC9305
:10557000F80182A193A1A4A1B5A1892B8A2B8B2B21
:1055800041F484E893E0A0E0B0E082A393A3A4A355
:10559000B5A3F80186A197A1A0A5B1A5892B8A2B57
:1055A0008B2B61F482A193A1A4A1B5A1B695A79577
:1055B0009795879586A397A3A0A7B1A7F80182A581
:1055C00093A5A4A5B5A5892B8A2B8B2BA9F482A121
:1055D00093A1A4A1B5A1AC01BD0123E07695679587
:1055E000579547952A95D1F7841B950BA60BB70BBA
:1055F00082A793A7A4A7B5A7F80186A197A1A0A504
:10560000B1A586A797A7A0ABB1AB82A593A5A4A58A
:10561000B5A582AB93ABA4ABB5AB81E090E09E8324
:105620008D83FDCE96E0891303C0D4011C92F7CE82
:10563000BFEF3B12F4CEF4011082F1CE1E821D8228
:105640001BCF8F929F92AF92BF92EF92FF920F93D8
:105650001F93CF93DF9300D000D0CDB7DEB700917A
:105660004C0C10914D0CF12CE12C0115110509F495
:10567000DAC00E940F824B015C0178012EE3E20E3A
:10568000F11CF70180819181A281B381A501940170
:10569000281B390B4A0B5B0BCA01B901683E33E08A
:1056A000730781059105A0F128EE33E040E050E05A
:1056B0000E9411AD861A970AA80AB90AD7018D92DD
:1056C0009D92AD92BC921397F80186A597A5A0A9CB
:1056D000B1A949015A01880C991CAA1CBB1C881548
:1056E0009905AA05BB0508F0B0C016A617A610AA12
:1056F00011AAF80182A993A9A4A9B5A988159905A9
:10570000AA05BB0508F0AAC012AA13AA14AA15AAD2
:10571000F80186A597A5A0A9B1A9892B8A2B8B2B67
:1057200009F0A5C0EE5BFF4F8081833009F09FC078
:1057300084E08083C8010E949D2901967C01F801C4
:1057400082A993A9A4A9B5A9892B8A2B8B2BA1F493
:10575000EE5BFF4F8081833011F081110DC010820C
:10576000F8013E9684E1DF011D928A95E9F7C801B0
:105770000E949D2903967C01B2E0EB16F10429F00A
:10578000E4E0EE16F10409F04EC080E591E00E94DD
:10579000317660914C0C70914D0C625F7F4FCE0161
:1057A00001960E94BB7DCE0103960E94F810609185
:1057B0004C0C70914D0C6A5E7F4FCE0101960E9499
:1057C000BB7D44E050E0BE016D5F7F4F81E090E023
:1057D0000E949A0E60914C0C70914D0C6E5E7F4F42
:1057E000CE0101960E94BB7D44E050E0BE016D5F9A
:1057F0007F4F85E090E00E949A0E60914C0C709172
:105800004D0C625E7F4FCE0101960E94BB7D8B8165
:105810009C81AD81BE818093190E90931A0EA09346
:105820001B0EB0931C0EC70126960FB6F894DEBF70
:105830000FBECDBFDF91CF911F910F91FF90EF90E1
:10584000BF90AF909F908F900895821B930BA40BF5
:10585000B50B86A797A7A0ABB1AB4BCF821B930B21
:10586000A40BB50B82AB93ABA4ABB5AB51CFF12C72
:10587000E12C65CFEF92FF920F931F93CF93DF93AD
:10588000CDB7DEB7E8970FB6F894DEBF0FBECDBF39
:105890006DE174E0CE0187960E94537C6DE174E067
:1058A000CE018D960E94537C82E0E82EF12C249646
:1058B000FFAEEEAE249786E0EBEFF2E0DE01D3968A
:1058C00001900D928A95E1F786E0FE01F396DE01E4
:1058D000AC5BBF4F01900D928A95E1F72C961FAEFD
:1058E0001EAE2C9701E010E02E961FAF0EAF2E9744
:1058F00088E0E1E0F3E0DE01599601900D928A958F
:10590000E1F788E0FE017996DE01A25BBF4F0190CE
:105910000D928A95E1F788E1E9E0F3E0DE01119666
:1059200001900D928A95E1F788E1FE013196DE0142
:10593000AA5ABF4F01900D928A95E1F780912103F9
:1059400090912203A0912303B0912403E2968CAF9F
:105950009DAFAEAFBFAFE29760E874E0CE0187962F
:105960000E94977960E0CE0187960E940C7B4BA540
:105970005CA5BE016E587F4FCE0187960E9450777E
:105980006DE376E0CE018D960E943F7B66ED74E07C
:1059900088EC90E10E94977960E0CE018D960E949C
:1059A0000C7B49A95AA9BE0166567F4FCE018D9640
:1059B0000E9450776DE174E0CE0187960E9497793E
:1059C0006DE174E0CE018D960E949779C250DF4F51
:1059D00019821882CE5FD04080918C0290918D0206
:1059E000C050DF4F99838883C050D14080E090E061
:1059F000A0E7B2E4CA5BDE4F88839983AA83BB83A6
:105A0000C654D140C65BDE4FF982E882CA54D14009
:105A100080E090E0A0E2B2E4C45BDE4F888399832B
:105A2000AA83BB83CC54D14080E090E0A4E3B2E4ED
:105A3000C05BDE4F88839983AA83BB83C055D14066
:105A400084EB90E0CC5ADE4F99838883C455D140D3
:105A500088E790E0CA5ADE4F99838883C655D140C3
:105A60008CE291E0A0E0B0E0C85ADE4F88839983D1
:105A7000AA83BB83C855D140C45ADE4F198308831B
:105A8000CC55D140C25ADE4FF982E882CE55D14082
:105A900060E08AED90E10E940C7B60E084ED90E193
:105AA0000E940C7B4091DE105091DF10BE016E5FB2
:105AB0007E4F8AED90E10E9450774091D81050912E
:105AC000D910BE01635F7E4F84ED90E10E94507754
:105AD00088E2EEE6FBE0DE01A75EBE4F01900D928C
:105AE0008A95E1F78CE390E0A0E0B0E0CE5BDE4F7A
:105AF00088839983AA83BB83C254D140CF5BDE4F96
:105B00001882C154D14084EE98E3AEE8B2E4C05AA2
:105B1000DE4F88839983AA83BB83C056D14084EE2D
:105B200098E3AEE8B1E4CC59DE4F88839983AA8329
:105B3000BB83C456D140C859DE4F19830883C85669
:105B4000D14080E590E0C659DE4F99838883CA56DC
:105B5000D14083E090E0C059DE4F99838883C057DD
:105B6000D14088E390E0CE58DE4F99838883C257B6
:105B7000D14084EF91E09093670280936602BE016A
:105B80006E5B7F4F0E944F0964EF71E080E090E010
:105B90000E94407F66E276E0CE0181960E94417CC1
:105BA000CE0181960E94F01ACE0181960E94B47BAC
:105BB000CE018D960E94B47BCE0187960E94B47B65
:105BC000E8960FB6F894DEBF0FBECDBFDF91CF9140
:105BD0001F910F91FF90EF9008959F92AF92BF9207
:105BE000CF92DF92EF92FF920F931F93CF93DF93A9
:105BF000CDB7DEB7C859D1090FB6F894DEBF0FBED6
:105C0000CDBF5C017B016A0160EE7FE0CE01895768
:105C10009F4F0E94537C68E674E08E010F5F1F4F18
:105C2000C8010E94537CB801CE0189579F4F0E9442
:105C30009E7A982EC8010E94B47B911014C068E629
:105C400074E0C8010E94537CBE0169577F4FC801B0
:105C50000E94CF7ABC01CE0189579F4F0E94647B7E
:105C6000C8010E94B47BB501CE0183579F4F0E94AB
:105C7000537C68E874E0E114F10471F066E974E0C3
:105C800021E0E216F10441F061EA74E032E0E3164B
:105C9000F10411F069EA74E0CE0189579F4F0E9428
:105CA0002E7B60E0CE0189579F4F0E940C7BB6018E
:105CB000C8010E944A7C6AE0C8010E94207BBC01A6
:105CC000CE018D569F4F0E944A7CC8010E94B47B32
:105CD000C557DF4F48815981CB58D040B801CE011C
:105CE00089579F4F0E9450778091510C882399F1DA
:105CF00061EB74E0CE018F579F4F0E94537CCE0121
:105D00008F579F4F0E94071BCE018F579F4F0E94B6
:105D1000B47BBE0169577F4FCE018F579F4F0E94C2
:105D20004A7CCE018F579F4F0E94071BCE018F5791
:105D30009F4F0E94B47BB801CE018F579F4F0E94A6
:105D4000537CCE018F579F4F0E94071BCE018F5768
:105D50009F4F0E94B47BCC56DF4F8881C459D040FE
:105D60008F93CD56DF4F8881C359D0408F93C25750
:105D7000DF4F8881CE58D0408F93C357DF4F888143
:105D8000CD58D0408F9381EC94E09F938F938EEC0D
:105D9000E82E89E0F82EFF92EF920E945EB14091CA
:105DA0003E0250913F026AE97BE087E69FE00E9455
:105DB000D5150FB6F894DEBF0FBECDBF019709F021
:105DC0007CC01F930F9387EC94E09F938F9304ED17
:105DD0001AE01F930F930E945EB1B80187E69FE01F
:105DE0000E94597D8AE99BE09F938F9388ED94E010
:105DF0009F938F931F930F930E945EB1B80187E624
:105E00009FE00E94597D6EE274E087E69FE00E9469
:105E1000977D67E779E087E69FE00E94B47CF70111
:105E200001900020E9F7CF018F5C99409F938F93F9
:105E300081EE94E09F938F931F930F930E945EB126
:105E4000B80187E69FE00E94597DB70187E69FE091
:105E50000E946D7D62E370E080E090E00E94407FF0
:105E600087E69FE00E9487150FB6F894DEBF0FBE4D
:105E7000CDBF11E0CE018D569F4F0E94B47BCE0165
:105E800083579F4F0E94B47BCE0189579F4F0E943A
:105E9000B47B812FC856DF4F0FB6F894DEBF0FBE1C
:105EA000CDBFDF91CF911F910F91FF90EF90DF90C9
:105EB000CF90BF90AF909F90089561E774E0CE01BE
:105EC0008F579F4F0E94417CCE018F579F4F0E945A
:105ED000F01ACE018F579F4F0E94B47B6DE774E09C
:105EE000CE018F579F4F0E94417CCE018F579F4F0D
:105EF0000E94071BCE018F579F4F0E94B47B6EEC10
:105F000079E0CE018F579F4F0E94537CCE018F576F
:105F10009F4F0E94F01ACE018F579F4F0E94B47B73
:105F200010E0A8CFEF92FF920F931F93CF93DF93D0
:105F3000CDB7DEB768970FB6F894DEBF0FBECDBF02
:105F400081E08093F80B0E94212B8C0160ED77E0BB
:105F500080E090E00E94407F8BE0E82EF12C0D7FE6
:105F60000130110571F481E0E81AF10851F00E9446
:105F7000212B8C0160ED77E080E090E00E94407F73
:105F8000EECF0E94FE7F7C0168EE73E080E090E03F
:105F90000E94407F0BE010E0EF2899F401501109B6
:105FA00081F060ED77E080E090E00E94407F0E9409
:105FB000FE7F7C0168EE73E080E090E00E94407F0D
:105FC000EBCF81E29EE00E94E6181092F80B0E944F
:105FD0004F276DE174E0CE0107960E94537C6CEA76
:105FE00075E0CE010D960E94417CCE0143960E9441
:105FF000E819888D1F928F938F891F928F938E89B6
:106000001F928F938D891F928F9380E794E09F93C7
:106010008F9384ED9AE09F938F930E945EB164ED1D
:106020007AE0CE0101960E94537CBE016F5F7F4FE4
:10603000CE0107960E947B7BCE0101960E94B47B25
:10604000BE01635F7F4FCE0101960E944A7CCE0164
:1060500001960E94071BCE0101960E94B47BBE01EF
:10606000695F7F4FCE0101960E944A7CCE01019666
:106070000E94F01ACE0101960E94B47BBE01695FB6
:106080007F4FCE0101960E944A7CAE014F5F5F4F69
:1060900063E070E080E092E00E94ED2D182FCE01C9
:1060A00001960E94B47B0FB6F894DEBF0FBECDBF41
:1060B00011112BC062EA75E0CE0101960E94417C6D
:1060C000CE0101960E94071BCE0101960E94B47B6F
:1060D000BE01635F7F4FCE0101960E944A7CCE01D4
:1060E00001960E94071BCE0101960E94B47B64E3D7
:1060F0007FE0CE0101960E944A7CCE0101960E946B
:10610000F01ACE0101960E94B47BCE010D960E943A
:10611000B47BCE0107960E94B47B68960FB6F894C4
:10612000DEBF0FBECDBFDF91CF911F910F91FF90CA
:10613000EF9008957F928F929F92AF92BF92CF92ED
:10614000DF92EF92FF920F931F93CF93DF93CDB720
:10615000DEB762970FB6F894DEBF0FBECDBF6FE813
:1061600075E0CE0101960E94417CCE0101960E940D
:10617000F01ACE0101960E94B47B04E010E030EAF0
:10618000C32E3AE0D32E40E3E42E53EEB52E66E064
:10619000A62E7CEE972EE1E3FE2EFEE48F2EA4E3E6
:1061A0007A2E68EB72E287E09FE00E941817F601F2
:1061B0008E2D11928A95E9F7B092A00AA092A20AB8
:1061C0009092A30AF092AC0A8092AD0AF092AE0AC5
:1061D0007092AF0A60E472E0CE0101960E94BB7D2E
:1061E0004BE750E0BE016F5F7F4F87E09FE00E946A
:1061F000A11740E350E060EA7AE087E09FE00E9468
:10620000361787E09FE00E94701768EE73E080E029
:1062100090E00E94407F87E09FE00E946C13892BF2
:1062200009F04FC00150110909F07CC08091D00ADB
:106230009091D10AA091D20AB091D30A892B8A2BCE
:106240008B2B09F089C06DE174E082E59FE00E942C
:10625000977962E57FE0CE0101960E944A7CAE010B
:106260004F5F5F4F70E060E082E792E00E94ED2DAB
:10627000182FCE0101960E94B47B11110EC067E762
:1062800075E0CE0101960E94417CCE0101960E94EC
:10629000F01ACE0101960E94B47B62960FB6F89474
:1062A000DEBF0FBECDBFDF91CF911F910F91FF9049
:1062B000EF90DF90CF90BF90AF909F908F907F90A6
:1062C000089540E350E060EA7AE087E09FE00E94B2
:1062D00023136091C80A7091C90A76276727762729
:1062E00090E080E0CB01772766270091CA0A1091E1
:1062F000CB0A10270127102730E020E0602B712BFC
:10630000822B932B7E508A4A93480E948A850E9452
:10631000AF856093D00A7093D10A8093D20A90938C
:10632000D30A84CF68EE73E080E090E00E94407F63
:106330004091D00A5091D10A6091D20A7091D30A4B
:106340002AE085E29DE00E94C37C67E779E085E270
:106350009DE00E94B47C25CF68EE73E080E090E081
:106360000E94407F0E94AF856093EF0B7093F00B0B
:106370008093F10B9093F20B0E94AF856093E90B31
:106380007093EA0B8093EB0B9093EC0BCE0101968C
:106390000E940922CE0101960E94F01ACE010196B8
:1063A0000E94B47B0E944987BC01CE0107960E94DF
:1063B000B21E6EE374E0CE0107960E942E7B0E940F
:1063C0004187BC01CE0101960E94B21EBE016F5FE3
:1063D0007F4FCE0107960E94387BCE0101960E9426
:1063E000B47B6EE374E0CE0107960E942E7B0E9480
:1063F0003787BC01CE0101960E94B21EBE016F5FBD
:106400007F4FCE0107960E94387BCE0101960E94F5
:10641000B47B66EF74E0CE0101960E94537CBE010E
:10642000695F7F4FCE0101960E94CF7ABC01CE01F9
:106430000D960E944A7C4AE050E06FEF7FEFCE015C
:106440000D960E94B926CE010D960E94B47BCE0116
:1064500001960E94B47BCE0107960E94B47B68EE41
:1064600073E080E090E00E94407F0E945987BC0169
:10647000CE010D960E94B21E0E945187BC01CE0132
:1064800001960E94B21E60E077E0CE0107960E945E
:10649000537CBE016F5F7F4FCE0107960E94CF7A7B
:1064A000BC01CE010D960E94387BCE0107960E945A
:1064B000B47BCE0101960E94B47B0E94AF850E94FE
:1064C0003E866091D20B70E0CE0101960E94B21E12
:1064D00060E077E0CE0107960E94537CBE016F5FBB
:1064E0007F4FCE0107960E94CF7ABC01CE010D9658
:1064F0000E94387BCE0107960E94B47BCE010196A4
:106500000E94B47B6CEF74E0CE0101960E94537C34
:10651000BE01635F7F4FCE0101960E94CF7ABC011E
:10652000CE0107960E944A7C4AE050E06FEF7FEF71
:10653000CE0107960E94B926CE0107960E94B47B31
:10654000CE0101960E94B47BCE010D960E94B47BD1
:1065500068EE73E080E090E00E94407FCE010196FB
:106560000E9488214AE050E06FEF7FEFCE01019654
:106570000E94B9268ECECF92DF92EF92FF920F93B8
:106580001F93CF93DF93CDB7DEB768970FB6F8941C
:10659000DEBF0FBECDBF6DE174E0CE0143960E9419
:1065A000537C6AE677E0CE0101960E94417CCE01E1
:1065B00001960E94071BCE0101960E94B47B6CA13C
:1065C0007DA1CE0101960E94A179CE0101960E9483
:1065D000F01ACE0101960E94B47B62E577E0CE010D
:1065E00001960E94417CCE0101960E94071BCE01BC
:1065F00001960E94B47BCE5ADE4F68817981C255E4
:10660000D140CE0101960E94A179CE0101960E944F
:10661000F01ACE0101960E94B47B65E477E0CE01CA
:1066200001960E94417CCE0101960E94071BCE017B
:1066300001960E94B47B0AEA1BE0EE24E394F12C5D
:10664000CE5ADE4F88819981C255D1408E159F0563
:106650000CF44AC0F80182819381C6979CF162E0F4
:1066600075E0CE0101960E94537CCE0101960E94F6
:10667000071BCE0101960E94B47BF80162817381F1
:1066800066537109CE0101960E94A179CE0101964F
:106690000E94071BCE0101960E94B47B60E476E065
:1066A000CE0101960E94537CCE0101960E94071BE9
:1066B000CE0101960E94B47BFFEFEF1AFF0A0E5F36
:1066C0001F4FBECF6DEB76E0CE0101960E94537C4A
:1066D000CE0101960E94071BCE0101960E94B47B59
:1066E000F80162817381CECF60E476E0CE0101963D
:1066F0000E94537CCE0101960E94F01ACE010196B1
:106700000E94B47B66E377E0CE0101960E94417C53
:10671000CE0101960E94071BCE0101960E94B47B18
:106720006091690B70916A0BCE0101960E94A1796C
:10673000CE0101960E94071BCE0101960E94B47BF8
:1067400060E476E0CE0101960E94537CCE01019672
:106750000E94071BCE0101960E94B47B60916B0BD7
:1067600070916C0BCE0101960E94A179CE01019629
:106770000E94F01ACE0101960E94B47B6FE177E08F
:10678000CE0101960E94417CCE0101960E94071B1A
:10679000CE0101960E94B47BBE01605D7F4FCE01A9
:1067A00001960E94537CCE0101960E94071BCE01E8
:1067B00001960E94B47B60E476E0CE0101960E94CF
:1067C000537CCE0101960E94071BCE0101960E94C8
:1067D000B47BBE016C5C7F4FCE0101960E94537C5E
:1067E000CE0101960E94F01ACE0101960E94B47B60
:1067F0006FE077E0CE0101960E94417CCE010196C8
:106800000E94F01ACE0101960E94B47B8E010C5DAD
:106810001F4FEE24E394F12C680188E0C80ED11CD0
:106820008CA19DA18E159F050CF449C0B701CE0126
:1068300007960E94A17968EC77E0CE0101960E944C
:10684000537CBE01695F7F4FCE0101960E94CF7AD3
:10685000BC01CE010D960E944A7CCE010D960E948D
:10686000071BCE010D960E94B47BCE0101960E94BB
:10687000B47BCE0107960E94B47B60E077E0CE0146
:1068800001960E94537CCE0101960E94071BCE0107
:1068900001960E94B47BB801645E7F4FCE010196E1
:1068A0000E94537CCE0101960E94F01ACE010196FF
:1068B0000E94B47BEFEFEE1AFE0A8601ADCF6EEFB9
:1068C00076E0CE0101960E94417CCE0101960E94A5
:1068D000071BCE0101960E94B47B7E01F2EBEF1AFA
:1068E000FEEFFF0A10E000E0F70161917F0170E028
:1068F000CE0101960E94A179CE0101960E94071B4C
:10690000CE0101960E94B47B0330110571F064E062
:1069100075E0CE0101960E94537CCE0101960E9443
:10692000071BCE0101960E94B47B0F5F1F4F0430FE
:106930001105D1F660E476E0CE0101960E94537C09
:10694000CE0101960E94F01ACE0101960E94B47BFE
:10695000C45BDE4F68817981CC54D140072E000C96
:10696000880B990B0E94CEAB9B01AC010E948EAEAE
:10697000882341F080E590E0C45BDE4F99838883F3
:10698000CC54D140C45BDE4F88819981CC54D14036
:1069900090933F0280933E0264EE76E0CE01019632
:1069A0000E94417CCE0101960E94071BCE010196F8
:1069B0000E94B47B6AE97BE0CE0101960E94537C81
:1069C000CE0101960E94071BCE0101960E94B47B66
:1069D00062EE76E0CE0101960E94417CCE010196E6
:1069E0000E94071BCE0101960E94B47B60913E027B
:1069F00070913F02CE0101960E94A179CE010196CD
:106A00000E94F01ACE0101960E94B47B63ED76E0FD
:106A1000CE0101960E94417CCE0101960E94071B87
:106A2000CE0101960E94B47BBE016C5A7F4FCE010D
:106A300001960E94537CCE0101960E94F01ACE016D
:106A400001960E94B47B66E075E0CE0101960E943B
:106A5000537CCE0101960E94071BCE0101960E9435
:106A6000B47BBE0164587F4FCE0101960E94537CD7
:106A7000CE0101960E94F01ACE0101960E94B47BCD
:106A8000C052DF4F88819981C05ED040892B71F45C
:106A90006BEC76E0CE0101960E94417CCE0101961E
:106AA0000E94F01ACE0101960E94B47BC052DF4FC3
:106AB00088819981C05ED040019771F461EC76E0E5
:106AC000CE0101960E94417CCE0101960E94F01AEF
:106AD000CE0101960E94B47BC052DF4F888199811C
:106AE000C05ED040029771F468EB76E0CE0101966B
:106AF0000E94417CCE0101960E94F01ACE010196BF
:106B00000E94B47B62EB76E0CE0101960E94417C4C
:106B1000CE0101960E94071BCE0101960E94B47B14
:106B2000CE51DF4F68817981C25ED040CE0101969F
:106B30000E94A179CE0101960E94F01ACE01019621
:106B40000E94B47B69EA76E0CE0101960E94417C06
:106B5000CE0101960E94071BCE0101960E94B47BD4
:106B6000CC5ADE4F88819981C455D140C6970CF428
:106B70001FC162E075E0CE0101960E94537CCE01F8
:106B800001960E94071BCE0101960E94B47BCC5A4D
:106B9000DE4F68817981C455D14066537109CE01B9
:106BA00001960E94A179CE0101960E94F01ACE01B1
:106BB00001960E94B47B4091E10B5091E20B6091F1
:106BC000E30B7091E40B21E0CE0107960E94BC7BA1
:106BD00061E175E0CE0101960E94537CBE01695FC0
:106BE0007F4FCE0101960E94CF7A6CE175E00E9442
:106BF000B97ABC01CE010D960E944A7CCE010D9659
:106C00000E94F01ACE010D960E94B47BCE0101962F
:106C10000E94B47BCE0107960E94B47B4091DD0BAD
:106C20005091DE0B6091DF0B7091E00B21E0CE0103
:106C300007960E94BC7B61E275E0CE0101960E943E
:106C4000537CBE01695F7F4FCE0101960E94CF7ACF
:106C50006CE175E00E94B97ABC01CE010D960E94EC
:106C60004A7CCE010D960E94F01ACE010D960E942C
:106C7000B47BCE0101960E94B47BCE0107960E94A0
:106C8000B47B6BE876E0CE0101960E94417CCE0198
:106C900001960E94071BCE0101960E94B47B409191
:106CA000290250912A0260912B0270912C0225E05A
:106CB000CE0101960E94BC7BCE0101960E94F01A83
:106CC000CE0101960E94B47B61E776E0CE01019689
:106CD0000E94417CCE0101960E94071BCE010196C5
:106CE0000E94B47B409125025091260260912702B8
:106CF0007091280225E0CE0101960E94BC7BCE0156
:106D000001960E94F01ACE0101960E94B47B61E6C2
:106D100076E0CE0101960E94417CCE0101960E9450
:106D2000071BCE0101960E94B47B60916C027091AA
:106D30006D02CE0101960E94A179CE0101960E94BA
:106D4000F01ACE0101960E94B47B6FE476E0CE018A
:106D500001960E94417CCE0101960E94071BCE0144
:106D600001960E94B47BC65BDE4F68817981CA546C
:106D7000D140CE0101960E94A179CE0101960E94D8
:106D8000F01ACE0101960E94B47BCE0143960E9478
:106D9000B47B68960FB6F894DEBF0FBECDBFDF910F
:106DA000CF911F910F91FF90EF90DF90CF900895BA
:106DB0006DEB76E0CE0101960E94537CCE010196E8
:106DC0000E94071BCE0101960E94B47BCC5ADE4F75
:106DD00068817981C455D140E2CE2F923F924F9283
:106DE0005F926F927F928F929F92AF92BF92CF925B
:106DF000DF92EF92FF920F931F93CF93DF93CDB764
:106E0000DEB7EC970FB6F894DEBF0FBECDBF9CA7E0
:106E10008BA71B0170E060E00E946D7A182F6DE176
:106E200074E0CE0149960E94537C80916C0290914F
:106E30006D02019709F07AC082E090E00E94F5852A
:106E400088E090E0909324028093230289E090E010
:106E500090932202809321028091670B9091680B9E
:106E60009093660B8093650B80911D0290911E029A
:106E7000A0911F02B09120028093190290931A02F0
:106E8000A0931B02B0931C028091350290913602B0
:106E9000A0913702B09138028093390290933A0260
:106EA000A0933B02B0933C028091640B8093630BF0
:106EB00080915F0B9091600BA091610BB091620B80
:106EC00080935B0B90935C0BA0935D0BB0935E0B78
:106ED0008AE390E090931802809317028091E10B6F
:106EE0009091E20BA091E30BB091E40B8093960B91
:106EF0009093970BA093980BB093990B80911502E8
:106F000090911602909314028093130280912902AB
:106F100090912A02A0912B02B0912C0280932D0215
:106F200090932E02A0932F02B093300280916C02B6
:106F300090916D02029709F07AC083E090E00E9480
:106F4000F5858AE090E090932402809323028BE001
:106F500090E090932202809321028091590B9091AE
:106F60005A0B9093660B8093650B80910F02909162
:106F70001002A0911102B091120280931902909315
:106F80001A02A0931B02B0931C02809131029091CF
:106F90003202A0913302B09134028093390290936F
:106FA0003A02A0933B02B0933C028091580B80932D
:106FB000630B8091540B9091550BA091560BB0919F
:106FC000570B80935B0B90935C0BA0935D0BB0937E
:106FD0005E0B8BE390E090931802809317028091F0
:106FE000DD0B9091DE0BA091DF0BB091E00B809355
:106FF000960B9093970BA093980BB093990B80915D
:107000000D0290910E0290931402809313028091CE
:10701000250290912602A0912702B0912802809328
:107020002D0290932E02A0932F02B09330021335BD
:10703000C1F41092660B1092650B80916D0B882342
:1070400071F068E275E0CE0101960E94537CCE019A
:1070500001960E94F01ACE0101960E94B47BE12CA9
:10706000E1C0C1010197029708F07AC181E090E088
:10707000A0E0B0E08093190290931A02A0931B0243
:10708000B0931C02ABA5BCA514968D919C9115974D
:10709000029750F141E050E0BD01CE0101960E94FF
:1070A000A61EBE016F5F7F4FCE0149960E947B7B7B
:1070B000CE0101960E94B47BCE014996B1E02B1619
:1070C000310471F50E94FA7920E030E040E251E4A9
:1070D0000E942DAC0E9453AE6093190270931A0265
:1070E00080931B0290931C0281E090E09093660BCA
:1070F0008093650B1134F9F480916D0B882371F046
:107100006DE275E0CE0101960E94537CCE0101969E
:107110000E94F01ACE0101960E94B47BE12C4FC070
:107120000E94FA7920912D0230912E0240912F0277
:1071300050913002CDCF163409F0FCC080916D0B18
:10714000882371F066E375E0CE0101960E94537CBE
:10715000CE0101960E94071BCE0101960E94B47BCE
:10716000EE24E394F12C60E0809121020E94877E5E
:1071700064E670E080E090E00E94407F6E2D809198
:1071800023020E94877E64EF71E080E090E00E941D
:10719000407F60E0809121020E94877E64E670E07B
:1071A00080E090E00E94407F6E2D809123020E943B
:1071B000877E64EF71E080E090E00E94407F8091E4
:1071C0006D0B882379F14091190250911A02609158
:1071D0001B0270911C022AE0CE0101960E94F27BF4
:1071E000BE016F5F7F4FCE0107960E944A7C6AE422
:1071F00075E0CE0107960E94B97ABC01CE010D96CA
:107200000E944A7CCE010D960E94F01ACE010D9686
:107210000E94B47BCE0107960E94B47BCE010196FA
:107220000E94B47B8091190290911A02A0911B02D6
:10723000B0911C02181619061A061B060CF053C54D
:10724000163409F459C4123509F45AC46E2D8091CC
:1072500023020E94877E64EF71E080E090E00E944C
:10726000407F6E2D809123020E94877E60ED77E043
:1072700080E090E00E94407F6E2D809123020E946A
:10728000877E6CED75E080E090E00E94407F81E0B9
:1072900090E09093660B8093650B61E080912102F2
:1072A0000E94877E61E070E080E090E00E94407F75
:1072B00060E0809121020E94877E6AE070E080E0B9
:1072C00090E00E94407FC12CD12C7601C394809124
:1072D000190290911A02A0911B02B0911C02C816CB
:1072E000D906EA06FB060CF00DC46091650B80918F
:1072F00021020E94877E61E070E080E090E00E94C1
:10730000407F60E0809121020E94877E6091390277
:1073100070913A0280913B0290913C026F5F7F4FE7
:107320008F4F9F4F0E94407FFFEFCF1ADF0AEF0A77
:10733000FF0ACDCF123591F480916D0B882371F047
:1073400060E475E0CE0101960E94537CCE01019667
:107350000E94071BCE0101960E94B47BE12C03CF53
:107360002114310429F0E3E02E16310409F077CE20
:1073700080916C0290916D0220E137E240E050E094
:107380008130910521F420E43CE940E050E02FA752
:1073900038AB49AB5AAB21E030E03093660B209319
:1073A000650B30935D0220935C02029761F433E039
:1073B0002316310441F48091AE109091AF10909358
:1073C0005D0280935C0240915C0250915D025EA779
:1073D0004DA7052F001F0027001F81E090E090932C
:1073E0005D0280935C0260E0809121020E94877EB2
:1073F00064E670E080E090E00E94407F602F809122
:1074000023020E94877E64EF71E080E090E00E949A
:10741000407F602F809123020E94877E68EE73E098
:1074200080E090E00E94407F60E0809121020E9415
:10743000877E64E670E080E090E00E94407F602FED
:10744000809123020E94877E64EF71E080E090E0EB
:107450000E94407F8FEF9FEF90931402809313025E
:10746000812C912C54011FA218A619A61AA61BA2A2
:107470001CA21DA21EA21F8E18A219A21AA2412C84
:10748000512C32011FAA18AE19AE1AAE1BAA1CAAA3
:107490001DAA1EAA61E0809121020E94877E61E000
:1074A00070E080E090E00E94407F60E080912102E7
:1074B0000E94877E61E070E080E090E00E94407F63
:1074C000C501B40126E030E040E050E00E9433AD59
:1074D000672B682B692B09F0F8C0A2E0B0E0BCAFC5
:1074E000ABAFC12CD12C760180911702863308F006
:1074F000865320917B00982F9870277F922B909332
:107500007B008770806480937C0080917A00806427
:1075100080937A0080917A0086FDFCCF809178007C
:1075200060917900762F682F072E000C880B990B3D
:107530000E94CEAB9B01AC01C701B6010E9475ADA4
:107540006B017C0162E070E080E090E00E94407F8F
:107550002BAD3CAD2130310509F0ADC020E030EC61
:107560004FEF54E4C701B6010E94E1AD6B017C010D
:1075700080916D0B882399F12DEC3CEC4CE45EE39B
:10758000C701B6010E9489AE87FD29C022E0B7017C
:10759000A601CE0107960E94BC7B61E575E0CE0195
:1075A00001960E94537CBE01695F7F4FCE01019618
:1075B0000E94CF7ABC01CE010D960E944A7CCE017A
:1075C0000D960E94F01ACE010D960E94B47BCE015A
:1075D00001960E94B47BCE0107960E94B47B2AE9F3
:1075E00039E949E95EE3C701B6010E9489AE87FD2A
:1075F00013C0411451046104710411F424013501D4
:107600008BA19CA1ADA1BEA1892B8A2B8B2B21F430
:107610008BA29CA2ADA2BEA22DEC3CEC4CE45EE39E
:10762000C701B6010E94C7AB18160CF449C041143B
:1076300051046104710409F448C02F8D38A149A197
:107640005AA1232B242B252B69F48FA198A5A9A53A
:10765000BAA5892B8A2B8B2B09F403C18F8E98A294
:10766000A9A2BAA22F8D38A149A15AA14216530648
:107670006406750654F5809113029091140297FFE9
:10768000F5C01092140210921302420E531E641E93
:10769000751ED301C201B595A795979587958FABB8
:1076A00098AFA9AFBAAF1F8E18A219A21AA2412C87
:1076B000512C32010AC0E1E0F0E0FCAFEBAF14CF97
:1076C000411451046104710469F6E0901302F090D2
:1076D000140292E0E916F1043CF4F7FCE3C0A3E0E5
:1076E0002A16310409F0DEC08FA498A8A9A8BAA868
:1076F000BAE08B0E911CA11CB11C8FA598A9A9A959
:10770000BAA988169906AA06BB060CF4C3CEF2E005
:10771000EF16F1040CF479C06BA97CA98DA99EA980
:107720002FA938AD49AD5AAD621B730B840B950B75
:107730000E94CEAB4B015C01B701FF0C880B990B8B
:107740000E94CEAB9B01AC01C501B4010E94E1AD2A
:1077500020E030E044EB53E40E94E1AD6B017C019A
:10776000C0922D02D0922E02E0922F02F0923002AF
:1077700020E030E040E85FE30E9489AE87FDACC0C6
:1077800080916C0290916D028130910509F090C05A
:10779000C092A610D092A710E092A810F092A91063
:1077A000C0922902D0922A02E0922B02F0922C027F
:1077B00065ED75E0CE0101960E94417CCE010196F7
:1077C0000E94071BCE0101960E94B47B40912D02BE
:1077D00050912E0260912F027091300225E0CE016F
:1077E00001960E94BC7BCE0101960E94F01ACE0148
:1077F00001960E94B47B84EF91E09093670280939E
:10780000660268E87FE00E944F0933E023163104E6
:1078100029F0E02E2114310409F004CD8BA59CA59C
:107820000E94FA796B017C01C092960BD092970B63
:10783000E092980BF092990B20E030E044EB53E497
:10784000C701B6010E9489AE87FD6AC020E030E022
:1078500044EB53E4C701B6010E9474AD6B017C0197
:10786000EBCF8FA298A6A9A6BAA6F8CE2114310410
:1078700009F02BCF019690931402809313022F8D61
:1078800038A149A15AA1420E531E641E751ED30190
:10789000C201B595A795979587958BAB9CABADAB82
:1078A000BEAB01CFEFEF8E1A9E0AAE0ABE0A25CFFD
:1078B000029709F07DCFC092AA10D092AB10E0924F
:1078C000AC10F092AD10C0922502D0922602E09248
:1078D0002702F09228026CCF69EB75E0CE01019689
:1078E0000E94417CCE0101960E94071BCE010196A9
:1078F0000E94B47B40912D0250912E0260912F0284
:107900007091300225E0CE0101960E94BC7BCE0131
:1079100001960E94F01ACE0101960E94B47B75CFA9
:1079200020E030E0A901C701B6010E94C7AB87FF84
:107930000BC020E030E044EB53E4C701B6010E94E5
:1079400075AD6B017C01ECCFC0925B0BD0925C0BF0
:10795000E0925D0BF0925E0B4FA058A469A47AA44C
:107960008BA19CA1ADA1BEA1481A590A6A0A7B0A43
:1079700021143104D9F410925B0B10925C0B10921D
:107980005D0B10925E0BADA5BEA5C12CD12C76016E
:10799000C394812C912C5401B7FF1CC0812C912CD5
:1079A0005401CC24CA94DC2C760114C0EDA5FEA5AC
:1079B000C12CD12C7601C394F7FF04C0CC24CA9407
:1079C000DC2C760180905B0B90905C0BA0905D0BA3
:1079D000B0905E0B20912D0230912E0240912F022B
:1079E00050913002C501B4010E942DAC4B015C01E5
:1079F000A3019201C701B6010E9401AD0E94CEAB66
:107A000020E030E040E05FE30E942DAC9B01AC0140
:107A1000C501B4010E9474AD0E9453AE6093190277
:107A200070931A0280931B0290931C0280916D0B3D
:107A3000882309F441C02AE04FA158A569A57AA579
:107A4000CE010D960E94F27B2AE04BA15CA16DA1B4
:107A50007EA1CE0107960E94F27B68E575E0CE011B
:107A600001960E94537CBE01695F7F4FCE01019653
:107A70000E94CF7A60E476E00E94B97ABE01635F2B
:107A80007F4F0E94CF7ABC01CE0143960E944A7C70
:107A9000CE0143960E94F01ACE0143960E94B47B19
:107AA000CE0101960E94B47BCE0107960E94B47B62
:107AB000CE010D960E94B47B8091190290911A021A
:107AC000A0911B02B0911C02E12C12E5B7FFAACBDA
:107AD000B095A095909581959F4FAF4FBF4F8093E4
:107AE000190290931A02A0931B02B0931C02EE2479
:107AF000E394F12C16E496CBEE24E394F12CA6CB80
:107B0000E12CA4CB22E02216310424F42114310408
:107B100009F0E1C061E080E00E945C8932E0231658
:107B2000310424F42114310409F09CC0C090960B58
:107B3000D090970BE090980BF090990B20E030E0FC
:107B400044EB53E4C701B6010E9489AE87FD0BC028
:107B500020E030E044EB53E4C701B6010E9474AD6D
:107B60006B017C01EBCF20E030E0A901C701B60139
:107B70000E94C7AB87FF0BC020E030E044EB53E42A
:107B8000C701B6010E9475AD6B017C01ECCFC092BC
:107B9000960BD092970BE092980BF092990B8091F4
:107BA0006C0290916D020197B1F461E175E083EE92
:107BB0009EE00E9497798091960B9091970BA091EF
:107BC000980BB091990B8093E10B9093E20BA093EB
:107BD000E30BB093E40B80916C0290916D020297DD
:107BE000B1F461E275E083EE9EE00E9497798091A6
:107BF000960B9091970BA091980BB091990B809355
:107C0000DD0B9093DE0BA093DF0BB093E00B409164
:107C1000960B5091970B6091980B7091990B20E007
:107C2000CE0107960E94BC7B63EE7EE0CE010196FA
:107C30000E944A7CBE01695F7F4FCE0101960E947F
:107C4000CF7A6DE175E00E94B97ABC0183EE9EE0C7
:107C50000E94647BCE0101960E94B47BCE01079600
:107C60000E94B47B41E02416310439F54091190299
:107C700050911A0260911B0270911C0221E0CE010A
:107C800007960E94F27B60E675E0CE0101960E94A5
:107C9000537CBE01695F7F4FCE0101960E94CF7A6F
:107CA000BC0183EE9EE00E94647BCE0101960E949F
:107CB000B47BCE0107960E94B47B63EE7EE0CE01DA
:107CC00001960E944A7CCE0101960E948E27CE0129
:107CD00001960E94B47B1092190210921A0210921F
:107CE0001B0210921C0280916C0290916D028130F7
:107CF000910509F083C08091650B9091660B90937C
:107D0000680B8093670B8091190290911A02A091E1
:107D10001B02B0911C0280931D0290931E02A0933F
:107D20001F02B09320028091390290913A02A091F3
:107D30003B02B0913C028093350290933602A093AF
:107D40003702B09338028091630B8093640B80916B
:107D50005B0B90915C0BA0915D0BB0915E0B8093DF
:107D60005F0B9093600BA093610BB093620B8091BB
:107D7000960B9091970BA091980BB091990B8093D3
:107D8000E10B9093E20BA093E30BB093E40B809193
:107D900013029091140290931602809315022328E7
:107DA00081F480912D0290912E02A0912F02B0912A
:107DB00030028093290290932A02A0932B02B09361
:107DC0002C02CE0149960E94B47BEC960FB6F89433
:107DD000DEBF0FBECDBFDF91CF911F910F91FF90FE
:107DE000EF90DF90CF90BF90AF909F908F907F905B
:107DF0006F905F904F903F902F900895029709F7F2
:107E00008091650B9091660B90935A0B8093590B60
:107E10008091190290911A02A0911B02B0911C024C
:107E200080930F0290931002A0931102B09312025C
:107E30008091390290913A02A0913B02B0913C02AC
:107E40008093310290933202A0933302B0933402B4
:107E50008091630B8093580B80915B0B90915C0B2E
:107E6000A0915D0BB0915E0B8093540B9093550BDA
:107E7000A093560BB093570B8091960B9091970B54
:107E8000A091980BB091990B8093DD0B9093DE0B32
:107E9000A093DF0BB093E00B80911302909114023A
:107EA00090930E0280930D02232809F08ACF8091CF
:107EB0002D0290912E02A0912F02B091300280935A
:107EC000250290932602A0932702B093280279CF2F
:107ED0006F927F928F929F92AF92BF92CF92DF92DA
:107EE000EF92FF920F931F93CF93DF93CDB7DEB73F
:107EF000C456D1090FB6F894DEBF0FBECDBF40E027
:107F000052EC61E070E085E29DE00E94347640E84A
:107F100055E260E070E088E89CE00E94347661E021
:107F200088E00E94EA7E61E089E00E94EA7E60E0EB
:107F30008AE30E94EA7E61E088E00E94877E60E03A
:107F400089E00E94877E61E08AE00E94EA7E61E02B
:107F50008BE00E94EA7E60E08BE30E94EA7E61E0B3
:107F60008AE00E94877E60E08BE00E94877E0E940C
:107F7000D37E84EF91E0909367028093660262EC77
:107F80007AE085E29DE00E94977D67E779E085E2EF
:107F90009DE00E94B47C60ED77E080E090E00E947C
:107FA000407F85E29DE00E94EA72982E0EE110E08B
:107FB00091100BC085E29DE00E94EA72982E6EE15E
:107FC00070E080E090E00E94407F0150110981F74D
:107FD000809166029091670208E81FE09C01285892
:107FE0003F407901C701800F911F0E94EBACF8015F
:107FF00081938F01F0E10A3B1F07A1F76091A21066
:108000007091A310072E000C880B990B0E94CEAB29
:108010009B01AC010E948EAE882331F081E090E09C
:108020009093A3108093A2106091A4107091A5105A
:10803000072E000C880B990B0E94CEAB9B01AC0164
:108040000E948EAE882331F082E090E09093A510DC
:108050008093A41025E79216B1F060919E10709164
:108060009F108091A0109091A1100E94CEAB9B0117
:10807000AC010E948EAE811106C08091880F909154
:10808000890F8197E8F08DB79EB7825391400FB664
:10809000F8949EBF0FBE8DBFADB7BEB7119682E3F9
:1080A00091E0E8E8FFE001900D920197E1F70E946E
:1080B0003A2C0FB6F894DEBF0FBECDBF05E7902E69
:1080C0002DB73EB7225331400FB6F8943EBF0FBED6
:1080D0002DBFADB7BEB7119682E391E0E8E8FFE0AF
:1080E00001900D920197E1F70E9440240FB6F89499
:1080F000DEBF0FBECDBF95E7991619F0E3E79E12DC
:108100001BC02DB73EB7225331400FB6F8943EBF87
:108110000FBE2DBFADB7BEB7119682E391E0E8E880
:10812000FFE001900D920197E1F70E94BB320FB67C
:10813000F894DEBF0FBECDBF60EB7AE08AE39FE02C
:108140000E943F7B6AE97AE084E39FE00E943F7BE4
:108150000E94D37E17E2C12ED12CE12CF12C10E02D
:1081600000E0BB24B394B092830CC092850C1092B3
:10817000840C1092860C81E00E942E8881114FC1E0
:10818000C09242110F5F1F4F9FEFC91AD90AE90A27
:10819000F90AE0E4CE16D104E104F10421F7012B41
:1081A00031F462E875E085E29DE00E94597D0E940D
:1081B000D37E1092431180914711823018F098E0DD
:1081C0009093431190914811992339F0813029F40B
:1081D0008091431184608093431162E370E080E0FA
:1081E00090E00E94407F609149118EE391E10E94EE
:1081F0001E8968EE73E080E090E00E94407F60E3BB
:108200008EE391E10E9432890BE416E4C8010197E4
:10821000F1F760E38EE391E10E943289C801019792
:10822000F1F760E38EE391E10E94328983E592E009
:108230000197F1F760E28EE391E10E94328980912B
:10824000431180620E944B8984E0809344118CE04A
:108250000E944B8981E00E944B890BE31FE1C8011A
:108260000197F1F782E08093451186E00E944B89E7
:1082700082E00E944B89C8010197F1F780E40E94D7
:108280004B890EE512E0F80161918F018EE391E1D7
:108290000E948989F2E006361F07A9F70E94010AA9
:1082A0000E94F10964E670E080E090E00E94407F67
:1082B00062E87AE0CE0101960E94417CCE010196EF
:1082C0000E94F01ACE0101960E94B47B61E085E322
:1082D0000E94EA7E61E085E30E94877E61E08AE099
:1082E0000E94EA7E61E08AE00E94877E68EC70E08E
:1082F00080E090E00E94407F68EE73E080E090E0D4
:108300000E94407F61E77AE0CE0101960E94417CA5
:108310004AE050E06FEF7FEFCE0101960E94B92650
:10832000CE0101960E94B47B1092D90D1092D70D08
:108330001092D40D1092D30D84E08093D20D0E9440
:108340000F828B0161E08091D20D0E94EA7E8EEC5B
:108350009DE00E949B0860E082E30E94EA7E61E06B
:1083600083E30E94EA7E61E084E30E94EA7E61E0AA
:1083700085E30E94EA7E61E085E30E94877E83E5D3
:108380008CBD8DB58E7F8DBDBAE0FB2E8FEF0E9428
:108390009007FA94F110FACF60E08091D20D0E941C
:1083A000877E20E030E0A90160E08EEC9DE00E9435
:1083B0009A0BF82E8093D80D21E0821709F446C05D
:1083C0000E940F82601B710B613D774050F381E08A
:1083D0008093D30D8EEC9DE00E949B0863E67AE0CB
:1083E000CE0101960E94417CCE0101960E94F01AB6
:1083F000CE0101960E94B47B62E57AE0CE0101963F
:108400000E94417C4AE050E06FEF7FEFCE01019681
:108410000E94250ACE0101960E94B47B2CC18430B3
:1084200009F0B2CE67E675E085E29DE00E946D7DC1
:1084300020E1B701A60185E29DE00E94C37C67E7C9
:1084400079E085E29DE00E94B47C9ECE2AEA31E08C
:1084500040E050E068E08EEC9DE00E949A0B82FFC5
:108460002AC0F092D90D8091D90DC12CD12CE12CCC
:10847000F0E4FF2E823019F0C12CD12C760120E0DF
:1084800030E0A90167E38EEC9DE00E949A0BA70102
:10849000960169E28EEC9DE00E949A0B8093D80DC4
:1084A0008823D1F00E940F82601B710B613D7740E1
:1084B00030F388E08DCFA4E0FA2E0E94950B8093D4
:1084C000D80DFA94F110F9CF8A3A11F082E080CFFA
:1084D00082E08093D90DC7CF8091D90D8230D1F43D
:1084E00020E030E0A9016AE38EEC9DE00E949A0B47
:1084F000882311F086E06CCF0E94950B807C803C35
:1085000019F483E08093D90D0E94950B0E94950B7E
:108510000E94950B8EEC9DE00E949B088DB58E7F8E
:108520008DBD8CB58C7F8CBD8CB58CBD81E00E94DF
:108530008877882309F4AAC28091FD0D81114ECF5E
:108540008091F10D803109F0A8C282E08093FD0D89
:1085500010920F0E1092100E1092110E1092120E19
:108560008091F20D9091F30DB0E0A0E0E5E0880F6E
:10857000991FAA1FBB1FEA95D1F780930B0E90930A
:108580000C0EA0930D0EB0930E0E8AED9DE090930D
:10859000140E8093130E81E08093FC0D1092FE0D5B
:1085A0001092FF0D1092000E1092010E1092020E0A
:1085B0001092030E1092040E1092050E1092060EE9
:1085C0001092070E1092080E1092090E10920A0EC9
:1085D00066E47AE0CE0101960E94417CCE010196CC
:1085E0000E94F01ACE0101960E94B47B41E068E639
:1085F00074E0CE0101960E941692BE016F5F7F4F1C
:1086000087E091E10E94171E8091091190910A1153
:108610009C838B8380910B1190910C11A0910D1173
:10862000B0910E118D839E83AF83B88780910F1117
:1086300090911011A0911111B091121189879A8710
:10864000AB87BC8784EF93E09A8389838DE0E3E175
:10865000F1E1DE011D9601900D928A95E1F780917E
:108660002011909121119B8F8A8F70E060E0CE01E4
:1086700001960E94E81E68EE73E080E090E00E94A0
:10868000407F43E162EB72E0CE0101960E941692B8
:10869000BE016F5F7F4F82E291E10E94171E6DE085
:1086A0007AE088E29FE00E943F7B62E07AE088E225
:1086B0009FE00E94E27A82E291E10E94500D8823BD
:1086C00009F41CC21EAE1DAE84E793E09CAF8BAFD5
:1086D00021961FAE219719A218A29F8F8E8F1BA2E1
:1086E000812C712C7E019BE3E90EF11C08EF1DE04B
:1086F00074E7A72E73E0B72E882D972DFC01EE545A
:10870000FD4F20812F3209F40196DC01AE54BD4F9C
:10871000FE01E85AFF4F30E020E06F014D914F32EB
:1087200049F0442339F001962F5F3F4F41932C309D
:108730003105A1F72C0D3D1DF9011082FC01EE540D
:10874000FD4F20812F3209F40196882E792E8E5408
:108750009D4FFC0160801C821B82BA82A9821E820E
:1087600021E0A601B801CE0101960E946C908823F9
:1087700009F4E1C1CE0101960E948F0A6110ACC1DB
:108780002DE0083F120719F0C8010E948F0A82E20B
:1087900091E10E945C0D66E970E080E090E00E944B
:1087A000407F10924E0C04E610E091100BC085E261
:1087B0009DE00E94EA72982E64E170E080E090E013
:1087C0000E94407F0150110981F76DED79E0CE01E3
:1087D00001960E94417C48EC50E070E060E0CE01E0
:1087E00001960E94250ACE0101960E94B47B32E7D1
:1087F00081E0931280E00E94800982E090E00E9474
:10880000F5856CE271E080E090E00E94407F83E0BB
:1088100090E00E94F5856CE271E080E090E00E94BB
:10882000407F01E010E010936D0200936C02109302
:108830005D0200935C026AEA75E08DED9EE00E94A5
:1088400097796DED7EE0CE0101960E944A7C62E050
:1088500070E0CE0101960E94ED36CE0101960E9495
:10886000B47B6CEC79E0CE0101960E94417CCE0194
:1088700001960E94F01ACE0101960E94B47B64E634
:1088800070E080E090E00E94407F6CEB79E0CE01E8
:1088900001960E94417C48EC50E070E060E0CE011F
:1088A00001960E94B926CE0101960E94B47B62ED2A
:1088B00076E08DED9EE00E94977962E370E080E0C3
:1088C00090E00E94407F6DED7EE0CE0101960E9417
:1088D0004A7C63E070E0CE0101960E94ED36CE0145
:1088E00001960E94B47B10936D0200936C0266EABD
:1088F00079E0CE0101960E94417CCE0101960E9452
:10890000F01ACE0101960E94B47B6BE979E0CE01AA
:1089100001960E94417C4AE050E06FEF7FEFCE016C
:1089200001960E94B926CE0101960E94B47B68EEA2
:1089300073E080E090E00E94407F0E94922F0E94AE
:108940009A301092F70B85E29BE69093920E8093FB
:10895000910E2091B30E2830D8F4822F90E0FC01C4
:10896000EE0FFF1FEE0FFF1FED56F14F4EEA55E0E1
:10897000518340832F5F2093B30E880F991F880F78
:10898000991FFC01EB56F14F88E690E291838083BA
:108990002091B30E2830D8F4822F90E0FC01EE0F26
:1089A000FF1FEE0FFF1FED56F14F44EB55E05183D3
:1089B00040832F5F2093B30E880F991F880F991F54
:1089C000FC01EB56F14F8BEB91E79183808381E2C1
:1089D0009EE00E94E61869E879E0CE0101960E94C7
:1089E000417CCE0101960E94F01ACE0101960E94B0
:1089F000B47B8DB79EB7825391400FB6F8949EBF5B
:108A00000FBE8DBFADB7BEB7119682E391E0E8E827
:108A1000FFE001900D920197E1F70E94BB321092A6
:108A2000F80B0FB6F894DEBF0FBECDBF0E94AF8526
:108A30006093F90B7093FA0B8093FB0B9093FC0BF4
:108A4000809187108093500C882351F00E94AF854D
:108A50006093EF0B7093F00B8093F10B9093F20BFC
:108A6000CC59DF4F0FB6F894DEBF0FBECDBFDF91FC
:108A7000CF911F910F91FF90EF90DF90CF90BF901B
:108A8000AF909F908F907F906F90089580E00E94AC
:108A90008877882309F4A2CC4FCD803209F09ECC90
:108AA00083E08093FD0D4091F40D5091F50D6091A0
:108AB000F60D7091F70D40930F0E5093100E6093CA
:108AC000110E7093120E2BE03EE08AED9DE00E94A5
:108AD0001F8C81115ACD82CC21E0A601B801C701BB
:108AE0000E946C90D82EFDE0083F1F0709F44DC08E
:108AF000C8010E948F0AD1104DC024C06DEE79E0EC
:108B0000CE0101960E94417CCE0101960E94071B76
:108B1000CE0101960E94B47B62EB72E0CE01019619
:108B20000E94537CCE0101960E94F01ACE0101965C
:108B30000E94B47B36CEFDE0083F1F0719F0C80144
:108B40000E948F0A68E975E0CE0101960E94537C6D
:108B5000CE0101960E94071BCE0101960E94B47BB4
:108B600062EB72E0CE0101960E94537CCE01019629
:108B70000E94F01ACE0101960E94B47B68E27FE069
:108B800082E291E10E94837D02CE8823D9F28E0198
:108B9000025E1F4F902F812F8701E92EF82EACCD5A
:108BA0002F923F924F925F926F927F928F929F92FD
:108BB000AF92BF92CF92DF92EF92FF920F931F93EB
:108BC000CF93DF93CDB7DEB7E3970FB6F894DEBF50
:108BD0000FBECDBF61E07FE0CE018E960E944A7C41
:108BE0000EA51FA50115110571F0D8018D918D01FC
:108BF000882349F0082E000C990B0E94D5B0F8018B
:108C000031978083F2CF68EB75E0CE0101960E9428
:108C1000537CBE016F5F7F4FCE018E960E949E7A7D
:108C2000182FCE0101960E94B47B112309F401C1D3
:108C300045E050E061E07FE0CE0101960E94A61E73
:108C4000BE016F5F7F4F8DED9EE00E947B7BCE016A
:108C500001960E94B47B8DED9EE00E94107A60E048
:108C60008DED9EE00E940C7B4091E10E5091E20E52
:108C700060EE7FE08DED9EE00E94507768E674E044
:108C8000CE0101960E94537CBE016F5F7F4F8DED38
:108C90009EE00E949E7A182FCE0101960E94B47B1E
:108CA00062E574E0111102C067E574E0CE0101963F
:108CB0000E94537C6DED7EE0CE0101960E94CF7A3A
:108CC000BC0186EE90E10E94647BCE0101960E9479
:108CD000B47B86EE90E10E94107A4091EA105091A8
:108CE000EB104150510966EE70E1CE0101960E94F1
:108CF000A61EBE016F5F7F4F88EC90E10E947B7BD8
:108D0000CE0101960E94B47B88EC90E10E94057A26
:108D10000E94CEAB9B01AC010E948EAE882309F469
:108D200048C06091EA107091EB106250710986EEB4
:108D300090E10E946D7A682FCE0101960E941F7CFF
:108D4000BE016F5F7F4F88EC90E10E947B7BCE017C
:108D500001960E94B47B68E674E0CE0101960E9401
:108D6000537CBE016F5F7F4F88EC90E10E949E7A3A
:108D7000182FCE0101960E94B47B1123D1F060918F
:108D8000EA107091EB106350710986EE90E10E9439
:108D90006D7A682FCE0101960E941F7CBE016F5F25
:108DA0007F4F88EC90E10E947B7BCE0101960E9470
:108DB000B47B84EF91E0909367028093660268E849
:108DC0007FE00E944F0964E670E080E090E00E943E
:108DD000407F80913D02882371F061E07FE0CE0109
:108DE00001960E944A7CCE0101960E945C21CE0130
:108DF00001960E94B47BCE018E960E94B47B81E0E6
:108E0000E3960FB6F894DEBF0FBECDBFDF91CF91D2
:108E10001F910F91FF90EF90DF90CF90BF90AF9098
:108E20009F908F907F906F905F904F903F902F908A
:108E300008956EEB75E0CE0101960E94537CBE0151
:108E40006F5F7F4FCE018E960E949E7A182FCE01C3
:108E500001960E94B47B112309F447C045E050E01D
:108E600061E07FE0CE0101960E94A61EBE016F5F09
:108E70007F4F8DED9EE00E947B7BCE0101960E948C
:108E8000B47B8DED9EE00E94107A60E08DED9EE057
:108E90000E940C7B4091E10E5091E20E68EB7FE066
:108EA0008DED9EE00E94507768EB7FE0CE014C96FE
:108EB0000E94537C6AE674E0CE0101960E94537CC6
:108EC000BE01645E7F4FCE0101960E94CF7ABC0145
:108ED00080EE90E10E94647BCE0101960E94B47BFB
:108EE000CE014C960E94B47B64CF64EC75E0CE0159
:108EF00001960E94537CBE016F5F7F4FCE018E961C
:108F00000E949E7A182FCE0101960E94B47B1123F5
:108F1000E1F043E050E061E07FE0CE0101960E9485
:108F2000A61EBE016F5F7F4F8DED9EE00E947B7B92
:108F3000CE0101960E94B47B6DED7EE0CE010196DC
:108F40000E944A7CCE010196CDCF68EC75E0CE013F
:108F500001960E94537CBE016F5F7F4FCE018E96BB
:108F60000E949E7A182FCE0101960E94B47B112395
:108F700001F144E050E061E07FE0CE0101960E9403
:108F8000A61EBE016F5F7F4F8DED9EE00E947B7B32
:108F9000CE0101960E94B47B8DED9EE00E94057A81
:108FA000709347106093461070938D0260938C020B
:108FB00000CF6DEC75E0CE0101960E94537CBE019E
:108FC0006F5F7F4FCE018E960E949E7A182FCE0142
:108FD00001960E94B47B112309F449C045E050E09A
:108FE00061E07FE0CE0101960E94A61EBE016F5F88
:108FF0007F4F8DED9EE00E947B7BCE0101960E940B
:10900000B47B8DED9EE00E94057A7093A31060936F
:10901000A21084EF91E0909367028093660268E863
:109020007FE00E944F0964E670E080E090E00E94DB
:10903000407F68EC77E0CE0101960E94537C61E0AE
:109040007FE0CE0101960E94CF7ABC01CE014C9602
:109050000E944A7CCE014C960E94F01ACE014C969A
:109060000E94B47BCE0101960E94B47BB2CE63ED28
:1090700075E0CE0101960E94537CBE016F5F7F4F69
:10908000CE018E960E949E7A182FCE0101960E94E4
:10909000B47B1123E1F044E050E061E07FE0CE01D9
:1090A00001960E94A61EBE016F5F7F4F8DED9EE070
:1090B0000E947B7BCE0101960E94B47B8DED9EE0E9
:1090C0000E94057A7093A5106093A410A2CF68ED5A
:1090D00075E0CE0101960E94537CBE016F5F7F4F09
:1090E000CE018E960E949E7A182FCE0101960E9484
:1090F000B47B1123A1F044E050E061E07FE0CE01B9
:1091000001960E94A61EBE016F5F7F4F8DED9EE00F
:109110000E947B7BCE0101960E94B47B84CF6DEDD3
:1091200075E0CE0101960E94537CBE016F5F7F4FB8
:10913000CE018E960E949E7A182FCE0101960E9433
:10914000B47B1123A1F047E050E061E07FE0CE0165
:1091500001960E94A61EBE016F5F7F4F8DED9EE0BF
:109160000E947B7BCE0101960E94B47B2CCE65EEE3
:1091700075E0CE0101960E94537CBE016F5F7F4F68
:10918000CE018E960E949E7A182FCE0101960E94E3
:10919000B47B1111D8CF6DEE75E0CE0101960E941F
:1091A000537CBE016F5F7F4FCE018E960E949E7AE8
:1091B000182FCE0101960E94B47B112321F081E08B
:1091C0000E94800900CE67EF75E0CE0101960E94F3
:1091D000537CBE016F5F7F4FCE018E960E949E7AB8
:1091E000182FCE0101960E94B47B112319F00E9422
:1091F000922FE9CD6FE779E0CE0101960E94417C84
:10920000BE016F5F7F4FCE018E960E949E7A182F0F
:10921000CE0101960E94B47B112309F485C064E756
:1092200079E0CE0101960E94417CBE016F5F7F4FC5
:10923000CE018E960E949E7A182FCE0101960E9432
:10924000B47B112309F454C04AE050E061E07FE0B0
:10925000CE0101960E94A61EBE016F5F7F4F8DED6D
:109260009EE00E947B7BCE0101960E94B47B8DED37
:109270009EE00E94057A0E948A850E94AF856093D5
:10928000EF0B7093F00B8093F10B9093F20B0E9415
:10929000AF856093E90B7093EA0B8093EB0B90938F
:1092A000EC0BCE014C960E9409226EEF75E0CE01C8
:1092B00001960E94537CBE01645E7F4FCE010196F1
:1092C0000E94CF7ABC01CE0182960E944A7CCE01D8
:1092D00082960E94F01ACE0182960E94B47BCE0143
:1092E00001960E94B47BCE014C960E94B47B71CD56
:1092F0004BE050E061E07FE0CE0101960E94A61EA7
:10930000BE016F5F7F4F8DED9EE00E947B7BCE01A3
:1093100001960E94B47B8DED9EE00E94057A605814
:109320007F488F4F9F4FA7CF64E477E0CE0101962F
:109330000E94537CBE016F5F7F4FCE018E960E94CC
:109340009E7A182FCE0101960E94B47B112309F456
:109350006AC045E050E061E07FE0CE0101960E94E6
:10936000A61EBE016F5F7F4F8DED9EE00E947B7B4E
:10937000CE0101960E94B47B0E94AF856093EF0BF3
:109380007093F00B8093F10B9093F20B8DED9EE0B8
:109390000E94057A60936E0270936F028093700250
:1093A00090937102609388107093891080938A1053
:1093B00090938B10209187102093500C672B682B73
:1093C000692B11F41092500C84EF91E09093670296
:1093D0008093660268E87FE00E944F0964E670E0CF
:1093E00080E090E00E94407F65E679E0CE01019642
:1093F0000E94417CCE0101960E94071BCE0101967E
:109400000E94B47B40916E0250916F026091700295
:1094100070917102CE0101960E94CD79CE01019624
:109420000E94F01ADBC16FE076E0CE0101960E9447
:10943000537CBE016F5F7F4FCE018E960E949E7A55
:10944000182FCE0101960E94B47B1123D9F14AE076
:1094500050E061E07FE0CE0101960E94A61EBE01B1
:109460006F5F7F4F8DED9EE00E947B7BCE0101966A
:109470000E94B47B8DED9EE00E94057A61307105FB
:109480008105910519F481E0809387108DED9EE0B0
:109490000E94057A672B682B692B11F410928710B4
:1094A000809187108093500C882309F4B2CD0E94DC
:1094B000AF856093EF0B7093F00B8093F10B90935B
:1094C000F20BA7CD6AE176E0CE0101960E94537CB3
:1094D000BE016F5F7F4FCE018E960E949E7A182F3D
:1094E000CE0101960E94B47B1123A1F048E050E028
:1094F00061E07FE0CE0101960E94A61EBE016F5F73
:109500007F4F8DED9EE00E947B7BCE0101960E94F5
:10951000B47B8FCD63E276E0CE0101960E94537C4E
:10952000BE016F5F7F4FCE018E960E949E7A182FEC
:10953000CE0101960E94B47B112321F145E050E059
:1095400061E07FE0CE0101960E94A61EBE016F5F22
:109550007F4F8DED9EE00E947B7BCE0101960E94A5
:10956000B47B8DED9EE00E94057A6130710521F497
:1095700081E08093510C2DCC672B09F02ACC1092FE
:10958000510C27CC69E276E0CE0101960E94537C13
:10959000BE016F5F7F4FCE018E960E949E7A182F7C
:1095A000CE0101960E94B47B112351F163E070E07B
:1095B00081E09FE00E946D7A682FCE0101960E94A3
:1095C0001F7CBE016F5F7F4F8DED9EE00E947B7B15
:1095D000CE0101960E94B47B8DED9EE00E94107A30
:1095E0008DED9EE00E94057A9B01215031092330C8
:1095F000310508F0EECB7093B7106093B610D9CB5D
:109600006DE276E0CE0101960E94537CBE016F5F51
:109610007F4FCE018E960E949E7A182FCE01019622
:109620000E94B47B112309F46AC066E070E081E017
:109630009FE00E946D7A682FCE0101960E941F7CE8
:10964000BE016F5F7F4F8DED9EE00E947B7BCE0160
:1096500001960E94B47B8DED9EE00E94107A60E03E
:109660008DED9EE00E940C7B8DED9EE00E94057AC0
:109670006B01CB010197039708F0ABCB48E050E0BA
:1096800061E07FE0CE0101960E94A61EBE016F5FE1
:109690007F4F8DED9EE00E947B7BCE0101960E9464
:1096A000B47B8DED9EE00E94107A8091E10E909146
:1096B000E20E0997A8F028E030E050E040E06DEDC0
:1096C0007EE0CE0101960E94687CBE016F5F7F4FF5
:1096D0008DED9EE00E947B7BCE0101960E94B47BC3
:1096E000B60113E0660F771F1A95E1F76456704FC5
:1096F00048E050E08DED9EE00E9450775ACB6DE53A
:1097000079E0CE0101960E94417CBE016F5F7F4FE0
:10971000CE018E960E949E7A182FCE0101960E944D
:10972000B47B112309F486C06DE174E0CE0101968B
:109730000E94537C47E050E0BE01625D7F4FCE0146
:109740004C960E94A61EBE01645E7F4FCE0101961C
:109750000E947B7BCE014C960E94B47B62E075E058
:10976000CE014C960E94537CBE01645E7F4FCE01B9
:1097700001960E949E7A182FCE014C960E94B47BCF
:10978000112379F141E050E0BE016F5F7F4FCE01C0
:109790004C960E94A61ECE014C960E94057A8B0123
:1097A0000A5C1F4FCE014C960E94B47B1093B910F7
:1097B0000093B81010938F0200938E0284EF91E013
:1097C000909367028093660268E87FE00E944F09E9
:1097D00064E670E080E090E00E94407FCE01019658
:1097E00084CD6DEB76E0CE014C960E94537CBE0199
:1097F000645E7F4FCE0101960E949E7A182FCE01A3
:109800004C960E94B47B112379F041E050E0BE01F8
:109810006F5F7F4FCE014C960E94A61ECE014C96E4
:109820000E94057A8B01BECFCE0101960E94057A77
:109830008B01BCCF66E579E0CE0101960E94417CA8
:10984000BE016F5F7F4FCE018E960E949E7A182FC9
:10985000CE0101960E94B47B112309F4AAC063E4EF
:1098600076E0CE0101960E94537C46E050E0BE01B6
:109870006F5F7F4FCE018E960E94A0A18C01CE011A
:1098800001960E94B47B980146E050E0BE01625D03
:109890007F4FCE0101960E94687CCE0101960E9406
:1098A000057A6B01CE0101960E94B47B6DE174E0F4
:1098B000CE0101960E94537CA8014F5F5F4FBE010D
:1098C000625D7F4FCE014C960E94A61EBE01645E73
:1098D0007F4FCE0101960E947B7BCE014C960E9469
:1098E000B47B62E075E0CE014C960E94537CBE01D1
:1098F000645E7F4FCE0101960E949E7A182FCE01A2
:109900004C960E94B47B112321F141E050E0BE014E
:109910006F5F7F4FCE014C960E94A61ECE014C96E3
:109920000E94057A8B010A5C1F4FCE014C960E9463
:10993000B47BF6013196EE0FFF1FE857F04F11830D
:109940000083F601EE0FFF1FE655F44F11830083ED
:1099500035CF6DEB76E0CE014C960E94537CBE0174
:10996000645E7F4FCE0101960E949E7A182FCE0131
:109970004C960E94B47B112379F041E050E0BE0187
:109980006F5F7F4FCE014C960E94A61ECE014C9673
:109990000E94057A8B01C9CFCE0101960E94057AFB
:1099A0000091AC0B1091AD0B01501109060F171F60
:1099B000C0CF67E374E0CE014C960E94537CBE0199
:1099C000645E7F4FCE018E960E949E7A11E08111D7
:1099D00015C064E376E0CE0101960E94537CBE017F
:1099E0006F5F7F4FCE018E960E949E7A11E08111AB
:1099F00001C010E0CE0101960E94B47BCE014C96CE
:109A00000E94B47B112309F411C260E476E0CE0118
:109A10004C960E94537C6BE376E0CE0101960E9447
:109A2000537CAE01445E5F4FBE016F5F7F4FCE013E
:109A30008E960E94A7A0CE0101960E94B47BCE0113
:109A40004C960E94B47B60E476E0CE014C960E9476
:109A5000537C6DE376E0CE0101960E94537CAE010B
:109A6000445E5F4FBE016F5F7F4FCE018E960E94B6
:109A7000A7A0CE0101960E94B47BCE014C960E9415
:109A8000B47B60E476E0CE014C960E94537C6FE399
:109A900076E0CE0101960E94537CAE01445E5F4F9A
:109AA000BE016F5F7F4FCE018E960E94A7A0CE01B0
:109AB00001960E94B47BCE014C960E94B47B63E475
:109AC00076E0CE014C960E94537C62E476E0CE01B3
:109AD00001960E94537CAE01445E5F4FBE016F5FF2
:109AE0007F4FCE018E960E94A7A0CE0101960E94C4
:109AF000B47BCE014C960E94B47B63E476E0CE0149
:109B00004C960E94537C6CE678E0CE0101960E9450
:109B1000537CAE01445E5F4FBE016F5F7F4FCE014D
:109B20008E960E94A7A0CE0101960E94B47BCE0122
:109B30004C960E94B47BCE018E960E94107A0E94B1
:109B4000AF856093F30B7093F40B8093F50B9093B8
:109B5000F60B56E0E52EF12C64E6462E512C612CD6
:109B6000712C22242394312C5701B3E0AB0EB11C8D
:109B70008AA99BA90197A816B90608F02AC9B701B6
:109B8000CE018E960E946D7A682FCE014C960E946F
:109B90001F7C6701E2E0CE0ED11CFFEFEF1AFF0A37
:109BA0009601A701BE01625D7F4FCE0101960E9422
:109BB000687CCE0101960E94057A8B01CE01019648
:109BC0000E94B47B0130110521F40091A210109184
:109BD000A3100330110521F40091A4101091A510D9
:109BE00060E476E0CE0101960E94537CA601BE019E
:109BF0006F5F7F4FCE018E960E94A0A16C01CE01B7
:109C000001960E94B47B6DE174E0CE0101960E9442
:109C1000537C480181E0881A91081C141D042CF51E
:109C20009601A501BE01625D7F4FCE0182960E9422
:109C3000687CBE016E5D7F4FCE0101960E947B7BEA
:109C4000CE0182960E94B47B93E08916910420F1A4
:109C50007601AFEFEA1AFA0ACE0101960E94B47BB0
:109C6000CE014C960E94B47B7FCFA501BE01625D00
:109C70007F4FCE0182960E94A61EBE016E5D7F4F71
:109C8000CE0101960E947B7BCE0182960E94B47B1E
:109C9000B3E08B16910400F770E060E0CE014C96C3
:109CA0000E946D7A823509F061C0CE0101960E9452
:109CB000057A672B682B692BB1F4F801EE0FFF1FB3
:109CC000E952FD4F11821082F801EE0FFF1FEE0FD7
:109CD000FF1FE154FD4F82E090E0A0E0B0E0808300
:109CE0009183A283B383CE0101960E94057A6130ED
:109CF000710581059105A9F5F801EE0FFF1FE952E5
:109D0000FD4F31822082000F111F000F111FF8013B
:109D1000E154FD4F80819181A281B381181619060B
:109D20001A061B0624F04082518262827382CE01A1
:109D300001960E94057A62307105810591053CF01B
:109D4000F801E154FD4F60837183828393830E9405
:109D5000AF8501521D4FD8016D937D938D939C93D8
:109D600013971C141D040CF473CF76CF8634E9F5D9
:109D7000CE0101960E94057A672B682B692B39F476
:109D8000F801EE0FFF1FEC5AFD4F11821082CE0139
:109D900001960E94057A613071058105910539F4BB
:109DA000F801EE0FFF1FEC5AFD4F31822082000FA9
:109DB000111F000F111FF801E154FD4F80819181A7
:109DC000A281B381181619061A061B0624F04082D8
:109DD0005182628273820E94AF8501521D4FF80149
:109DE0006083718382839383BCCF843461F4CE011A
:109DF00001960E94057A000F111F000F111FF80134
:109E0000EC5BFD4FA0CF843509F0ABCFCE010196BE
:109E10000E94057A000F111F000F111FF801E15475
:109E2000FD4F6083718382839383D5CF60E579E0B2
:109E3000CE0101960E94417CBE016F5F7F4FCE0133
:109E40008E960E949E7A182FCE0101960E94B47BB6
:109E5000112309F49DC045E050E061E07FE0CE01B0
:109E600001960E94A61EBE016F5F7F4F8DED9EE0A2
:109E70000E947B7BCE0101960E94B47B8DED9EE01B
:109E80000E94107A60E08DED9EE00E940C7B64E001
:109E900075E0CE014C960E94537C6DED7EE0CE01C4
:109EA00001960E944A7CAE014E5D5F4FBE01645E2A
:109EB0007F4FCE0101960E94BCA1182FCE010196C2
:109EC0000E94B47BCE014C960E94B47B112311F406
:109ED0000C94E9468E010E5D1F4F52EBA52E50E10A
:109EE000B52E60E4C62E62E0D62EF12CE12CD8010E
:109EF0006D918D01F50161935F01D6016D936D0147
:109F0000CE0101960E942FA0CE0101960E94071B50
:109F1000CE0101960E94B47BB3E0EB16F10471F020
:109F200064E075E0CE0101960E94537CCE0101965B
:109F30000E94071BCE0101960E94B47BEFEFEE1A40
:109F4000FE0AF4E0EF16F10491F66DE174E0CE0143
:109F500001960E94537CCE0101960E94F01ACE0118
:109F600001960E94B47B68E87FE080916602909140
:109F700067020E944F0964E670E080E090E00E9472
:109F8000407F68E379E0CE0101960E94417C46CA99
:109F900063E379E0CE0101960E94417CBE016F5FD0
:109FA0007F4FCE018E960E949E7A182FCE01019689
:109FB0000E94B47B112309F47CC044E050E061E0CE
:109FC0007FE0CE0101960E94A61EBE016F5F7F4F0B
:109FD0008DED9EE00E947B7BCE0101960E94B47BBA
:109FE0008DED9EE00E94107A60E08DED9EE00E9473
:109FF0000C7B4091E10E5091E20E6AE97BE08DED21
:10A000009EE00E94507764E075E0CE014C960E947D
:10A01000537C6DED7EE0CE0101960E944A7CAE013C
:10A020004E5D5F4FBE01645E7F4FCE0101960E9480
:10A03000BCA1182FCE0101960E94B47BCE014C9694
:10A040000E94B47B112311F40C94E9468E010E5D3D
:10A050001F4F44EBE42E4FE0F42E6E0186E2C80E53
:10A06000D11CD8016D918D01F70161937F01CE0163
:10A0700001960E942FA0CE0101960E94F01ACE01F7
:10A0800001960E94B47BC016D10659F784EF91E087
:10A09000909367028093660268E87FE00E944F0910
:10A0A00064E670E080E090E00E94407F68E279E042
:10A0B0006ACF61E279E0CE0101960E94417CBE0147
:10A0C0006F5F7F4FCE018E960E949E7A182FCE0131
:10A0D00001960E94B47B1123F1F146E050E061E06B
:10A0E0007FE0CE0101960E94A61EBE016F5F7F4FEA
:10A0F0008DED9EE00E947B7BCE0101960E94B47B99
:10A100008DED9EE00E94107A8091E10E9091E20E1A
:10A11000892B11F40C94E9468DED9EE00E94057A9E
:10A120007093B1106093B01070933F0260933E0241
:10A1300084EF91E0909367028093660268E87FE085
:10A140000E944F0964E670E080E090E00E94407F4A
:10A150006DE079E018CF66E079E0CE0101960E94CB
:10A16000417CBE016F5F7F4FCE018E960E949E7A2A
:10A17000182FCE0101960E94B47B1123B9F069EF2C
:10A1800078E0CE0101960E94417C44E650E06FEFFA
:10A190007FEFCE0101960E94250ACE0101960E9412
:10A1A000B47BF0E0E0E019950C94E94661EF78E0CB
:10A1B000CE0101960E94417CBE016F5F7F4FCE01B0
:10A1C0008E960E949E7A182FCE0101960E94B47B33
:10A1D000112301F165E476E0CE0101960E94537CE3
:10A1E0006EEC70E1CE0101960E94CF7ABC0183EE45
:10A1F0009EE00E94647BCE0101960E94B47B63EED8
:10A200007EE0CE0101960E944A7CCE0101960E941A
:10A21000F01A8DC46AEE78E0CE0101960E94417C6E
:10A22000BE016F5F7F4FCE018E960E949E7A182FDF
:10A23000CE0101960E94B47B112369F06BED78E0AA
:10A2400083EE9EE00E943F7B64ED70E183EE9EE032
:10A250000E94387BD4CF60E576E0CE0101960E9463
:10A26000537CBE016F5F7F4FCE018E960E949E7A17
:10A27000182FCE0101960E94B47B112331F00E9469
:10A280009A3010923D020C94E94669E576E0CE01E1
:10A290004C960E94537CBE01645E7F4F81E09FE03C
:10A2A0000E949E7A11E0811115C06EE576E0CE0124
:10A2B00001960E94537CBE016F5F7F4F81E09FE05B
:10A2C0000E949E7A11E0811101C010E0CE0101963A
:10A2D0000E94B47BCE014C960E94B47B112309F4FA
:10A2E00041C063E476E0CE0101960E94537C409128
:10A2F000050F5091060F8D819E81481B590BBE01A1
:10A300006F5F7F4F81E09FE00E9459A0AC014F5FDB
:10A310005F4F61E07FE0CE014C960E94A61EBE0119
:10A32000645E7F4F8DED9EE00E947B7BCE014C965C
:10A330000E94B47BCE0101960E94B47B8DED9EE01D
:10A340000E94057A6115710531F481E08093F00275
:10A350000E94C29496CF6130710509F092CF10929D
:10A36000F002F6CF63E676E0CE0101960E94537CC0
:10A37000BE016F5F7F4FCE018E960E949E7A182F8E
:10A38000CE0101960E94B47B112309F43BC143E046
:10A3900050E061E07FE0CE0101960E94A61EBE0162
:10A3A0006F5F7F4F8DED9EE00E947B7BCE0101961B
:10A3B0000E94B47B6DED7EE0CE0101960E944A7C46
:10A3C000CE0101960E945C21CE0101960E94B47BD1
:10A3D00084EF91E090936702809366026DED7EE0DA
:10A3E000CE0101960E944A7C60E0CE0101960E9457
:10A3F000207BBC018AED90E10E94647BCE01019636
:10A400000E94B47B6DED7EE0CE0101960E944A7CF5
:10A4100060E0CE0101960E94207BBC0184ED90E1BA
:10A420000E94647BCE0101960E94B47B4091DE10B5
:10A430005091DF1068E470E18AED90E10E9450775E
:10A440004091D8105091D91063E570E184ED90E10E
:10A450000E94507768E87FE08091660290916702E1
:10A460000E944F0967E676E0CE0101960E94537C78
:10A470006DED7EE0CE0101960E94CF7ABC01CE0147
:10A4800082960E944A7CCE0101960E94B47B809104
:10A49000441090914510892B39F4BE016E5D7F4FB9
:10A4A00088E89CE00E94757D68EB7BE080E090E0AE
:10A4B0000E94407F8091441090914510029709F0CE
:10A4C00087C06DED7EE0CE0188960E944A7C6FE6E3
:10A4D00076E0CE0101960E94537CCE0101960E9447
:10A4E000EE94CE0101960E94B47B64EF71E080E0AF
:10A4F00090E00E94407F62E776E0CE0101960E94E4
:10A50000537CCE0101960E94EE94CE0101960E94EA
:10A51000B47B6CED75E080E090E00E94407F6BE7DB
:10A5200076E0CE0101960E94537CCE0101960E94F6
:10A53000EE94CE0101960E94B47B64EF71E080E05E
:10A5400090E00E94407F69E876E0CE0101960E948B
:10A55000537CCE0101960E94EE94CE0101960E949A
:10A56000B47B64EF71E080E090E00E94407F67E69A
:10A5700076E0CE0101960E94537CBE01685D7F4F5C
:10A58000CE0101960E94CF7ABC01CE014C960E946A
:10A590004A7CCE0101960E94B47BCE014C960E946B
:10A5A000107ABE01645E7F4FCE0101960E944A7C04
:10A5B000CE0101960E94EE94CE0101960E94B47BDA
:10A5C000CE014C960E94B47BCE0188960E94B47B4B
:10A5D00068EB7BE080E090E00E94407F68E470E1FF
:10A5E000CE0101960E94537CCE0101960E945C210F
:10A5F000CE0101960E94B47B10923D02CE0182965C
:10A600000C94754967E976E0CE0101960E94537C6F
:10A61000BE016F5F7F4FCE018E960E949E7A182FEB
:10A62000CE0101960E94B47B112309F486C044E058
:10A6300050E061E07FE0CE0101960E94A61EBE01BF
:10A640006F5F7F4F8DED9EE00E947B7BCE01019678
:10A650000E94B47B6CE976E0CE0101960E94537CA7
:10A660006DED7EE0CE0101960E94CF7ABC01CE0155
:10A670004C960E944A7CCE0101960E94B47B809148
:10A68000441090914510892B39F4BE01645E7F4FD0
:10A6900088E89CE00E94757D68E873E180E090E0C6
:10A6A0000E94407F8091441090914510029759F587
:10A6B00063EA76E0CE0101960E94537C8091E10E20
:10A6C0009091E20E892B19F56CEA76E0CE010196A5
:10A6D0000E949779BE01645E7F4FCE0182960E94F0
:10A6E0004A7CCE0182960E94EE94CE0182960E9410
:10A6F000B47B68E873E180E090E00E94407FCE0187
:10A7000001960E94B47B10923D020C947349BE01E5
:10A710006F5F7F4FCE0182960E944A7CCE01829667
:10A720000E94EE94CE0182960E94B47B60E777E1AE
:10A7300080E090E00E94407FCDCF65EB76E0CE01D7
:10A7400001960E94537CBE016F5F7F4FCE018E96B3
:10A750000E949E7A182FCE0101960E94B47B11238D
:10A7600009F475C061E07FE08DED9EE00E94647B9E
:10A7700081E080933D0261E07FE0CE0101960E947E
:10A780004A7CCE0101960E945C21CE0101960E9476
:10A79000B47B8091441090914510029709F16DEDC2
:10A7A0007EE088E89CE00E94757D68EB7BE080E0BD
:10A7B00090E00E94407FCE0101960E948795BE01E5
:10A7C0006F5F7F4F81E09FE00E947B7BCE0101960F
:10A7D0000E94B47B60ED77E080E090E00E94407FD3
:10A7E0008091441090914510029771F46DED7EE0D8
:10A7F000CE0101960E944A7CCE0101960E94EE9401
:10A80000CE0101960E94B47B8091050F9091060FB6
:10A81000892B09F436CD68EC77E0CE0101960E94D1
:10A82000537C61E07FE0CE0101960E94CF7ABC01AB
:10A83000CE014C960E944A7CCE014C960E94F01AA2
:10A84000CE014C960E94B47BCE01019650C269EBBA
:10A8500076E0CE0101960E94537CBE016F5F7F4F70
:10A86000CE018E960E949E7A182FCE0101960E94EC
:10A87000B47B112309F495C1809144109091451047
:10A88000019709F0FECC6FEB76E0CE0188960E942E
:10A89000537CBE01685D7F4F88E89CE00E94757D17
:10A8A0006CE271E080E090E00E94407FCE018296F1
:10A8B0000E94879564E670E080E090E00E94407F0F
:10A8C00010E000E025E0C22ED12C3AE0A32EB12CFE
:10A8D0006AEC76E0CE0101960E94537C50E040E0A5
:10A8E000BE016F5F7F4FCE0182960E94A0A17C01C6
:10A8F000CE0101960E94B47BA7014F5F5F4FBE015E
:10A900006E5D7F4FCE0101960E94A61EBE016F5F55
:10A910007F4FCE0188960E947B7BCE0101960E94DC
:10A92000B47B8CA59DA5892B09F170E060E0CE0178
:10A9300088960E946D7A082E000C990BC0970A9792
:10A94000A8F46CEC76E0CE0101960E94537CBE0127
:10A950006F5F7F4FCE0188960E949E7AE82ECE01CF
:10A9600001960E94B47BFF24F394E110F12C6AE776
:10A9700077E0CE0101960E94417C64E170E0CE0157
:10A9800001960E9476A2CE0101960E94B47B0F5FD1
:10A990001F4F62E370E080E090E00E94407FC801BA
:10A9A000B6010E9493AE0197C1F4CE0101960E94B8
:10A9B000F5228D819E81892B09F4BEC0BE016F5F97
:10A9C0007F4F81E09FE00E94647B0E94D045FF247E
:10A9D000F394CE0101960E94B47BCE0101960E94B1
:10A9E0008795BE016F5F7F4FCE0182960E947B7B71
:10A9F000CE0101960E94B47B62E370E080E090E0BB
:10AA00000E94407F0436110519F0FF2009F460CF41
:10AA100080916D0B8823F1F068EC77E0CE014C96C5
:10AA20000E94537CBE01685D7F4FCE014C960E9410
:10AA3000CF7ABC01CE0101960E944A7CCE010196DC
:10AA40000E94F01ACE0101960E94B47BCE014C9672
:10AA50000E94B47B8CA59DA5892B69F070E060E015
:10AA6000CE0188960E946D7A082E000C990BC09733
:10AA70000A9708F47AC064ED76E0CE0101960E9450
:10AA8000537CCE0182960E94B47BCE0188960E94B0
:10AA9000B47B8D819E81009709F449C0E981FA81D8
:10AAA0002081222309F443C0079708F440C062EDD7
:10AAB00078E0CE014C960E94417C68EC70E0CE01BB
:10AAC0004C960E9476A2CE014C960E94B47BBE01A9
:10AAD0006F5F7F4FCE014C960E944A7C40ED57E05D
:10AAE0006FEF7FEFCE014C960E94250ACE014C9667
:10AAF0000E94B47B60EE76E0CE014C960E94537CBF
:10AB000061E07FE0CE014C960E94CF7ABC01CE017D
:10AB100082960E944A7CCE0182960E94F01ACE0153
:10AB200082960E94B47BCE014C960E94B47BCE01EB
:10AB300001960E94B47BA5CB043111050CF449CFDA
:10AB4000C801B5010E9493AE892B09F042CFBE0126
:10AB5000685D7F4F88E89CE00E94757D68EC70E03E
:10AB600080E090E00E94407F34CF6CEC76E0CE0134
:10AB700001960E94537CBE016F5F7F4FCE01889685
:10AB80000E949E7A182FCE0101960E94B47B11116B
:10AB900072CFBE01685D7F4FCE0101960E94387C66
:10ABA00070CF6EEE76E0CE0101960E94537CBE011E
:10ABB0006F5F7F4FCE018E960E949E7A182FCE0136
:10ABC00001960E94B47B112309F4EAC025E030E02D
:10ABD00044E050E061E07FE0CE0101960E94687C95
:10ABE000BE016F5F7F4F8DED9EE00E947B7BCE01AB
:10ABF00001960E94B47B61E07FE0CE0101960E9445
:10AC00004A7CCE0101960E945C21CE0101960E94F1
:10AC1000B47B8DED9EE00E94057A6130710509F0EC
:10AC200069C0709345106093441069EA77E0CE01E3
:10AC300001960E94417CCE0101960E945C21CE01CA
:10AC400001960E94B47B63EF76E0CE014C960E94A1
:10AC5000537C64ED70E1CE014C960E94CF7ABC012A
:10AC6000CE0101960E944A7C48EC50E06FEF7FEFE6
:10AC7000CE0101960E94B926CE0101960E94B47BB6
:10AC8000CE014C960E94B47B0E9412A040E052EC90
:10AC900061E070E088E89CE00E94347684EF91E007
:10ACA000909367028093660268E87FE00E944F09F4
:10ACB00062E077E0CE014C960E94537C6EEC70E12E
:10ACC000CE014C960E94CF7ABC01CE0101960E9423
:10ACD0004A7C40ED57E06FEF7FEFCE0101960E9476
:10ACE000250ACE0101960E94B47BCE014C960E94AB
:10ACF000B47BC7CA61157105D1F510924510109249
:10AD000044106BE977E0CE0101960E94417CCE01B0
:10AD100001960E945C21CE0101960E94B47B69EFEE
:10AD200076E0CE014C960E94537C64ED70E1CE013A
:10AD30004C960E94CF7ABC01CE0101960E944A7CBB
:10AD400048EC50E06FEF7FEFCE0101960E94B926EC
:10AD5000CE0101960E94B47BCE014C960E94B47B3A
:10AD60000E9412A040E855E260E070E093CF6230AC
:10AD7000710509F086CA70934510609344106AE823
:10AD800077E0CE0101960E94417CCE0101960E949F
:10AD90005C21CE0101960E94B47B6DEF76E0C1CFBD
:10ADA00067E077E0CE0101960E94537CBE016F5FA1
:10ADB0007F4FCE018E960E949E7A182FCE0101966B
:10ADC0000E94B47B112309F441C047E050E061E0E8
:10ADD0007FE0CE0101960E94A61EBE016F5F7F4FED
:10ADE0008DED9EE00E947B7BCE0101960E94B47B9C
:10ADF00062ED76E0CE0101960E94537CBE016F5F4A
:10AE00007F4F8DED9EE00E949E7A182FCE01019615
:10AE10000E94B47B111110924F0C66ED74E0CE01CC
:10AE200001960E94537CBE016F5F7F4F8DED9EE0C7
:10AE30000E949E7A182FCE0101960E94B47B1123A6
:10AE400009F4E9CC81E080934F0CE5CC6FE077E02A
:10AE5000CE0101960E94537CBE016F5F7F4FCE01F1
:10AE60008E960E949E7A182FCE0101960E94B47B86
:10AE7000112381F146E050E061E07FE0CE010196D0
:10AE80000E94A61EBE016F5F7F4F8DED9EE00E9467
:10AE90007B7BCE0101960E94B47B8DED9EE00E94EB
:10AEA000FA7960938C1070938D1080938E1090932C
:10AEB0008F1084EF91E0909367028093660268E8B8
:10AEC0007FE00E944F0964E670E080E090E00E941D
:10AED000407FA1CC66E177E0CE0101960E94537CD1
:10AEE000BE016F5F7F4FCE018E960E949E7A182F13
:10AEF000CE0101960E94B47B112301F148E050E09D
:10AF000061E07FE0CE0101960E94A61EBE016F5F48
:10AF10007F4F8DED9EE00E947B7BCE0101960E94CB
:10AF2000B47B8DED9EE00E94FA796093921070934D
:10AF300093108093941090939510BBCF6FE177E0BE
:10AF4000CE0101960E94537CBE016F5F7F4FCE0100
:10AF50008E960E949E7A182FCE0101960E94B47B95
:10AF6000112301F149E050E061E07FE0CE0101965C
:10AF70000E94A61EBE016F5F7F4F8DED9EE00E9476
:10AF80007B7BCE0101960E94B47B8DED9EE00E94FA
:10AF9000FA7960939610709397108093981090931D
:10AFA000991087CF69E277E0CE0101960E94537C29
:10AFB000BE016F5F7F4FCE018E960E949E7A182F42
:10AFC000CE0101960E94B47B1123F1F049E050E0DC
:10AFD00061E07FE0CE0101960E94A61EBE016F5F78
:10AFE0007F4F8DED9EE00E947B7BCE0101960E94FB
:10AFF000B47B8DED9EE00E94FA790E9453AE70936F
:10B000009D1060939C1055CF63E377E0CE010196CD
:10B010000E94537CBE016F5F7F4FCE018E960E94CF
:10B020009E7A182FCE0101960E94B47B1123F1F075
:10B030004AE050E061E07FE0CE0101960E94A61E4A
:10B04000BE016F5F7F4F8DED9EE00E947B7BCE0146
:10B0500001960E94B47B8DED9EE00E94FA790E94D9
:10B0600053AE70939B1060939A1023CF6EE377E0FA
:10B07000CE0101960E94537CBE016F5F7F4FCE01CF
:10B080008E960E949E7A182FCE0101960E94B47B64
:10B09000112311F14BE050E061E07FE0CE01019619
:10B0A0000E94A61EBE016F5F7F4F8DED9EE00E9445
:10B0B0007B7BCE0101960E94B47B8DED9EE00E94C9
:10B0C000FA790E9453AE60939E1070939F10809304
:10B0D000A0109093A110EDCE6AE477E0CE01019626
:10B0E0000E94537CBE016F5F7F4FCE018E960E94FF
:10B0F0009E7A182FCE0101960E94B47B1123E1F0B5
:10B1000045E050E061E07FE0CE0101960E94A61E7E
:10B11000BE016F5F7F4F8DED9EE00E947B7BCE0175
:10B1200001960E94B47B8DED9EE00E94057A70939B
:10B13000911060939010BDCE60E577E0CE0101964E
:10B140000E94537CBE016F5F7F4FCE018E960E949E
:10B150009E7A182FCE0101960E94B47B112359F0DC
:10B160000E94AF856093F30B7093F40B8093F50B03
:10B170009093F60B86C866E577E0CE0101960E94B3
:10B18000537CBE016F5F7F4FCE018E960E949E7AE8
:10B19000182FCE0101960E94B47B112389F143E060
:10B1A00050E0BE01625D7F4FCE0101960E94A61E57
:10B1B000BE016F5F7F4F8DED9EE00E947B7BCE01D5
:10B1C00001960E94B47B8091E10E9091E20E892B52
:10B1D00041F08DED9EE00E94057A70936D026093C0
:10B1E0006C0280916C0290916D020197029708F4B5
:10B1F00012CB81E090E090936D0280936C020BCBB8
:10B2000067E377E0CE014C960E94537CBE01645EFA
:10B210007F4FCE018E960E949E7A11E0811115C05B
:10B220006DE977E0CE0101960E94537CBE016F5F0D
:10B230007F4FCE018E960E949E7A11E0811101C04F
:10B2400010E0CE0101960E94B47BCE014C960E9484
:10B25000B47B112309F468C067E377E0CE0101965F
:10B260000E94537CBE016F5F7F4FCE018E960E947D
:10B270009E7A182FCE0101960E94B47B1123A1F073
:10B2800046E050E0BE01625D7F4FCE0101960E9414
:10B29000A61EBE016F5F7F4F8DED9EE00E947B7BFF
:10B2A000CE0101960E94B47B6DE977E0CE01019654
:10B2B0000E94537CBE016F5F7F4FCE018E960E942D
:10B2C0009E7A182FCE0101960E94B47B1123A1F023
:10B2D00042E050E0BE01625D7F4FCE0101960E94C8
:10B2E000A61EBE016F5F7F4F8DED9EE00E947B7BAF
:10B2F000CE0101960E94B47B8091E10E9091E20E06
:10B30000892B09F488CA6DED7EE0CE0101960E947A
:10B310004A7C61E070E0CE0101960E94ED36CE01DC
:10B3200001960E94B47B77CA63E677E0CE018296ED
:10B330000E94537CBE016E5D7F4FCE018E960E94AF
:10B340009E7A11E0811129C06AE577E0CE014C9622
:10B350000E94537CBE01645E7F4FCE018E960E9498
:10B360009E7A11E0811115C062E677E0CE01019668
:10B370000E94537CBE016F5F7F4FCE018E960E946C
:10B380009E7A11E0811101C010E0CE0101960E9469
:10B39000B47BCE014C960E94B47BCE0182960E9473
:10B3A000B47B112309F4E6C063E677E0CE01019691
:10B3B0000E94537CBE016F5F7F4FCE018E960E942C
:10B3C0009E7A182FCE0101960E94B47B112309F4B6
:10B3D00066C046E050E0BE01625D7F4FCE0101963F
:10B3E0000E94A61EBE016F5F7F4F8DED9EE00E9402
:10B3F0007B7BCE0101960E94B47B8DED9EE00E9486
:10B40000FA796B017C0120E030E0A9010E9489AE4D
:10B4100018160CF08EC0A701960160E070E08AE774
:10B4200094E40E94E1AD0E9453AE609339027093A0
:10B430003A0280933B0290933C02809139029091B2
:10B440003A02A0913B02B0913C02181619061A0666
:10B450001B0664F081E090E0A0E0B0E08093390248
:10B4600090933A02A0933B02B0933C0280916C020D
:10B4700090916D028130910509F068C08091390288
:10B4800090913A02A0913B02B0913C028093350228
:10B4900090933602A0933702B0933802BCC947E0BC
:10B4A00050E0BE01625D7F4FCE0101960E94A61E54
:10B4B000BE016F5F7F4F8DED9EE00E947B7BCE01D2
:10B4C00001960E94B47B6EE774E0CE0101960E9463
:10B4D000537CBE016F5F7F4FCE018E960E949E7A95
:10B4E000182FCE0101960E94B47B112331F081E028
:10B4F00090E090936D0280936C0260E776E0CE015D
:10B5000001960E94537CBE016F5F7F4FCE018E96E5
:10B510000E949E7A182FCE0101960E94B47B1123BF
:10B5200009F46BCF82E090E090936D0280936C02FF
:10B5300064CF81E090E0A0E0B0E080933902909386
:10B540003A02A0933B02B0933C0277CF029709F0F6
:10B5500062C98091390290913A02A0913B02B09168
:10B560003C028093310290933202A0933302B09355
:10B57000340251C96AE677E0CE014C960E94537CB2
:10B58000BE01645E7F4FCE018E960E947E7A11E0EE
:10B59000811115C06FE677E0CE0101960E94537CC1
:10B5A000BE016F5F7F4FCE018E960E949E7A11E0A2
:10B5B000811101C010E0CE0101960E94B47BCE0142
:10B5C0004C960E94B47B112309F48DC268EF77E09A
:10B5D000CE0101960E94537CBE016F5F7F4FCE016A
:10B5E0008E960E949E7A182FCE0101960E94B47BFF
:10B5F000112309F4FBC001E010E010936D020093E9
:10B600006C0210935D0200935C026AEA75E08DEDB6
:10B610009EE00E94977910935D0200935C0281E0A6
:10B6200090E0A0E0B0E08093390290933A02A093BA
:10B630003B02B0933C028093350290933602A09374
:10B640003702B09338026DED7EE0CE0101960E9484
:10B650004A7C62E070E0CE0101960E94ED36CE0198
:10B6600001960E94B47B61EC78E0CE0101960E94C5
:10B67000417CCE0101960E94F01ACE0101960E94F3
:10B68000B47B61EB78E0CE0101960E94417CCE0153
:10B6900001960E948E27CE0101960E94B47B62ED36
:10B6A00076E08DED9EE00E9497796DED7EE0CE0113
:10B6B00001960E944A7C63E070E0CE0101960E94F0
:10B6C000ED36CE0101960E94B47B82E090E090932B
:10B6D0006D0280936C0260EA78E0CE0101960E94D0
:10B6E000417CCE0101960E94F01ACE0101960E9483
:10B6F000B47B64E978E0CE0101960E94417CCE01E2
:10B7000001960E948E27CE0101960E94B47B6AEAC0
:10B7100075E08DED9EE00E9497798091AE1090913A
:10B72000AF1097FF06C066E777E08DED9EE00E94C0
:10B7300097796DED7EE0CE0101960E944A7C62E031
:10B7400070E0CE0101960E94ED36CE0101960E9476
:10B75000B47B62ED76E08DED9EE00E94977982E009
:10B7600090E090936D0280936C026DED7EE0CE01CF
:10B7700001960E944A7C63E070E0CE0101960E942F
:10B78000ED36CE0101960E94B47B84EF91E0909358
:10B7900067028093660268E87FE00E944F0964E6D2
:10B7A00070E080E090E00E94407F81E090E0909324
:10B7B0006D0280936C021092DA021092D90282E03C
:10B7C00090E0A0E0B0E08093C3029093C402A09305
:10B7D000C502B093C6020E94AF856093E3027093E6
:10B7E000E4028093E5029093E60215C86AE677E0EA
:10B7F000CE0101960E94537CBE016F5F7F4FCE0148
:10B800008E960E949E7A182FCE0101960E94B47BDC
:10B8100011110C940B546EE774E0CE0101960E9456
:10B82000537CBE016F5F7F4FCE018E960E949E7A41
:10B83000182FCE0101960E94B47B112331F081E0D4
:10B8400090E090936D0280936C0260E776E0CE0109
:10B8500001960E94537CBE016F5F7F4FCE018E9692
:10B860000E949E7A182FCE0101960E94B47B11236C
:10B8700031F082E090E090936D0280936C0281E061
:10B8800090E0A0E0B0E08093390290933A02A09358
:10B890003B02B0933C0280916C0290916D0281302A
:10B8A000910509F099C090935D0280935C026FE668
:10B8B00077E0CE0101960E94537CBE016F5F7F4FFF
:10B8C000CE018E960E949E7A182FCE0101960E947C
:10B8D000B47B112319F146E050E0BE01625D7F4F59
:10B8E000CE014C960E94A61E6AE777E0CE01019633
:10B8F0000E94537CBE01645E7F4FCE0101960E9480
:10B90000CF7ABC018DED9EE00E94647BCE01019652
:10B910000E94B47BCE014C960E94B47B8091390288
:10B9200090913A02A0913B02B0913C028093350283
:10B9300090933602A0933702B09338026AEA75E01A
:10B940008DED9EE00E9497796DED7EE0CE0101962F
:10B950000E944A7C62E070E0CE0101960E94ED36C2
:10B96000CE0101960E94B47B63E878E0CE01019697
:10B970000E94417CCE0101960E94F01ACE010196F0
:10B980000E94B47B81E090E090935D0280935C0222
:10B9900062ED76E08DED9EE00E9497796DED7EE0A0
:10B9A000CE0101960E944A7C63E070E0CE010196D0
:10B9B0000E94ED36CE0101960E94B47B63E778E0E9
:10B9C000CE0101960E94417CCE0101960E948E27F5
:10B9D000CE0101960E94B47B80916C0290916D0221
:10B9E000029711F00C940B546AEA75E08DED9EE01D
:10B9F0000E9497798091AE109091AF1097FF06C08A
:10BA000066E777E08DED9EE00E94977901E010E017
:10BA100010935D0200935C026DED7EE0CE01019615
:10BA20000E944A7C62E070E0CE0101960E94ED36F1
:10BA3000CE0101960E94B47B62ED76E08DED9EE032
:10BA40000E94977962E678E0CE0101960E94417CDF
:10BA5000CE0101960E94F01ACE0101960E94B47B9D
:10BA60006DED7EE0CE0101960E944A7C63E070E0BD
:10BA7000CE0101960E94ED36CE0101960E94B47B64
:10BA800066E578E0CE0101960E94417CCE010196E8
:10BA90000E948E27CE0101960E94B47B8091AE1049
:10BAA0009091AF109195819591099093AF108093EB
:10BAB000AE1010935D0200935C0284EF91E09093CE
:10BAC00067028093660268E87FE00E944F0964E69F
:10BAD00070E080E090E00E94407F10936D02009340
:10BAE0006C020C940B546CE777E0CE0188960E94B0
:10BAF000537CBE01685D7F4FCE018E960E949E7A78
:10BB000001E081113DC06DEC77E0CE0182960E948C
:10BB1000537CBE016E5D7F4FCE018E960E949E7A51
:10BB200001E0811129C06CEC77E0CE014C960E94B7
:10BB3000537CBE01645E7F4FCE018E960E949E7A3A
:10BB400001E0811115C063E877E0CE0101960E9403
:10BB5000537CBE016F5F7F4FCE018E960E949E7A0E
:10BB600001E0811101C000E0CE0101960E94B47B8A
:10BB7000CE014C960E94B47BCE0182960E94B47B8B
:10BB8000CE0188960E94B47B002309F41FC26CE7A3
:10BB900077E0CE0101960E94537CBE016F5F7F4F1C
:10BBA000CE018E960E949E7A082FCE0101960E94A9
:10BBB000B47B46E050E0011117C06DEC77E0CE0198
:10BBC00001960E94537CBE016F5F7F4FCE018E961F
:10BBD0000E949E7A082FCE0101960E94B47B00231A
:10BBE00009F48BC042E050E0BE01625D7F4FCE01A0
:10BBF00001960E94A61EBE016F5F7F4F8DED9EE0F5
:10BC00000E947B7BCE0101960E94B47B8091E10E65
:10BC10009091E20E892B11F40C940B546AE777E0B3
:10BC2000CE014C960E94537CBE01645E7F4F8DED29
:10BC30009EE00E949E7A811114C06CEB78E0CE01E8
:10BC400001960E94537CBE016F5F7F4F8DED9EE099
:10BC50000E949E7A11E0811110E0CE0101960E94AF
:10BC6000B47BCE014C960E94B47BC12CD12C7601C2
:10BC7000112309F46AC18DED9EE00E94FA796B01EF
:10BC80007C0180916C0290916D02019709F09FC038
:10BC90008DED9EE00E94FA799B01AC016091960BBC
:10BCA0007091970B8091980B9091990B0E9475ADB4
:10BCB0006093960B7093970B8093980B9093990BCE
:10BCC0008090960B9090970BA090980BB090990B4A
:10BCD00020E030E044EB53E4C501B4010E9489AE9A
:10BCE00087FD86C020E030E044EB53E4C501B40199
:10BCF0000E9474AD4B015C01EBCF43E050E0BE010C
:10BD0000625D7F4FCE0101960E94A61EBE016F5F4D
:10BD10007F4F8DED9EE00E947B7BCE0101960E94BD
:10BD2000B47B6EE774E0CE0101960E94537CBE01A5
:10BD30006F5F7F4FCE018E960E949E7A082FCE01B4
:10BD400001960E94B47B0023B1F081E090E09093D3
:10BD50006D0280936C028091E10B9091E20BA091B7
:10BD6000E30BB091E40B8093960B9093970BA09309
:10BD7000980BB093990B60E776E0CE0101960E9494
:10BD8000537CBE016F5F7F4FCE018E960E949E7ADC
:10BD9000082FCE0101960E94B47B002309F436CF10
:10BDA00082E090E090936D0280936C028091DD0BB5
:10BDB0009091DE0BA091DF0BB091E00B8093960B7E
:10BDC0009093970BA093980BB093990B1FCF8DED89
:10BDD0009EE00E94FA799B01AC016091960B7091F4
:10BDE000970B8091980B9091990B0E9474AD60CF46
:10BDF00020E030E0A901C501B4010E94C7AB87FF74
:10BE00000BC020E030E044EB53E4C501B4010E94D4
:10BE100075AD4B015C01ECCF8092960B9092970B25
:10BE2000A092980BB092990B20E030E0A901C701D5
:10BE3000B6010E9489AE87FD15C06CEB78E0CE019B
:10BE400001960E94537C6DED7EE0CE0101960E942A
:10BE5000CF7ABC018DED9EE00E94647BCE010196FD
:10BE60000E94B47B20E030E0A901C701B6010E9426
:10BE7000C7AB87FF6AC080916C0290916D020197F9
:10BE800099F520E030E0A901C701B6010E9489AE12
:10BE900018160CF092C020E030E040E251E4C701F7
:10BEA000B6010E9475AD22E0AB01BC01CE014C96FB
:10BEB0000E94BC7B6AE777E0CE0101960E94537C2A
:10BEC000BE01645E7F4FCE0101960E94CF7ABC0115
:10BED0008DED9EE00E94647BCE0101960E94B47BB2
:10BEE000CE014C960E94B47B80916C0290916D02C1
:10BEF000019759F120E030E0A901C701B6010E9485
:10BF000089AEB701A60118160CF0705822E0CE01D8
:10BF10004C960E94BC7B6AE777E0CE0101960E94B6
:10BF2000537CBE01645E7F4FCE0101960E94CF7AA2
:10BF3000BC018DED9EE00E94647BCE0101960E94C3
:10BF4000B47BCE014C960E94B47B81E090E090934C
:10BF50005D0280935C026DED7EE0CE0101960E9451
:10BF60004A7C62E070E0CE0101960E94ED36CE017F
:10BF700001960E94B47B20E030E0A901C701B60120
:10BF80000E94C7AB87FD02C00C940B5480916C02D9
:10BF900090916D02019711F00C940B5467E877E0D3
:10BFA0008DED9EE00E9497796DED7EE0CE010196C9
:10BFB0000E944A7C62E070E0AEC9A701960160E091
:10BFC00070E080E291E40E9474AD6DCF6CE877E0A0
:10BFD000CE0182960E94537CBE016E5D7F4FCE01E2
:10BFE0008E960E949E7A11E0811129C06BE877E05D
:10BFF000CE014C960E94537CBE01645E7F4FCE0101
:10C000008E960E949E7A11E0811115C062E977E058
:10C01000CE0101960E94537CBE016F5F7F4FCE011F
:10C020008E960E949E7A11E0811101C010E0CE012F
:10C0300001960E94B47BCE014C960E94B47BCE0147
:10C0400082960E94B47B112309F49BC0CE018E9688
:10C050000E94107A6AEA75E08DED9EE00E94977961
:10C060006EE774E0CE0101960E94537CBE016F5FC3
:10C070007F4FCE018E960E949E7A182FCE01019698
:10C080000E94B47B112331F081E090E090936D0227
:10C0900080936C0260E776E0CE0101960E94537CAB
:10C0A000BE016F5F7F4FCE018E960E949E7A182F41
:10C0B000CE0101960E94B47B112391F082E090E0C2
:10C0C00090936D0280936C028091AE109091AF10AE
:10C0D00097FF06C066E777E08DED9EE00E949779B6
:10C0E00081E090E090935D0280935C026DED7EE0D4
:10C0F000CE0101960E944A7C62E070E0CE0101967A
:10C100000E94ED36CE0101960E94B47B6CE877E088
:10C11000CE0101960E94537CBE016F5F7F4FCE011E
:10C120008E960E949E7A182FCE0101960E94B47BB3
:10C1300045E050E0111102C046E050E0BE01625DF2
:10C140007F4FCE0101960E94A61EBE016F5F7F4FFA
:10C150008DED9EE00E947B7BCE0101960E94B47B18
:10C160008091E10E9091E20E892B11F40C940B5406
:10C170006DED7EE0CE0101960E944A7C63E070E0A6
:10C18000CAC86AE977E0CE0182960E94537CBE015C
:10C190006E5D7F4FCE018E960E949E7A11E08111D6
:10C1A00029C069E977E0CE014C960E94537CBE011C
:10C1B000645E7F4FCE018E960E949E7A11E08111BF
:10C1C00015C060EA77E0CE0101960E94537CBE0163
:10C1D0006F5F7F4FCE018E960E949E7A11E0811193
:10C1E00001C010E0CE0101960E94B47BCE014C96B6
:10C1F0000E94B47BCE0182960E94B47B112309F485
:10C2000026C16AE977E0CE0101960E94537CBE0107
:10C210006F5F7F4FCE018E960E949E7A182FCE01BF
:10C2200001960E94B47B112309F443C045E050E01D
:10C23000BE01625D7F4FCE0101960E94A61EBE0127
:10C240006F5F7F4F8DED9EE00E947B7BCE0101965C
:10C250000E94B47B8091E10E9091E20E892B61F0F7
:10C260008DED9EE00E94FA796093960B7093970B88
:10C270008093980B9093990BC090960BD090970B4E
:10C28000E090980BF090990B20E030E044EB53E401
:10C29000C701B6010E9489AE87FD55C020E030E09D
:10C2A00044EB53E4C701B6010E9474AD6B017C01FD
:10C2B000EBCF46E050E0BE01625D7F4FCE010196BC
:10C2C0000E94A61EBE016F5F7F4F8DED9EE00E9413
:10C2D0007B7BCE0101960E94B47B6EE774E0CE01B9
:10C2E00001960E94537CBE016F5F7F4FCE018E96F8
:10C2F0000E949E7A182FCE0101960E94B47B1123D2
:10C3000031F081E090E090936D0280936C0260E7E1
:10C3100076E0CE0101960E94537CBE016F5F7F4F95
:10C32000CE018E960E949E7A182FCE0101960E9411
:10C33000B47B112309F48ECF82E090E090936D02DC
:10C3400080936C0287CF20E030E0A901C701B601DD
:10C350000E94C7AB87FF0BC020E030E044EB53E402
:10C36000C701B6010E9475AD6B017C01ECCFC09294
:10C37000960BD092970BE092980BF092990B8091CC
:10C380006C0290916D02019771F4C092E10BD09212
:10C39000E20BE092E30BF092E40B61E175E083EED7
:10C3A0009EE00E9497798091960B9091970BA091B7
:10C3B000980BB091990B20916C0230916D02223054
:10C3C000310571F48093DD0B9093DE0BA093DF0BAE
:10C3D000B093E00B61E275E083EE9EE00E949779F6
:10C3E0004091960B5091970B6091980B7091990B1F
:10C3F00021E0CE014C960E94BC7B63EE7EE0CE0134
:10C4000001960E944A7CBE01645E7F4FCE01019678
:10C410000E94CF7A6CE175E00E94B97ABC0183EE8C
:10C420009EE00E94647BCE0101960E94B47BCE0107
:10C430004C960E94B47B63EE7EE0CE0101960E9492
:10C440004A7CCE0101960E948E270C948F5968EA8F
:10C4500077E0CE0182960E94537CBE016E5D7F4FD5
:10C46000CE018E960E949E7A11E0811129C067EA62
:10C4700077E0CE014C960E94537CBE01645E7F4FF4
:10C48000CE018E960E949E7A11E0811115C06DEA50
:10C4900077E0CE0101960E94537CBE016F5F7F4F13
:10C4A000CE018E960E949E7A11E0811101C010E0AB
:10C4B000CE0101960E94B47BCE014C960E94B47BC3
:10C4C000CE0182960E94B47B112309F412C2C0905F
:10C4D0003902D0903A02E0903B02F0903C0263EBCC
:10C4E00077E0CE0101960E94537CBE016F5F7F4FC3
:10C4F000CE018E960E949E7A182FCE0101960E9440
:10C50000B47B112309F465C044E050E0BE01625DD4
:10C510007F4FCE0101960E94A61EBE016F5F7F4F26
:10C520008DED9EE00E947B7BCE0101960E94B47B44
:10C5300080916C0290916D028130910509F093C059
:10C54000C0903502D0903602E0903702F090380269
:10C5500081E090E0A0E0B0E0809335029093360255
:10C56000A0933702B09338028091E10E9091E20ED1
:10C57000892B09F090C068EB77E08DED9EE00E947A
:10C5800097798091E10E9091E20E892B81F06DED0B
:10C590007EE0CE0101960E944A7C70E060E0CE0110
:10C5A00001960E94ED36CE0101960E94B47B8091E7
:10C5B0006C0290916D028130910509F08CC1C0929E
:10C5C0003502D0923602E0923702F09238020C9493
:10C5D0000B5445E050E0BE01625D7F4FCE010196F5
:10C5E0000E94A61EBE016F5F7F4F8DED9EE00E94F0
:10C5F0007B7BCE0101960E94B47B6EE774E0CE0196
:10C6000001960E94537CBE016F5F7F4FCE018E96D4
:10C610000E949E7A182FCE0101960E94B47B1123AE
:10C6200031F081E090E090936D0280936C0260E7BE
:10C6300076E0CE0101960E94537CBE016F5F7F4F72
:10C64000CE018E960E949E7A182FCE0101960E94EE
:10C65000B47B112309F46CCF82E090E090936D02DB
:10C6600080936C0265CF029709F07ECFC0903102B3
:10C67000D0903202E0903302F090340281E090E0FA
:10C68000A0E0B0E08093310290933202A093330295
:10C69000B093340269CF6EEB77E0CE0101960E9431
:10C6A000537CBE016F5F7F4F8DED9EE00E947E7ACE
:10C6B000182FCE0101960E94B47B112309F477CF85
:10C6C0008DED9EE00E94FA7920E030E0A9010E9401
:10C6D000C7AB811128C080916C0290916D020197C7
:10C6E00031F461EC77E08DED9EE00E9497798091C6
:10C6F0006C0290916D02029731F468EB77E08DED5A
:10C700009EE00E9497798091E10E9091E20E892B34
:10C7100009F44DCF6DED7EE0CE0101960E944A7C7A
:10C7200061E070E03CCF63E476E0CE0101960E94C8
:10C73000537CBE016F5F7F4F8DED9EE00E947E7A3D
:10C74000182FCE0101960E94B47B112309F42FCF3C
:10C7500041E050E06DED7EE0CE0101960E94A61E04
:10C76000CE0101960E94FA794B015C01CE0101963F
:10C770000E94B47B20E030E0A901C501B4010E9411
:10C78000C7AB181634F0812C912C90E8A92E9FE3AA
:10C79000B92E00916C0210916D020130110509F063
:10C7A00075C0A501940160E070E48CE995E40E94F5
:10C7B000E1AD60932D0270932E0280932F0290932F
:10C7C00030026093A6107093A7108093A8109093E6
:10C7D000A9106093290270932A0280932B029093F0
:10C7E0002C02B801CE014C960E94A17966EC77E04C
:10C7F000CE0101960E94537CBE01645E7F4FCE0144
:10C8000001960E94CF7ABC01CE0182960E944A7C9A
:10C81000CE0182960E94071BCE0182960E94B47BB5
:10C82000CE0101960E94B47BCE014C960E94B47B4F
:10C8300064E478E0CE0101960E94417CCE0101962D
:10C840000E94071BCE0101960E94B47B40912D02ED
:10C8500050912E0260912F027091300225E0CE019E
:10C8600001960E94BC7BCE0101960E94F01ACE0177
:10C8700001960E94B47B84EF91E0909367028093CD
:10C88000660268E87FE00E944F0991CE02301105F0
:10C8900009F0A7CFA501940160E070E48CE196E473
:10C8A0000E94E1AD60932D0270932E0280932F02BF
:10C8B000909330026093AA107093AB108093AC10E9
:10C8C0009093AD1060932502709326028093270207
:10C8D0009093280286CF029711F00C940B54C092CB
:10C8E0003102D0923202E0923302F09234020C9480
:10C8F0000B546BEC77E0CE0182960E94537CBE0114
:10C900006E5D7F4FCE018E960E949E7A11E081115E
:10C9100029C06AEC77E0CE014C960E94537CBE01A0
:10C92000645E7F4FCE018E960E949E7A11E0811147
:10C9300015C060ED77E0CE0101960E94537CBE01E8
:10C940006F5F7F4FCE018E960E949E7A11E081111B
:10C9500001C010E0CE0101960E94B47BCE014C963E
:10C960000E94B47BCE0182960E94B47B112309F40D
:10C9700029C18AA99BA9059710F40C940B5444E093
:10C9800050E0BE01625D7F4FCE0101960E94A61E5F
:10C99000BE016F5F7F4F8DED9EE00E947B7BCE01DD
:10C9A00001960E94B47B6BEC77E0CE0101960E9469
:10C9B000537CBE016F5F7F4FCE018E960E949E7AA0
:10C9C000182FCE0101960E94B47B112309F49BC05D
:10C9D00044E050E0BE01625D7F4FCE0101960E94AF
:10C9E000A61EBE016F5F7F4F8DED9EE00E947B7B98
:10C9F000CE0101960E94B47B8DED9EE00E94FA79F3
:10CA000020E030E0A9010E9489AE181614F00C94C1
:10CA10000B548DED9EE00E94FA7960932D02709385
:10CA20002E0280932F029093300220916C0230915D
:10CA30006D022130310509F0B0C06093A6107093EB
:10CA4000A7108093A8109093A91060932902709367
:10CA50002A0280932B0290932C02B901CE014C96AE
:10CA60000E94A17966EC77E0CE0101960E94537C8A
:10CA7000BE01645E7F4FCE0101960E94CF7ABC0159
:10CA8000CE0182960E944A7CCE0182960E94071BAC
:10CA9000CE0182960E94B47BCE0101960E94B47BA7
:10CAA000CE014C960E94B47B62E378E0CE01019601
:10CAB0000E94417CCE0101960E94071BCE01019687
:10CAC0000E94B47B40912D0250912E0260912F0262
:10CAD0007091300225E0CE0101960E94BC7BCE0110
:10CAE00001960E94F01ACE0101960E94B47B84EF59
:10CAF00091E0909367028093660268E87FE00E946D
:10CB00004F090C940B5445E050E0BE01625D7F4F2D
:10CB1000CE0101960E94A61EBE016F5F7F4F8DED74
:10CB20009EE00E947B7BCE0101960E94B47B6EE763
:10CB300074E0CE0101960E94537CBE016F5F7F4F6F
:10CB4000CE018E960E949E7A182FCE0101960E94E9
:10CB5000B47B112331F081E090E090936D028093DB
:10CB60006C0260E776E0CE0101960E94537CBE0124
:10CB70006F5F7F4FCE018E960E949E7A182FCE0156
:10CB800001960E94B47B112309F436CF82E090E035
:10CB900090936D0280936C022FCF2230310509F003
:10CBA0005CCF6093AA107093AB108093AC109093FD
:10CBB000AD10609325027093260280932702909314
:10CBC00028024BCF65ED75E0CE014C960E94537C58
:10CBD000BE01645E7F4FCE018E960E949E7A11E068
:10CBE000811115C066ED77E0CE0101960E94537C5D
:10CBF000BE016F5F7F4FCE018E960E949E7A11E03C
:10CC0000811101C010E0CE0101960E94B47BCE01DB
:10CC10004C960E94B47B112309F463C065ED75E066
:10CC2000CE0101960E94537CBE016F5F7F4FCE0103
:10CC30008E960E949E7A182FCE0101960E94B47B98
:10CC4000112399F042E050E061E07FE0CE010196CF
:10CC50000E94A61EBE016F5F7F4F8DED9EE00E9479
:10CC60007B7BCE0101960E94B47B66ED77E0CE011E
:10CC700001960E94537CBE016F5F7F4FCE018E965E
:10CC80000E949E7A182FCE0101960E94B47B112338
:10CC900099F043E050E061E07FE0CE0101960E9410
:10CCA000A61EBE016F5F7F4F8DED9EE00E947B7BD5
:10CCB000CE0101960E94B47B8DED9EE00E94057A24
:10CCC000653B710510F40C940B546FE178E0CE01D4
:10CCD00001960E94417CCE0101960E94071B0C9494
:10CCE0008F596AED77E0CE0101960E94537CBE0118
:10CCF0006F5F7F4FCE018E960E949E7A182FCE01D5
:10CD000001960E94B47B112309F474C026E030E040
:10CD100044E050E061E07FE0CE0101960E94687C33
:10CD2000BE016F5F7F4F8DED9EE00E947B7BCE0149
:10CD300001960E94B47B63E476E0CE0101960E94E6
:10CD4000537C4091050F5091060F8D819E81481BA9
:10CD5000590BBE016F5F7F4F81E09FE00E9459A099
:10CD6000AC014F5F5F4F61E07FE0CE014C960E94C7
:10CD7000A61EBE01645E7F4F8DED9EE00E947B7B10
:10CD8000CE014C960E94B47BCE0101960E94B47BEA
:10CD90008DED9EE00E94FA7988E2EEE6FBE0AFE5D9
:10CDA000B0E101900D928A95E1F784EF91E09093C4
:10CDB00067028093660268E87FE00E944F096EEF89
:10CDC00077E083EE9EE00E943F7B44E050E061E02C
:10CDD0007FE0CE0101960E94A61EBE016F5F7F4FCD
:10CDE00083EE9EE00E94387BCE0101960E94B47BC8
:10CDF0000C94FF506EED77E0CE0101960E94537CBB
:10CE0000BE016F5F7F4FCE018E960E949E7A182FD3
:10CE1000CE0101960E94B47B11110C94E55666EE8A
:10CE200077E0CE0101960E94537CBE016F5F7F4F79
:10CE3000CE018E960E949E7A182FCE0101960E94F6
:10CE4000B47B112371F141E068E972E0CE010196F3
:10CE50000E941692BE016F5F7F4F8CEE90E10E94A0
:10CE6000171E8CEE90E10E94500D811104C062EB00
:10CE700077E00C94C34F8CEE90E10E949507892BCC
:10CE800051F08CEE90E10E94BA0D682F85E29DE092
:10CE90000E944E73F0CF8CEE90E10E945C0D0C94DA
:10CEA000E9466DEE77E0CE0101960E94537CBE010B
:10CEB0006F5F7F4FCE018E960E949E7A182FCE0113
:10CEC00001960E94B47B1123E9F08DB79EB782537F
:10CED00091400FB6F8949EBF0FBE8DBFADB7BEB7E1
:10CEE000119682E391E0E8E8FFE001900D9201974E
:10CEF000E1F70E94BB320FB6F894DEBF0FBECDBF84
:10CF00000C94E94666EF77E0CE0101960E94537CCF
:10CF1000BE016F5F7F4FCE018E960E949E7A182FC2
:10CF2000CE0101960E94B47B112309F457C0EDB7DE
:10CF3000FEB7E253F1400FB6F894FEBF0FBEEDBF4F
:10CF4000ADB7BEB7119682E391E0E8E8FFE001904B
:10CF50000D920197E1F70E943A2C0FB6F894DEBFCC
:10CF60000FBECDBF6DEE77E0CE0101960E94417CF1
:10CF7000ADB7BEB7A253B1400FB6F894BEBF0FBE57
:10CF8000ADBF119682E391E0E8E8FFE001900D92D9
:10CF90000197E1F70E9440240FB6F894DEBF0FBE60
:10CFA000CDBF8DB79EB7825391400FB6F8949EBF08
:10CFB0000FBE8DBFADB7BEB7119682E391E0E8E832
:10CFC000FFE001900D920197E1F70E94BB320FB68E
:10CFD000F894DEBF0FBECDBF0C94EE4B68EF77E048
:10CFE000CE0101960E94537CBE016F5F7F4FCE0140
:10CFF0008E960E949E7A182FCE0101960E94B47BD5
:10D000001123F9F06BED77E0CE0101960E94417C8F
:10D01000BE016F5F7F4FCE014C960E944A7CCE01CD
:10D020004C960E94F01ACE014C960E94B47BEDB74C
:10D03000FEB7E253F1400FB6F894FEBF0FBEEDBF4E
:10D04000B9CF6CEF77E0CE0101960E94537CBE0110
:10D050006F5F7F4FCE018E960E949E7A182FCE0171
:10D0600001960E94B47B112309F4F5C06FEB77E0C1
:10D07000CE0182960E94417CBE016E5D7F4FCE0143
:10D0800001960E944A7CAE014F5F5F4F62E070E004
:10D090008FE792E00E94ED2D182FCE0101960E949D
:10D0A000B47B111122C0BE016E5D7F4FCE014C9644
:10D0B0000E944A7C60E078E0CE014C960E94B97AEA
:10D0C00064E37FE00E94CF7ABC01CE0101960E940A
:10D0D0004A7CCE0101960E94F01ACE0101960E9470
:10D0E000B47BCE014C960E94B47B68EE73E080E086
:10D0F00090E00E94407FBE016E5D7F4FCE010196A1
:10D100000E944A7CAE014F5F5F4F63E070E082E7B0
:10D1100092E00E94ED2D182FCE0101960E94B47B63
:10D12000111122C0BE016E5D7F4FCE014C960E9450
:10D130004A7C60E178E0CE014C960E94B97A64E3C3
:10D140007FE00E94CF7ABC01CE0101960E944A7C0A
:10D15000CE0101960E94F01ACE0101960E94B47B86
:10D16000CE014C960E94B47B68EE73E080E090E0C4
:10D170000E94407F68E27FE0CE0101960E944A7CD7
:10D18000AE014F5F5F4F61E070E082EB92E00E9482
:10D19000ED2D182FCE0101960E94B47B111121C0F4
:10D1A00068E27FE0CE014C960E944A7C60E178E024
:10D1B000CE014C960E94B97A64E37FE00E94CF7A58
:10D1C000BC01CE0101960E944A7CCE0101960E94CC
:10D1D000F01ACE0101960E94B47BCE014C960E94BB
:10D1E000B47B68EE73E080E090E00E94407F809125
:10D1F0004F0C882311F40C94FE5243E162EB72E071
:10D20000CE0101960E941692BE016F5F7F4F82E2AF
:10D2100091E10E94171E82E291E10E94500D882345
:10D2200011F40C94FE5268E27FE082E291E10E94E8
:10D23000837D66E970E080E090E00E94407F82E2BA
:10D2400091E10E945C0D62E370E080E090E00E945A
:10D25000407F0C94FE526CE178E0CE0101960E9472
:10D26000537CBE016F5F7F4FCE018E960E949E7AE7
:10D27000182FCE0101960E94B47B1123C1F00CEA55
:10D280001BE082EBE82E8BE0F82ED8018C910E5F2C
:10D290001F4F60E00E94877E6CE271E080E090E0CA
:10D2A0000E94407FE016F10681F70C94E94660E2A7
:10D2B00078E0CE0101960E94537CBE016F5F7F4FE4
:10D2C000CE018E960E949E7A182FCE0101960E9462
:10D2D000B47B1123A9F00CEA1BE0F80180810E5FFA
:10D2E0001F4F61E00E94877E6CE271E080E090E079
:10D2F0000E94407FFBE0023B1F0779F70C94E94650
:10D3000065E278E0CE0101960E94537CBE016F5F1A
:10D310007F4FCE018E960E949E7A182FCE010196E5
:10D320000E94B47B112311F40C94E94627E030E00D
:10D3300046E050E061E07FE0CE0101960E94687C0B
:10D34000BE016F5F7F4F8DED9EE00E947B7BCE0123
:10D3500001960E94B47B8DED9EE00E94057A672BBA
:10D3600071F410926D0B61E07FE0CE0101960E9496
:10D370004A7CCE0101960E945C210C94975581E075
:10D3800080936D0BF0CF2F923F924F925F926F92EE
:10D390007F928F929F92AF92BF92CF92DF92EF9245
:10D3A000FF920F931F93CF93DF9300D000D01F9273
:10D3B0001F92CDB7DEB760918E0270918F0280917F
:10D3C0008C0290918D020E941E1B84E1482E512CEC
:10D3D000612C712C312C212C8FEF281A380AC301B3
:10D3E000B2010E94407F60918E0270918F02809105
:10D3F0008C0290918D020E941E1B8C0183E02816E6
:10D40000310434F08EE12816310444F4012B51F03C
:10D4100084E1480E511C611C711CDECF0115110501
:10D4200009F0A6C080918C0290918D028B309105FD
:10D4300009F086C08090BE109090BF10A090C010E0
:10D44000B090C110C090BA10D090BB10E090BC104A
:10D45000F090BD1064E670E080E090E00E94407FB4
:10D4600061E275E0CE0101960E94417CCE010196F9
:10D470000E948E27CE0101960E94B47B61E082E07B
:10D480000E945C8921E0B501A401CE0101960E94B1
:10D49000BC7BBE016F5F7F4F8EE391E10E94757D83
:10D4A000CE0101960E94B47B6FED8EE391E10E9464
:10D4B00089896CE175E08EE391E10E94977D20E01F
:10D4C000B701A601CE0101960E94BC7BBE016F5F31
:10D4D0007F4F8EE391E10E94757DCE0101960E94FF
:10D4E000B47B6CE278E08EE391E10E946D7D8982ED
:10D4F0009A82AB82BC82CD82DE82EF82F88629815D
:10D500003A814B815C816D817E818F8198852896DF
:10D510000FB6F894DEBF0FBECDBFDF91CF911F9144
:10D520000F91FF90EF90DF90CF90BF90AF909F90C2
:10D530008F907F906F905F904F903F902F900895C5
:10D540008631910509F476CF0C9709F083CF80904E
:10D55000920A9090930AA090940AB090950AC09075
:10D560008E0AD0908F0AE090900AF090910A72CFC4
:10D570000F3F8FEF1807CCF06EE075E0CE010196FB
:10D580000E94417C4AE050E070E060E0CE010196EC
:10D590000E94B926CE0101960E94B47B6BEE74E026
:10D5A00083EE9EE00E943F7B32C00E3F8FEF180754
:10D5B000B9F16DED74E0CE0101960E94417C4AE024
:10D5C00050E070E060E0CE0101960E94B926CE01E5
:10D5D00001960E94B47B6EEC74E083EE9EE00E94A4
:10D5E0003F7BB801CE0101960E94A179BE016F5F19
:10D5F0007F4F83EE9EE00E94387BCE0101960E9411
:10D60000B47B68EB74E083EE9EE00E94E27A1982BC
:10D610001A821B821C821D821E821F8218866FCF77
:10D620006DEA74E0CE0101960E94417C4AE050E030
:10D6300070E060E0CE0101960E94B926CE0101960D
:10D640000E94B47B6DE874E0ABCF2F923F924F9273
:10D650005F926F927F928F929F92AF92BF92CF9282
:10D66000DF92EF92FF920F931F93CF93DF93CDB78B
:10D67000DEB7AC970FB6F894DEBF0FBECDBF8C01FE
:10D680007B018091DB0B9091DC0B01969093DC0B7E
:10D690008093DB0B2091F80B222341F06AE070E0CD
:10D6A0000E9493AE181619060CF4C0C281E0809354
:10D6B000F80B1092DC0B1092DB0B50E040E06EE1B7
:10D6C00074E0C8010E94611E82E0E816F10409F4CA
:10D6D000C6C26DE174E082E29FE00E94977960919A
:10D6E0008E0270918F0280918C0290918D020E9427
:10D6F0001E1B1C016DEF7AE0C8010E94481E6EE2FD
:10D7000078E0C8010E946D7D68EC70E1CE01019661
:10D710000E944A7CBE016F5F7F4FC8010E94757DE9
:10D72000CE0101960E94B47B67E378E0C8010E94B5
:10D730006D7D61E176E0C8010E94977D6EEC70E13D
:10D74000CE0101960E944A7CBE016F5F7F4FC801E7
:10D750000E94757D67E076E0C8010E94977D60EECB
:10D760007FE0CE0109960E94537CBE01675F7F4F28
:10D77000C8010E94757D6AEF75E0C8010E94977D1F
:10D7800068E470E1CE010F960E94537CBE01615F98
:10D790007F4FC8010E94757D63EF75E0C8010E944C
:10D7A000977DCE010F960E94B47BCE0109960E9410
:10D7B000B47BCE0101960E94B47B0E940F8228EEBA
:10D7C00033E040E050E00E9411AD29013A0169EEDA
:10D7D00075E0C8010E94977DCE0101960E94092242
:10D7E000BE016F5F7F4FC8010E94757DCE0101961B
:10D7F0000E94B47BC301B20120E13EE040E050E072
:10D800000E9433AD4B015C01B901CE0187960E94A5
:10D81000B21E4CE3C42ED12CE12CF12CC501B40175
:10D82000A70196010E9433ADB901CE0101960E9475
:10D83000B21E60E077E0CE0109960E94537CBE01E3
:10D840006F5F7F4FCE0109960E94CF7ABC01CE0157
:10D8500087960E94387BCE0109960E94B47BCE0148
:10D8600001960E94B47BC301B201A70196010E94F8
:10D8700033ADCE0101960E94B21E60E077E0CE018A
:10D8800009960E94537CBE016F5F7F4FCE010996BF
:10D890000E94CF7ABC01CE0187960E94387BCE01D0
:10D8A00009960E94B47BCE0101960E94B47B6DE381
:10D8B00078E0CE0109960E94537CBE01695D7F4FDE
:10D8C000CE0109960E94CF7A60E478E00E94B97A8E
:10D8D000BC01CE0101960E944A7CBE016F5F7F4F62
:10D8E000C8010E94757DCE0101960E94B47BCE01D5
:10D8F00009960E94B47B6EE478E0C8010E946D7DB9
:10D90000CE0101960E94E819B801CE0101960E944D
:10D910000F7D69E478E0C8010E94597D0E94C369C7
:10D9200029833A834B835C836D837E838F839887BF
:10D9300049815A816B817C8121E0CE010F960E9442
:10D94000BC7BBE01615F7F4FCE0109960E944A7C7D
:10D9500066E578E0CE0109960E94B97ABC0182E2C0
:10D960009FE00E94647BCE0109960E94B47BCE01A9
:10D970000F960E94B47B6DE578E0CE010F960E9471
:10D98000537C62E27FE0CE010F960E94CF7ABC0109
:10D99000CE0109960E944A7CBE01675F7F4FC80195
:10D9A0000E94757DCE0109960E94B47BCE010F9630
:10D9B0000E94B47B4D815E816F81788521E0CE012C
:10D9C00009960E94BC7BBE01675F7F4F82E29FE0A9
:10D9D0000E947B7BCE0109960E94B47B6FE678E0C3
:10D9E000CE010F960E94537C62E27FE0CE010F963B
:10D9F0000E94CF7A60E878E00E94B97ABC01CE013B
:10DA000009960E944A7CBE01675F7F4FC8010E9451
:10DA1000757DCE0109960E94B47BCE010F960E94BF
:10DA2000B47B4091E10B5091E20B6091E30B70915C
:10DA3000E40B22E0CE010F960E94BC7B67E878E001
:10DA4000CE0145960E94537CBE01615F7F4FCE019F
:10DA500045960E94CF7A69E978E00E94B97ABC01C4
:10DA6000CE0109960E944A7CBE01675F7F4FC801C4
:10DA70000E94757DCE0109960E94B47BCE01459629
:10DA80000E94B47BCE010F960E94B47B4091DD0BC7
:10DA90005091DE0B6091DF0B7091E00B22E0CE0124
:10DAA0000F960E94BC7B62EA78E0CE0145960E9408
:10DAB000537CBE01615F7F4FCE0145960E94CF7AB5
:10DAC00069E978E00E94B97ABC01CE0109960E940A
:10DAD0004A7CBE01675F7F4FC8010E94757DCE0101
:10DAE00009960E94B47BCE0145960E94B47BCE017C
:10DAF0000F960E94B47BE6EF2E16EFEF3E062CF455
:10DB000068EF7BE0C8010E94481E65ED7AE0C8011D
:10DB10000E94481E98E8E92E9FE0F92E27EDA22EDC
:10DB200022E0B22ECC24C394D12C4701F8E08F0E12
:10DB3000911C82E0A80EB11C8091880F9091890FF2
:10DB40008C159D050CF464C0B601CE010F960E94A1
:10DB5000A17968EC77E0CE0145960E94537CBE0126
:10DB6000615F7F4FCE0145960E94CF7A60E476E0F8
:10DB70000E94B97ABC01CE0109960E944A7CBE017E
:10DB8000675F7F4FC8010E94757DB701645E7F4F5C
:10DB9000CE014B960E94537CBE01655E7F4FC8014B
:10DBA0000E94757D60EB78E0C8010E946D7DF501F3
:10DBB00060817181660F771F660F771F6C56704FFB
:10DBC000CE0181960E94537CBE016F5D7F4FC801DC
:10DBD0000E94757D65EB78E0C8010E946D7DCE01E5
:10DBE00081960E94B47BCE014B960E94B47BCE01FD
:10DBF00009960E94B47BCE0145960E94B47BCE016B
:10DC00000F960E94B47BFFEFCF1ADF0A74018DCF0D
:10DC1000CE0187960E94B47B81E08093520C66EB24
:10DC20007BE0C8010E94481E1092F80BAC960FB61C
:10DC3000F894DEBF0FBECDBFDF91CF911F910F9142
:10DC4000FF90EF90DF90CF90BF90AF909F908F901C
:10DC50007F906F905F904F903F902F90089568EF66
:10DC60007BE0C8010E94481EDACF8F929F92AF924C
:10DC7000BF92CF92DF92EF92FF920F931F93CF93B9
:10DC8000DF93CDB7DEB7A0970FB6F894DEBF0FBE17
:10DC9000CDBF6DE174E08CE49FE00E9497796DE167
:10DCA00074E080E49FE00E94977948E4842E42E08B
:10DCB000942E58E8C52E5FE0D52E61EDA62E62E0C9
:10DCC000B62E77EDE72E72E0F72E01E010E0F401BA
:10DCD00081919191A191B1914F01892B8A2B8B2B2D
:10DCE00019F5F70182819381F50120813181821735
:10DCF0009307D1F0880F991FFC01E759F44FD80121
:10DD0000AA0FBB1FA655B44F60818C910E94877EDD
:10DD1000F70182819381F5019183808364E670E04D
:10DD200080E090E00E94407FF501619171915F0178
:10DD30008091880F9091890F801791070CF4E2C2AF
:10DD4000CE0145960E94A179B801CE010F960E949E
:10DD5000A179B601645E7F4FCE0109960E94537C83
:10DD600060E476E0CE0101960E94537CBE01675FBD
:10DD70007F4FCE0101960E94CF7A6BEB78E00E9434
:10DD8000B97ABE01615F7F4F0E94CF7A63E476E08B
:10DD90000E94B97ABE016B5E7F4F0E94CF7ABC01B0
:10DDA0008CE49FE00E94387BCE0101960E94B47BF8
:10DDB000CE0109960E94B47BCE010F960E94B47BDF
:10DDC000CE0145960E94B47B0F5F1F4FF8E0CF0E47
:10DDD000D11C22E0E20EF11C0430110509F077CFCE
:10DDE000E091A210F091A310EE0FFF1FE153FD4F41
:10DDF00060817181CE0101960E94A17946E050E0D8
:10DE0000BE016F5F7F4FCE0109960E94AE22BE0118
:10DE1000675F7F4F80E49FE00E94387BCE010996C8
:10DE20000E94B47BCE0101960E94B47BE091A410C5
:10DE3000F091A510EE0FFF1FE153FD4F608171813E
:10DE4000CE0101960E94A17946E050E0BE016F5FCD
:10DE50007F4FCE0109960E94AE22BE01675F7F4FC1
:10DE600080E49FE00E94387BCE0109960E94B47B3B
:10DE7000CE0101960E94B47B60E476E0CE01459627
:10DE80000E94537C0E940F8228EE33E040E050E075
:10DE90000E9411AD69017A016DE174E0CE014B96EB
:10DEA0000E94537C6DE174E082E59FE00E949779C7
:10DEB000CE0101960E94092244E150E0BE016F5F4D
:10DEC0007F4FCE0109960E94AE22BE01675F7F4F51
:10DED00082E59FE00E947B7BCE0109960E94B47B85
:10DEE000CE0101960E94B47B2AE0B701A601CE01C3
:10DEF00009960E94F27B48E050E0BE01675F7F4FC9
:10DF0000CE010F960E94AE2262E57FE0CE0101961F
:10DF10000E944A7CBE01615F7F4FCE0101960E9444
:10DF2000CF7ABC0186E49FE00E94647BCE0101961B
:10DF30000E94B47BCE010F960E94B47BCE0109965D
:10DF40000E94B47B2AE0B701A601CE0109960E9487
:10DF5000F27B6EEB78E0CE0101960E94537CBE010D
:10DF6000675F7F4FCE0101960E94CF7ABE016B5E44
:10DF70007F4F0E94CF7ABC0182E59FE00E94387BF0
:10DF8000CE0101960E94B47BCE0109960E94B47B1B
:10DF90004091E10B5091E20B6091E30B7091E40B27
:10DFA00021E0CE0101960E94BC7BBE016F5F7F4FD6
:10DFB000CE014B960E947B7BCE0101960E94B47BE2
:10DFC00065EC78E0CE0101960E94537CBE01655E4F
:10DFD0007F4FCE0101960E94CF7ABE016B5E7F4FCC
:10DFE0000E94CF7ABC0182E59FE00E94387BCE017F
:10DFF00001960E94B47BBE01655E7F4FCE01019603
:10E000000E944A7C46E050E0BE016F5F7F4FCE0128
:10E0100009960E94AE22BE01675F7F4F86E49FE0B3
:10E020000E94387BCE0109960E94B47BCE010196F6
:10E030000E94B47B4091DD0B5091DE0B6091DF0BB1
:10E040007091E00B21E0CE0101960E94BC7BBE01E5
:10E050006F5F7F4FCE014B960E947B7BCE01019676
:10E060000E94B47B63ED78E0CE0101960E94537C60
:10E07000BE01655E7F4FCE0101960E94CF7ABE0140
:10E080006B5E7F4F0E94CF7ABC0182E59FE00E94C9
:10E09000387BCE0101960E94B47BBE01655E7F4F46
:10E0A000CE0101960E944A7C46E050E0BE016F5FBF
:10E0B0007F4FCE0109960E94AE22BE01675F7F4F5F
:10E0C00086E49FE00E94387BCE0109960E94B47BD3
:10E0D000CE0101960E94B47B60918E0270918F02F6
:10E0E00080918C0290918D020E941E1B9093EE0BEA
:10E0F0008093ED0B892B71F060918E0270918F02ED
:10E1000080918C0290918D020E941E1B9093EE0BC9
:10E110008093ED0B8091ED0B9091EE0B8C3F9F4F18
:10E120000CF410C10E94C36929833A834B835C833A
:10E130006D837E838F83988749815A816B817C812F
:10E1400021E0CE0109960E94BC7BBE01675F7F4F34
:10E15000CE014B960E947B7BCE0109960E94B47B38
:10E160006DED78E0CE0109960E94537CBE01655E9C
:10E170007F4FCE0109960E94CF7ABE016B5E7F4F22
:10E180000E94CF7ABC0182E59FE00E94387BCE01DD
:10E1900009960E94B47BBE01655E7F4FCE01099651
:10E1A0000E944A7C46E050E0BE01675F7F4FCE018F
:10E1B0000F960E94AE22BE01615F7F4F86E49FE012
:10E1C0000E94387BCE010F960E94B47BCE01099647
:10E1D0000E94B47B4D815E816F81788521E0CE0104
:10E1E00009960E94BC7BBE01675F7F4FCE014B96B4
:10E1F0000E947B7BCE0109960E94B47B68EE78E09A
:10E20000CE0109960E94537CBE01655E7F4FCE0110
:10E2100009960E94CF7ABE016B5E7F4F0E94CF7A33
:10E22000BC0182E59FE00E94387BCE0109960E94E6
:10E23000B47BBE01655E7F4FCE0109960E944A7C89
:10E2400046E050E0BE01675F7F4FCE010F960E940F
:10E25000AE22BE01615F7F4F86E49FE00E94387B63
:10E26000CE010F960E94B47BCE0109960E94B47B2A
:10E270006CE47FE082E59FE00E94387B60E476E01A
:10E28000CE0101960E94537C60E47FE0CE010196AE
:10E290000E94CF7ABC0186E49FE00E94387BCE01C9
:10E2A00001960E94B47B66E47FE0CE0101960E9455
:10E2B0004A7CCE0101960E94F01ACE0101960E947E
:10E2C000B47B6AE070E080E090E00E94407FCE0185
:10E2D0004B960E94B47BCE0145960E94B47BA096DB
:10E2E0000FB6F894DEBF0FBECDBFDF91CF911F9167
:10E2F0000F91FF90EF90DF90CF90BF90AF909F90E5
:10E300008F900895CE0145960E94A179B801CE0163
:10E310000F960E94A179B6016C5E7F4FCE010996DF
:10E320000E94537C60E476E0CE0101960E94537C0B
:10E33000BE01675F7F4FCE0101960E94CF7A6AEBE4
:10E3400078E01DCD6EEE78E082E59FE00E942E7BA6
:10E350006DEF78E086E49FE00E942E7B64E079E038
:10E3600082E59FE00E942E7B6DEF78E086E49FE0DF
:10E370000E942E7B7DCFBF92CF92DF92EF92FF92D1
:10E380000F931F93CF93DF93CDB7DEB7C455D10959
:10E390000FB6F894DEBF0FBECDBF6C018B01659642
:10E3A0005FAF4EAF65978091DB0B9091DC0B0196D0
:10E3B0009093DC0B8093DB0B8091F80B81113CC0B8
:10E3C000BB24B394B092F80B1092DC0B1092DB0BD1
:10E3D0006DE174E0CE01895B9F4F0E94537C6DE13B
:10E3E00074E0CE01835B9F4F0E94537C50E040E07D
:10E3F0006EE174E0C6010E94611E0130110509F052
:10E40000A6C06DE174E082E59FE00E949779659671
:10E41000EEADFFAD65978081811124C00E94356EFD
:10E42000B092520CCE01835B9F4F0E94B47BCE0111
:10E43000895B9F4F0E94B47B0FB6F894DEBF0FBE7E
:10E44000CDBFCC5ADF4F0FB6F894DEBF0FBECDBFA5
:10E45000DF91CF911F910F91FF90EF90DF90CF90C0
:10E46000BF9008956596EEADFFAD659780818823D6
:10E4700009F467C000E210E09E012F5F3F4F40E2C9
:10E4800050E0BE016F5D7F4FCE018D5A9F4F0E94BD
:10E490007876049739F3BE016F5D7F4FCE018F5BB5
:10E4A0009F4F0E94537CBE016F5B7F4FCE01895B03
:10E4B0009F4F0E947B7BCE018F5B9F4F0E94B47B5E
:10E4C000BE016F5F7F4FCE018F5B9F4F0E94537CD9
:10E4D000BE016F5B7F4FCE01835B9F4F0E947B7BB2
:10E4E000CE018F5B9F4F0E94B47BBE01695B7F4F63
:10E4F00082E59FE00E94387B63968EAD9FAD639767
:10E50000892B09F4AFCF63E476E0CE018F5B9F4F98
:10E510000E94537CBE01635B7F4FCE018F5B9F4F98
:10E520000E94CF7A60E476E00E94B97ABC0182E56D
:10E530009FE00E94387BCE018F5B9F4F0E94B47B8F
:10E5400091CF62E57FE08EE29FE00E94647B1092B3
:10E55000F80B68CF0895089508950895AF92BF927B
:10E56000CF92DF92EF92FF920F931F93CF93DF939F
:10E570006C017B018B01040F151FEB015E01AE18CE
:10E58000BF08C017D10759F06991D601ED91FC91F0
:10E590000190F081E02DC6011995892B79F7C5010D
:10E5A000DF91CF911F910F91FF90EF90DF90CF906F
:10E5B000BF90AF900895FC01538D448D252F30E01E
:10E5C000842F90E0821B930B541710F0CF96089580
:10E5D00001970895FC01918D828D981761F0A28DAD
:10E5E000AE0FBF2FB11D5D968C91928D9F5F9F7373
:10E5F000928F90E008958FEF9FEF0895FC01918D29
:10E60000828D981731F0828DE80FF11D858D90E095
:10E6100008958FEF9FEF0895FC01918D228D892F32
:10E6200090E0805C9F4F821B91098F73992708951A
:10E6300088E89CE00E940C7321E0892B09F420E01B
:10E64000822F089585E29DE00E940C7321E0892BC2
:10E6500009F420E0822F0895FC01A48DA80FB92FA2
:10E66000B11DA35ABF4F2C91848D90E001968F73FA
:10E670009927848FA689B7892C93A089B1898C9119
:10E68000837080648C93938D848D981306C0028868
:10E69000F389E02D80818F7D80830895EF92FF9232
:10E6A0000F931F93CF93DF93EC0181E0888F9B8DB5
:10E6B0008C8D98131AC0E889F989808185FF15C06F
:10E6C0009FB7F894EE89FF896083E889F989808192
:10E6D0008370806480839FBF81E090E0DF91CF9161
:10E6E0001F910F91FF90EF900895F62E0B8D10E083
:10E6F0000F5F1F4F0F731127E02E8C8D8E110CC0F2
:10E700000FB607FCFACFE889F989808185FFF5CF3C
:10E71000CE010E942C73F1CFEB8DEC0FFD2FF11D7C
:10E72000E35AFF4FF0829FB7F8940B8FEA89FB8979
:10E7300080818062CFCFCF93DF93EC01888D8823D7
:10E74000B9F0AA89BB89E889F9898C9185FD03C054
:10E75000808186FD0DC00FB607FCF7CF8C9185FF39
:10E76000F2CF808185FFEDCFCE010E942C73E9CFDF
:10E77000DF91CF91089580E090E0892B29F00E94ED
:10E78000227381110E94000080E090E0892B49F003
:10E7900080E090E0892B29F00E94000081110E9406
:10E7A000000080E090E0892B49F080E090E0892B28
:10E7B00029F00E94000081110E94000080E090E09A
:10E7C000892B29F00E94187381110C940000089580
:10E7D0008150823108F05AC0E82FF0E08827EC50D1
:10E7E000FC488F4F0C94A7AE1474187406740C7404
:10E7F000107446741B74217425742B742F74337435
:10E8000039743D744674417447744B748091800030
:10E810008F77809380000895809180008F7DF9CF5D
:10E8200080918000877FF5CF84B58F7784BD089570
:10E8300084B58F7DFBCF8091B0008F778093B0003F
:10E8400008958091B0008F7DF9CF809190008F77EF
:10E85000809390000895809190008F7DF9CF8091F2
:10E860009000877FF5CF8091A0008F778093A000E4
:10E8700008958091A0008F7DF9CF8091A000877FBF
:10E88000F5CF809120018F778093200108958091AA
:10E8900020018F7DF9CF80912001877FF5CFCF9325
:10E8A000DF93282F30E0F901E95BF34F8491F90100
:10E8B000E85FF24FD491F901E25BF24FC491CC23AF
:10E8C000A1F081110E94E873EC2FF0E0EE0FFF1F22
:10E8D000E35DF34FA591B491EC91ED2381E090E0DD
:10E8E00009F480E0DF91CF91089580E090E0FACFC5
:10E8F00020917611260F3327331F21323105ECF496
:10E9000020917D0CFC0190E080E0243069F082E0F1
:10E910000895A09176112191AC014A5A5E4EA40F40
:10E92000B52FB11D2C930196861798F3809176111F
:10E93000680F6093761180E0089581E00895E0917A
:10E94000460C8091450CE81730F4F0E0EE54F44F9B
:10E95000808190E008958FEF9FEF08959091460C8D
:10E960008091450C2FEF3FEF981748F4E92FF0E026
:10E97000EE54F44F208130E09F5F9093460CC90124
:10E9800008958091450C9091460C891B990B089530
:10E99000CF92DF92EF92FF920F931F93CF93DF936B
:10E9A0007C01CB018A012091830C222389F0EB01A9
:10E9B0006B01C40ED51ECC15DD0569F06991D70138
:10E9C000ED91FC910190F081E02DC7011995F3CFF5
:10E9D000642F0E947874C801DF91CF911F910F912D
:10E9E000FF90EF90DF90CF900895CF93DF931F9229
:10E9F000CDB7DEB769832091830C2223F9F02091F3
:10EA0000860C203258F021E030E0FC013383228371
:10EA100090E080E00F90DF91CF9108958091840C79
:10EA2000E82FF0E0E550FB4E998190838F5F809353
:10EA3000840C8093860C81E090E0ECCF61E0CE0105
:10EA400001960E947874F7CF0E94D0B00F931F9365
:10EA5000CF93DF93EC0188819981009759F02A8147
:10EA60003B812617370730F081E0DF91CF911F916E
:10EA70000F9108958B016F5F7F4F0E94EFAF00975A
:10EA800059F0998388831B830A832C813D81232B32
:10EA900059F7FC011082E8CF80E0E7CFEF92FF92B8
:10EAA0000F931F93CF93DF936115710541F480E0BD
:10EAB000DF91CF911F910F91FF90EF900895411535
:10EAC0005105B1F07B01EC010C811D81040F151F74
:10EAD000B8010E942675882351F3288139818C81E1
:10EAE0009D81B701820F931F0E9420B11D830C836B
:10EAF00081E0DECFCF93DF93EC018881998100978D
:10EB000011F00E9466AF198218821D821C821B823E
:10EB10001A82DF91CF910895EF92FF920F931F9386
:10EB2000CF93DF93EC017B018A01BA010E94267525
:10EB300081110BC0CE010E947A75CE01DF91CF9179
:10EB40001F910F91FF90EF9008951D830C83B701E3
:10EB5000888199810E9420B1F0CF80915011882343
:10EB6000A9F1409168025091690260916A02709126
:10EB70006B022FE832E180918F14909190140E94E3
:10EB8000930C811102C080E0089540915111509181
:10EB90005211609153117091541141155105610545
:10EBA000710591F02FE832E180918F1490919014CB
:10EBB0000E94930C882339F3109251111092521134
:10EBC00010925311109254111092501181E0089537
:10EBD0008F929F92AF92BF92EF92FF920F931F93EB
:10EBE000CF934B015C01C42F809168029091690220
:10EBF000A0916A02B0916B0288159905AA05BB0520
:10EC000049F10E94AD7581110BC080E0CF911F9139
:10EC10000F91FF90EF90BF90AF909F908F900895CD
:10EC20008FE8E82E82E1F82E00E012E030E020E0EC
:10EC3000B501A40180918F14909190140E94EC0B67
:10EC4000882319F38092680290926902A0926A0266
:10EC5000B0926B02409150114C2B4093501181E0C7
:10EC6000D5CF8CBD9DBD0895CF93DF93EC019A0164
:10EC7000AB01E889F98982E08083211581EE3807AC
:10EC80004105510581F160E079E08DE390E00E945B
:10EC900011AD2150310941095109569547953795D4
:10ECA0002795EC85FD851082EE85FF852083188EE3
:10ECB000EC89FD8986E08083EA89FB898081806117
:10ECC0008083EA89FB89808188608083EA89FB8967
:10ECD000808180688083EA89FB8980818F7D808341
:10ECE000DF91CF910895E889F989108220E1D9CF89
:10ECF0002F923F924F925F926F927F928F929F924C
:10ED0000AF92BF92CF92DF92EF92FF920F931F9339
:10ED1000CF93DF9300D0CDB7DEB71C013B014A0192
:10ED200029015801FC01C080D18070E060E0C3017E
:10ED30000E9405B1A80170E060E0C2010E9405B127
:10ED4000F601808110E000E0811162C004E010E073
:10ED500004C07601F101F182E082C8010F900F90AA
:10ED60000F90DF91CF911F910F91FF90EF90DF9067
:10ED7000CF90BF90AF909F908F907F906F905F905B
:10ED80004F903F902F9008956B3209F482C06D33FD
:10ED900009F04EC081818823E9F2F7018FEFE81A6C
:10EDA000F80A6081653209F452C00CF048C066234D
:10EDB00009F456C082E0A816B1040CF061C0012B22
:10EDC00009F46BC003E010E0E8CF818189838823D8
:10EDD00009F282818A837601811104C0F2E0EF0E8C
:10EDE000F11CB8CF83E0E80EF11C1B8240E150E03B
:10EDF00070E060E0CE0101960E948AA319C0F30181
:10EE00006083F1E08F1A9108C30101963C0167010C
:10EE10007601FFEFEF1AFF0AF6016081663209F40E
:10EE200099CF0CF0B1CF662309F493CF653269F224
:10EE3000F2E08F1691041CF701E010E0E8CF663293
:10EE400009F488CF6B3209F0B5CF60E2B3CF81818E
:10EE50008983882301F182818A83811103C03296DC
:10EE60007F0178CF7F0193E0E90EF11C1B8240E126
:10EE700050E070E060E0CE0101960E948AA39ACF34
:10EE8000F2016083F1E0AF1AB108C20101962C01D2
:10EE900084CF60E2CDCFF701E3CF02E010E07DCF79
:10EEA0000F931F93CF93DF934115510541F0FC0160
:10EEB000048115810115110539F4FB011082DF91E0
:10EEC000CF911F910F91089541505109401751075B
:10EED00008F48A01EB01FC0160817181A801CE0177
:10EEE0000E9435B1C00FD11F1882E9CF20E3FC0189
:10EEF00020833296862F82958F706F706A3030F43F
:10EF0000605D6293682F8111F5CF0895695CF9CF38
:10EF10008F929F92AF92BF92CF92DF92EF92FF9229
:10EF2000CF932EEC3DE03093901420938F148823E0
:10EF300009F46DC040E060E070E0CB010E94E8752C
:10EF400081110BC080E0CF91FF90EF90DF90CF90C8
:10EF5000BF90AF909F908F90089580914D148F77C0
:10EF600089F78091591490915A14A0915B14B09133
:10EF70005C1484369105A105B10520F3C0905514A9
:10EF8000D0905614E0905714F0905814C114D10446
:10EF9000E104F104B9F240E0C701B6010E94E8754E
:10EFA000882381F280919A1290919B128115924050
:10EFB00049F6A0919F12AA2329F260919D127091A7
:10EFC0009E126115710509F4BDCF20919C12222378
:10EFD00009F4B8CFA093EC0D2093DE0D90E080E013
:10EFE00030E0E1E0F0E0C82FAF01082E02C0440F8E
:10EFF000551F0A94E2F72417350769F041E0480FDE
:10F0000001968930910579F74093E70D9BCFC12C8C
:10F01000D12C7601C0CF8093E70D2091A5123091BD
:10F02000A61250E040E02115310541F42091B312C1
:10F030003091B4124091B5125091B6122093DF0D69
:10F040003093E00D4093E10D5093E20D46015701DE
:10F05000860E971EA11CB11C8092ED0D9092EE0DB4
:10F06000A092EF0DB092F00DE091A012F091A112DC
:10F07000F093F30DE093F20DB0E00E9452ADDC018D
:10F08000CB01880D991DAA1DBB1D8093F40D909393
:10F09000F50DA093F60DB093F70D25E0EE0FFF1FD1
:10F0A0002A95E1F7E150FE4FEF2FFF27E6958E0FEF
:10F0B0009F1FA11DB11D8093E80D9093E90DA093B2
:10F0C000EA0DB093EB0D8090A2129090A312B12C98
:10F0D000A12C8114910441F48090AF129090B01251
:10F0E000A090B112B090B212C81AD90AEA0AFB0A6B
:10F0F000C80CD91CEA1CFB1C04C0F694E794D794F6
:10F10000C794CA95D2F7C092E30DD092E40DE09275
:10F11000E50DF092E60D85EFC8168FE0D806E10404
:10F12000F10428F48CE08093F10D81E00CCF80E1B4
:10F1300025EFC2162FEFD206E104F104A0F380916F
:10F14000BB129091BC12A091BD12B091BE128093DF
:10F15000F40D9093F50DA093F60DB093F70D80E2AA
:10F16000E2CF8F929F92AF92BF92CF92DF92EF92B7
:10F17000FF920F931F93CF93DF93CDB7DEB76097C6
:10F180000FB6F894DEBF0FBECDBF7C0190914A0C44
:10F19000992351F108E0933309F404E06B0180E511
:10F1A00091E00E9431769E012F5F3F4F5901490146
:10F1B00010E0812F0E94840FF40181934F01882376
:10F1C000D9F01F5F0113F5CF00E0F50181915F01D8
:10F1D0008D3161F0883151F08A51823038F00F5F03
:10F1E0001013F3CF0E94FF1018E08AC060E170E0B6
:10F1F000802F0E94E20F102FA12EB12CF501EE0FEF
:10F20000FF1FEB5CF34F1182108283EE93E00197B6
:10F21000F1F742E870E060E0812F0E94C50F4FEFE8
:10F2200062E070E0812F0E94C50FB601C114D104C5
:10F2300091F4809190029091910201968115F0ECE9
:10F240009F0708F471C0909391028093900260919F
:10F25000900270919102812F0E94AF0F86E0E5E24B
:10F26000F3E0DE01199601900D928A95E1F7F7011E
:10F2700083818F778C8784818D8785818E87A70195
:10F280004E5F5F4F24E030E06CE070E0812F0E9421
:10F29000880FB601812F0E94990F26E030E0AE0161
:10F2A000475F5F4F66E070E0812F0E94880F61E04A
:10F2B00070E0812F0E94E20F27E02A9DC0012B9D64
:10F2C000900D11249C012350344F7901F9011182D2
:10F2D000108222E030E0AE01415F5F4F68E270E0F3
:10F2E000812F0E94F20F8F85988998278927982768
:10F2F000F701938382831682158214820E94FF1085
:10F30000812F60960FB6F894DEBF0FBECDBFDF91A0
:10F31000CF911F910F91FF90EF90DF90CF90BF9012
:10F32000AF909F908F90089580E090EC8CCFFB0180
:10F3300001900020E9F73197AF01461B570B0C9461
:10F340008C750F931F93CF93DF93CDB7DEB7629782
:10F350000FB6F894DEBF0FBECDBF8C01CB01F80114
:10F360001182108213821282158214824AE0BE0139
:10F370006F5F7F4F0E94D1A4BE016F5F7F4FC801B6
:10F380000E94977962960FB6F894DEBF0FBECDBF8C
:10F39000DF91CF911F910F9108950F931F93CF93FA
:10F3A000DF93CDB7DEB7A1970FB6F894DEBF0FBEDF
:10F3B000CDBF8C01CB01BA01F801118210821382FA
:10F3C0001282158214822AE0AE014F5F5F4F0E94C5
:10F3D0000BA5BE016F5F7F4FC8010E949779A19670
:10F3E0000FB6F894DEBF0FBECDBFDF91CF911F9156
:10F3F0000F910895FC0180819181009711F00C9488
:10F400008DA460E070E0CB010895FC0180819181C2
:10F41000009711F00C9491A460E070E0CB01089586
:10F42000AF92BF92CF92DF92EF92FF920F931F9312
:10F43000CF93DF93DC01CD90DC901197C114D10400
:10F4400039F01496CD91DC918C017601209761F40E
:10F45000DF91CF911F910F91FF90EF90DF90CF90B0
:10F46000BF90AF90089575015701BFEFAB1ABB0A6B
:10F47000F7018081082E000C990B0E94B8A4892BFB
:10F4800091F72197CC0DDD1D8881082E000C990B7A
:10F490000E94B8A4892B29F0CE15DF0510F0219722
:10F4A000F3CFAE014F5F5F4F4E195F09D80115963C
:10F4B0005C934E931497CE14DF0420F4B701C60179
:10F4C0000E94EAB0D801ED91FC91119714968D91AC
:10F4D0009C91E80FF91F1082BBCFFC01248135817C
:10F4E0006217730748F480819181009729F0860F95
:10F4F000971FFC018081089580E00895FC0124811C
:10F500003581FB014481558124173507A0F0FC01AA
:10F5100080819181009779F0FB0160817181611593
:10F52000710549F0241B350B820F931F0E9417B100
:10F5300021E0892B09F020E0822F0895FB0144810E
:10F540005581FC01248135812417350778F08081AD
:10F550009181009759F0FB016081718161157105FE
:10F5600029F00E9427B121E0892B09F020E0822FA9
:10F570000895CF93DF93EC01FB0101900020E9F7A0
:10F580003197AF01461B570B0E944E75811103C086
:10F59000CE010E947A75CE01DF91CF910895CF936D
:10F5A000DF93EC01FB0144815581608171810E94F0
:10F5B0004E75811103C0CE010E947A75CE01DF9194
:10F5C000CF910895EF92FF920F931F93CF93DF9304
:10F5D000EC017B01CB010E94C8A40097A9F00C812B
:10F5E0001D81080F191FB801CE010E9426758823BE
:10F5F00061F0288139818C819D81B701820F931F31
:10F600000E94C1A41D830C8381E0DF91CF911F91E3
:10F610000F91FF90EF900895CF93DF931F921F9269
:10F62000CDB7DEB769831A8241E050E0BE016F5F5B
:10F630007F4F0E944E750F900F90DF91CF910895EC
:10F64000CF93DF93EC010E940C7B811103C0CE01AC
:10F650000E947A75CE01DF91CF910895FB01019050
:10F660000020E9F73197AF01461B570B0C944E75FC
:10F67000FB0144815581608171810C944E75EF923C
:10F68000FF920F931F93CF93DF93EC018B01CB017C
:10F690000E94C8A47C01BC01CE010E942675811184
:10F6A0000BC0CE010E947A75CE01DF91CF911F91E0
:10F6B0000F91FF90EF900895FD82EC82B801888150
:10F6C00099810E94C1A4F0CFCF93DF93EC01FB019D
:10F6D0008617970749F0608171816115710541F0C6
:10F6E000448155810E948C75CE01DF91CF910895A0
:10F6F0000E947A75F9CF0F931F93CF93DF938C01FC
:10F70000EB01FC01808191810097E1F068817981B2
:10F7100061157105A9F0428153812C813D81421709
:10F72000530770F00E9420B18C819D81F801958370
:10F7300084831D821C82DF91CF911F910F910895C8
:10F740000E9466AF88819981F801918380838A81C4
:10F750009B81938382838C819D819583848319828D
:10F7600018821B821A82E5CFFC018081918100976B
:10F7700011F00C9466AF0895EF92FF920F931F93D0
:10F78000CF93DF93CDB7DEB7A1970FB6F894DEBF66
:10F790000FBECDBF7C01CB01BA01F70111821082EF
:10F7A000138212821582148242E0420F8E010F5F93
:10F7B0001F4F0E94C8A2009789F0BC01C7010E9498
:10F7C0009779A1960FB6F894DEBF0FBECDBFDF913B
:10F7D000CF911F910F91FF90EF900895C7010E9464
:10F7E0007A75EFCF0F931F93CF93DF93CDB7DEB72B
:10F7F000A2970FB6F894DEBF0FBECDBF8C01CB0130
:10F80000BA01F801118210821382128215821482C9
:10F8100030E0AE014F5F5F4F0E94DCA4BE016F5F1E
:10F820007F4FC8010E949779A2960FB6F894DEBF69
:10F830000FBECDBFDF91CF911F910F910895CF9350
:10F84000DF931F921F92CDB7DEB7FC0111821082A9
:10F85000138212821582148269831A82BE016F5F3D
:10F860007F4F0E9497790F900F90DF91CF9108956D
:10F87000FC011182108213821282158214820C9470
:10F880007B7BFC011182108213821282158214820A
:10F890000C943F7BFC01118210821382128215822C
:10F8A00014820C94647BFC011182108213821282F8
:10F8B000158214826115710551F0FB010190002041
:10F8C000E9F73197AF01461B570B0C948C750895DF
:10F8D000AF92BF92CF92DF92EF92FF920F931F935E
:10F8E000CF93DF936C015B017A01890124173507FF
:10F8F00020F48F2D7901042F182F6DE174E0C601DB
:10F900000E94537CD5011496CD91DC91EC16FD0636
:10F91000E0F40C171D0708F4E801D501ED91FC9106
:10F920001197EC0FFD1F108110826D917C916E0D6F
:10F930007F1DC60161157105A1F00E949779F5013F
:10F9400080819181C80FD91F1883C601DF91CF91A3
:10F950001F910F91FF90EF90DF90CF90BF90AF90ED
:10F9600008950E947A75EBCFFB0101900020E9F722
:10F970003197AF01461B570BDC01ED91FC910280E2
:10F98000F381E02D19948F929F92AF92BF92EF92E4
:10F99000FF920F931F93CF93DF93CDB7DEB7A1975D
:10F9A0000FB6F894DEBF0FBECDBF7C01FA01CB01CC
:10F9B00019A2223008F42AE08E010F5D1F4F822E1B
:10F9C000912CB12CA12CBF01A50194010E9411AD75
:10F9D000F901CA016A300CF5605DD8016E938D01A2
:10F9E000232B242B252B79F790E080E0109721F032
:10F9F000BD01C7010E94B47CA1960FB6F894DEBF8A
:10FA00000FBECDBFDF91CF911F910F91FF90EF906F
:10FA1000BF90AF909F908F900895695CDECF8F92DA
:10FA20009F92AF92BF92CF92DF92EF92FF920F938D
:10FA30001F93CF93DF937C01EB016C0182E0C80E32
:10FA4000D11C4701E5E08E0E911C10E000E0F601AC
:10FA500041916F0150E070E060E02AE0CE010E9429
:10FA6000C37C5C01E881F9810190F081E02D6EE2B8
:10FA7000CE0119958A0D9B1D080F191FC814D904B2
:10FA800031F7F701458150E070E060E02AE0CE01F7
:10FA90000E94C37C800F911FDF91CF911F910F9126
:10FAA000FF90EF90DF90CF90BF90AF909F908F909E
:10FAB00008950F931F93CF93DF93EC010E94B47CC2
:10FAC0008C0167E779E0CE010E94B47C800F911F22
:10FAD000DF91CF911F910F9108956115710511F07C
:10FAE0000C94B47C90E080E00895DB0114964D9175
:10FAF0005C9115976D917C91DC01ED91FC910280F8
:10FB0000F381E02D19940F931F93CF93DF93EC01B2
:10FB10000E94757D8C0167E779E0CE010E94B47C7C
:10FB2000800F911FDF91CF911F910F910895EF9258
:10FB3000FF920F931F93CF93DF938C017B01D0E053
:10FB4000C0E0F701EC0FFD1F6491662361F0D8015E
:10FB5000ED91FC910190F081E02DC8011995892B60
:10FB600011F02196EECFCE01DF91CF911F910F9131
:10FB7000FF90EF900895DC0182E194E08D939D93D6
:10FB800084E0FB0101900D928A95E1F708951F92A0
:10FB90000F920FB60F9211240BB60F922F933F9333
:10FBA0004F935F936F937F938F939F93AF93BF9385
:10FBB000EF93FF9388E89CE00E942C73FF91EF91F4
:10FBC000BF91AF919F918F917F916F915F914F9175
:10FBD0003F912F910F900BBE0F900FBE0F901F9073
:10FBE00018951F920F920FB60F9211240BB60F9219
:10FBF0002F938F939F93EF93FF93E091980CF09145
:10FC0000990C8081E0919E0CF0919F0C82FD1DC0AB
:10FC100090818091A10C8F5F8F732091A20C82172D
:10FC200041F0E091A10CF0E0E857F34F958F8093FD
:10FC3000A10CFF91EF919F918F912F910F900BBE8F
:10FC40000F900FBE0F901F9018958081F2CF1F92DA
:10FC50000F920FB60F9211240BB60F922F933F9372
:10FC60004F935F936F937F938F939F93AF93BF93C4
:10FC7000EF93FF9385E29DE00E942C73FF91EF913B
:10FC8000BF91AF919F918F917F916F915F914F91B4
:10FC90003F912F910F900BBE0F900FBE0F901F90B2
:10FCA00018951F920F920FB60F9211240BB60F9258
:10FCB0002F938F939F93EF93FF93E091350DF091E6
:10FCC000360D8081E0913B0DF0913C0D82FD1DC011
:10FCD000908180913E0D8F5F8F7320913F0D821731
:10FCE00041F0E0913E0DF0E0EB5DF24F958F809397
:10FCF0003E0DFF91EF919F918F912F910F900BBE31
:10FD00000F900FBE0F901F9018958081F2CF1F9318
:10FD1000CF93DF93282F30E0F901E95BF34F849113
:10FD2000F901E85FF24FD491F901E25BF24FC4911F
:10FD3000CC23A9F0162F81110E94E873EC2FF0E07C
:10FD4000EE0FFF1FEC52F34FA591B4918FB7F894CB
:10FD5000EC91111108C0D095DE23DC938FBFDF91A9
:10FD6000CF911F910895DE2BF8CF10927D0C81E08A
:10FD700080937C0C1092570C61E084E10E94877E96
:10FD800061E085E10E94877EE9EBF0E080818E7F73
:10FD9000808380818D7F808388E48093B80085E4B0
:10FDA0008093BC0008951092460C1092450C10925E
:10FDB000840C1092860C0E94B57E8BEA92E7909399
:10FDC0008E1280938D128CEA92E790938C1280931E
:10FDD0008B120895CF93DF9390E0FC01E85FF24F20
:10FDE0002491825B924FFC0184918823D1F090E0B2
:10FDF000880F991FFC01E251F34FA591B491FC01CA
:10FE0000EC52F34FC591D49161110EC09FB7F89495
:10FE10008C91E22FE0958E238C932881E223E88356
:10FE20009FBFDF91CF9108958FB7F894EC91E22BAB
:10FE3000EC938FBFF6CF3FB7F894809181129091E9
:10FE40008212A0918312B091841226B5A89B05C09E
:10FE50002F3F19F00196A11DB11D3FBFBA2FA92F49
:10FE6000982F8827BC01CD01620F711D811D911D46
:10FE700042E0660F771F881F991F4A95D1F70895B2
:10FE80008F929F92AF92BF92CF92DF92EF92FF92AA
:10FE90006B017C010E941B7F4B015C01C114D104EA
:10FEA000E104F104B9F00E941B7F681979098A09FD
:10FEB0009B09683E73408105910580F321E0C21AD9
:10FEC000D108E108F10888EE880E83E0981EA11C95
:10FED000B11CE4CFFF90EF90DF90CF90BF90AF9038
:10FEE0009F908F900895AF92BF92CF92DF92EF9242
:10FEF000FF920F931F93CF93DF93C82FD62F1092AB
:10FF0000C2101092C3101092C4101092C51010921B
:10FF1000C61061E00E94EA7E60E08C2F0E94877E1E
:10FF20006D2F70E090E080E00E94407F60E08C2FB9
:10FF30000E94EA7E8BE990E00197F1F700E911E079
:10FF40008C2F0E944F74892B81F401501109C1F745
:10FF50008EEF9FEFDF91CF911F910F91FF90EF9068
:10FF6000DF90CF90BF90AF90089500E911E08C2F03
:10FF70000E944F74019721F401501109C1F7E8CF95
:10FF800018E2D0E800E090E9E92EFF24F3948C2FEA
:10FF90000E944F74892B29F481E0E81AF108B9F71F
:10FFA000D7CF0E941B7F6B017C0180E9A82EBB2468
:10FFB000B3948C2F0E944F74019729F481E0A81A02
:10FFC000B108B9F7C5CF0E941B7F6C197D098E0956
:10FFD0009F09693271058105910538F0E02FF0E045
:10FFE000E654FF4E80858D2B8087D69511F40F5FE8
:10FFF000D0E8115041F690E080E0ACCF0F931F9312
:020000040001F9
:10000000CF93DF9300D000D01F921F92CDB7DEB701
:100010008091F11481112AC01092D9141092D81431
:1000200088EE93E0A0E0B0E08093DA149093DB14C4
:10003000A093DC14B093DD148CE993E09093D71473
:100040008093D61482E194E09093E5148093E414B5
:100050001092E6141092E7141092E8141092E9142A
:1000600088E08093EE1481E08093F11483E994E1B9
:1000700090934D0C80934C0C8091921481119DC0F3
:1000800060E372E080E090E00E94407F1FB7F89448
:1000900080919114811127C0E3E8FDE08491EDE3A4
:1000A000FDE09491E82FF0E0EE0FFF1FE251F34FD7
:1000B000A591B491EC91E92321F461E085E30E94DC
:1000C000877E61E085E30E94EA7E8CB580618CBD0D
:1000D0008CB580648CBD61E084E30E94EA7E61E0BF
:1000E00083E30E94EA7E809191148F5F8093911444
:1000F0001FBFE8E5FDE0E491F0E0EE0FFF1FEC52DA
:10010000F34F859194919093490C8093480CE2E1D0
:10011000FDE0E491E093470C61E08AE00E94EA7E12
:100120000E94E80D80E591E00E94317684E380939F
:100130004A0C80E80E94710F0E945B0F882309F42B
:10014000F5C088E00E94710F0E94480F883009F0C6
:10015000EDC080E10E94710F0E94480F803109F0CC
:10016000E5C080E00E94710F0E94480F182F811196
:10017000DDC041E050E0BE016F5F7F4F8FE190E056
:100180000E94F20D8981833009F0D0C080E4809311
:100190004B0C42E06EE170E0812F0E94C50F42E0FF
:1001A0006FE170E0812F0E94C50F1F5F183089F743
:1001B0000E94FF1081E08093921480E591E00E94FC
:1001C000317646E050E062E972E089E090E00E941A
:1001D0009A0E82E194E09A8389831B821C821D829D
:1001E0001E82CE0103960E94F8100E94FF1080919B
:1001F0004C0C90914D0CDC0192961D921D921D921B
:100200001C929597FC0116A217A210A611A69A9609
:100210001D921D921D921C929D9740E65AEE60E041
:1002200070E046AB57AB60AF71AF40EA5FE060E0B3
:1002300070E0DA964D935D936D937C93DD973E96D7
:1002400024E1DF011D922A95E9F726E0E2E9F2E0D8
:10025000DC01189601900D922A95E1F7FC01EE5B06
:10026000FF4F10820E949D298C01019709F0CBC09D
:1002700080E591E00E94317660914C0C70914D0CBC
:10028000625F7F4FCE0101960E94BB7DCE01039637
:100290000E94F81060914C0C70914D0C6A5E7F4F7B
:1002A000CE0101960E94BB7D44E050E0BE016D5F2F
:1002B0007F4F81E090E00E949A0E60914C0C70910B
:1002C0004D0C6E5E7F4FCE0101960E94BB7D44E0D7
:1002D00050E0BE016D5F7F4F85E090E00E949A0E76
:1002E0000E94FF1060914C0C70914D0C625E7F4F2C
:1002F000CE0101960E94BB7D8B819C81AD81BE8128
:100300008093190E90931A0EA0931B0EB0931C0E9F
:100310000E941B7F7F7380919002909191026827C9
:10032000792770939102609390026DC087E3809368
:100330004A0C80E80E94710F0E945B0F882329F10C
:1003400088E00E94710F0E94480F8830F1F480E12C
:100350000E94710F0E94480F182F8031B1F480E085
:100360000E94710F0E94480F81110FC041E050E0C0
:10037000BE016F5F7F4F89E390E00E94F20D89819B
:10038000843019F410934B0C13CF83E380934A0C01
:1003900080E80E94710F0E945B0F882371F180E159
:1003A0000E94710F0E94480F803139F582E10E944E
:1003B000710F0E94480F823101F580E00E94710F99
:1003C0000E94480F811119C084E080934B0C15E501
:1003D000188741E050E0BE01685F7F4F8BE190E0FD
:1003E0000E949A0E1F8341E050E0BE01695F7F4F7B
:1003F0008AE190E00E949A0EDBCE10924A0C0E9495
:10040000FF1010E000E0C80128960FB6F894DEBF98
:100410000FBECDBFDF91CF911F910F9108952FB7E0
:10042000F89460917D1270917E1280917F1290916C
:1004300080122FBF0895CF92DF92EF92FF92CF9359
:10044000DF938091330E883050F0CFEFDFEFCE0195
:10045000DF91CF91FF90EF90DF90CF900895E091E2
:10046000580EE11142C00E940F826B017C0128EE00
:10047000C20E23E0D21EE11CF11C87E29EE00E9426
:100480006515882311F380918E0E882331F08091B9
:10049000590E90915A0E892BC1F287E29EE00E947C
:1004A000C813EC01CF3FDC0771F080918E0E8823DA
:1004B00071F28091590E90915A0E019790935A0EB5
:1004C0008093590EC4CF0E940F82C616D706E80645
:1004D000F90698F61092580E87E29EE00E94C01529
:1004E00087E29EE00E948715B2CFE150E093580E5C
:1004F000F0E0E35EF14FC38DD0E0A9CF0F931F93DF
:10050000CF93DF93EC018C01F80181918F01882357
:10051000A1F10E941B82F8012291022E000C330BE4
:100520008217930789F38F3F980781F0A091580EA7
:1005300091E09A0F9093580EB0E0A35EB14F5B9696
:100540008C93903219F48FE18093580E2FE1EC17C1
:10055000FD07C9F092919F3FD1F3A091580E81E021
:100560008A0F8093580EB0E0A35EB14F5B969C93C8
:10057000803269F72093580EEACF81E0DF91CF9166
:100580001F910F91089580E0F9CF0F931F93CF93A0
:10059000DF93EC010E940F828B010E94950B8F3F2D
:1005A00069F00E940F82601B710B6C177D07A8F326
:1005B00080E0DF91CF911F910F91089581E0F9CFF5
:1005C0004F925F926F927F928F929F92AF92BF9263
:1005D000CF92DF92EF92FF920F931F93CF93DF930F
:1005E000CDB7DEB763970FB6F894DEBF0FBECDBFB1
:1005F0007C016B013A01FB0120E090E080E06AE0C1
:100600003191332309F461C040ED430F4A3008F0C3
:100610004DC0689FA001699F500D1124CA01C09769
:10062000830F911D37FD9A958F3F910549F340F354
:10063000F7014281538164817581809141159091C8
:100640004215A0914315B0914415481759076A0700
:100650007B0709F40DC28701085F1F4F0E940F82BC
:100660006F7077277C5FC8010E941817813009F0EE
:1006700004C282E194E09A838983F70182819381A5
:10068000A481B5818B839C83AD83BE8345E350E019
:10069000BE016F5F7F4FC8010E94A117892BA9F58A
:1006A000D12CC12CC8010E94441417C03E3209F05D
:1006B000BFCF233009F4BCCFD301A20FB11D1296D6
:1006C0008C932F5F90E080E09BCF233009F0B0CF78
:1006D000F3018583CC24C394D12CC60163960FB655
:1006E000F894DEBF0FBECDBFDF91CF911F910F9168
:1006F000FF90EF90DF90CF90BF90AF909F908F9042
:100700007F906F905F904F9008950E940F82F70145
:100710007783668342E050E0B7016A5F7F4FC8018C
:100720000E94361781E090E09A83898342E050E08E
:10073000BE016F5F7F4FC8010E94361780E091E0D5
:100740009A83898342E050E0BE016F5F7F4FC8010A
:100750000E9436171A82198242E050E0BE016F5F94
:100760007F4FC8010E94361742E050E0BE016F5F24
:100770007F4FC8010E94361742E050E0BE016F5F14
:100780007F4FC8010E9436175601F60180818823E9
:1007900001F16501F60181912F01882311F08E325C
:1007A000B1F446018A189B081814190474F48D8654
:1007B00041E050E0BE01635F7F4FC8010E943617E1
:1007C000A401B501C8010E9436175201DECF6201B3
:1007D000E1CF1D8641E050E0BE01635F7F4FC8015D
:1007E0000E943617C12CDD24D394DA82C98242E0FC
:1007F00050E0BE016F5F7F4FC8010E943617DA825A
:10080000C98242E050E0BE016F5F7F4FC8010E9485
:100810003617C8010E947017892B09F441CFF3E005
:10082000AF2EB12C230122E0420E511CD4C0F7019F
:100830004281538164817581808D918DA28DB38DAC
:10084000481759076A077B0709F008C1848D958D01
:10085000C59709F003C181A192A15DEFC52EDD24EA
:10086000DA940C970CF4ADC04CE050E0BE016F5F21
:100870007F4FC8010E9423138B819C819827892771
:1008800098279A8B898BF7014681578129813A8174
:100890004217530709F0E7C097FFE5C08F709270C9
:1008A0003BEFC32EDD24DA94892B09F08AC06F80D8
:1008B00078847624672476242AEFC22EDD24DA9405
:1008C0006114710409F47DC0D12CC12C8D819E81ED
:1008D000982789279827C816D906F8F441E050E0F0
:1008E000BE01635F7F4FC8010E9423134D854423DF
:1008F00031F050E070E060E0C8010E9423138D8564
:100900008111ECCF44E050E070E060E0C8010E944B
:100910002313FFEFCF1ADF0AD9CF912C812C41E0AE
:1009200050E0BE016D5E7F4FC8010E9423134B89CA
:10093000842F807C09F06CC0442331F050E070E0DB
:1009400060E0C8010E9423138B898111E8CF42E047
:1009500050E0BE01615F7F4FC8010E94231342E057
:1009600050E0BE01635F7F4FC8010E94231344E043
:1009700050E070E060E0C8010E94231342E050E0C4
:10098000BE016F5E7F4FC8010E9423138F85988937
:1009900049895A898115914009F043C0CD84DE848C
:1009A000DC24CD24DC2481E0C816D104D1F5411526
:1009B000544009F04AC044E050E0B201C8010E942E
:1009C000231321E0A21AB10809F46CCEFFEFCF1671
:1009D000DF0609F067CE0E940F823B014C01C8017F
:1009E0000E946C13181619060CF421CF0E940F8276
:1009F0006619770988099909693873418105910554
:100A000048F562E370E080E090E00E94407FE7CF2D
:100A100041E050E070E060E0C8010E9423131B8AAF
:100A200093CF54274527542770E060E0C8010E9407
:100A30002313FFEF8F1A9F0A6814790409F06FCF10
:100A400096EFC92EDD24DA94BCCFE7EFCE2EDD245D
:100A5000DA94B7CFCC24CA94DC2CB3CF6EEFC62E79
:100A6000DD24DA94AECF4CEFC42EDD24DA94A9CF86
:100A70008EEFC82EDD24DA9430CED12CC12C2DCEB1
:100A80001F920F920FB60F9211242F933F938F93C3
:100A90009F93AF93BF9380917D1290917E12A0910E
:100AA0007F12B091801230917C1223E0230F2D37FA
:100AB00058F50196A11DB11D20937C1280937D12E3
:100AC00090937E12A0937F12B09380128091811236
:100AD00090918212A0918312B09184120196A11D6F
:100AE000B11D8093811290938212A0938312B093D0
:100AF0008412BF91AF919F918F913F912F910F9051
:100B00000FBE0F901F90189526E8230F0296A11D87
:100B1000B11DD2CF609378127093791280937A12BC
:100B200090937B12645D7E4F8F4F9F4F6093741242
:100B300070937512809376129093771282E090E012
:100B400090937312809372120E940F8260936E12C0
:100B500070936F1280937012909371120895CF92D8
:100B6000DF92EF92FF920F931F930E940F828B01EF
:100B70009C01C0906E12D0906F12E0907012F090B5
:100B80007112609178127091791280917A1290911D
:100B90007B120C191D092E093F09083E134021053F
:100BA0003105E0F0DC01CB010196A11DB11D809360
:100BB000781290937912A0937A12B0937B12B701B6
:100BC000A60148515C4F6F4F7F4F40936E12509378
:100BD0006F126093701270937112C7CF1F910F91B3
:100BE000FF90EF90DF90CF900895CF93DF93EC01CB
:100BF0000E94AF859E01220F331F220F331FF90180
:100C0000E152FD4F6083718382839383CE01880F0D
:100C1000991FFC01E952FD4F4081518114161506C0
:100C200044F4FC01E153FD4F408151811416150637
:100C300014F1FC01E952FD4F41E050E05183408343
:100C400081539D4FFC015183408321543D4F88E0E7
:100C500097E0A0E0B0E0F90180839183A283B383A1
:100C6000CE010E94041A64EF71E080E090E0DF9111
:100C7000CF910C94407FDF91CF9108954F925F9276
:100C80006F927F928F929F92AF92BF92CF92DF929C
:100C9000EF92FF920F931F93CF93DF934B015C0171
:100CA00080916A1290916B12A0916C12B0916D12AA
:100CB00088159905AA05BB0509F4C6C08CE3C82EA2
:100CC000D12CE12CF12CC501A70196010E9411AD98
:100CD0006093D20BCA01B901A70196010E9411AD20
:100CE0006093D30BC501B40120E13EE040E050E049
:100CF0000E9411ADCA01B90128E130E040E050E0A6
:100D00000E9411AD6093D40BC501B40120E831E518
:100D100041E050E00E9411AD69017A01CA01B901B8
:100D20006C5F7F4F8F4F9F4F27E030E040E050E0F7
:100D30000E9411AD6F5F6093D50B412C512C320195
:100D400040E004E610E0C0E9D1E0242F30E02E546A
:100D5000384FF901E370FF273097F9F4C901B80162
:100D60000E9493AE892B31F4C901BE010E9493AE5B
:100D7000892B99F48EE691E0A0E0B0E0480E591E70
:100D80006A1E7B1ED301C201AA27BB27C816D9063B
:100D9000EA06FB0638F04F5FD8CF8DE691E0A0E081
:100DA000B0E0ECCF4093D80BC90164E670E00E943C
:100DB00093AEEC01C90160E971E00E9493AE3097F7
:100DC00021F42097D9F40097C9F04DE651E060E096
:100DD00070E0441A550A660A770AC418D508E6086E
:100DE000F708A5E3B3E020E0213069F43097E9F596
:100DF000209711F40097C9F54DE106C04EE651E089
:100E000060E070E0E6CF4C9150E070E060E031E0EF
:100E1000320FC416D506E606F70640F0C41AD50A06
:100E2000E60AF70A1196232F3C30F1F62F5F209344
:100E3000D70BC394C092D60B80926A1290926B1219
:100E4000A0926C12B0926D12DF91CF911F910F9111
:100E5000FF90EF90DF90CF90BF90AF909F908F90DA
:100E60007F906F905F904F9008954CE1CDCF0E949E
:100E7000AF850E943E868091D80B90E08E54984FAB
:100E800008950E94AF850E943E868091D70B90E026
:100E900008950E94AF850E943E868091D60B90E017
:100EA00008950E94AF850E943E868091D30B90E00A
:100EB00008950E94AF850E943E868091D40B90E0F9
:100EC00008951F920F920FB60F9211240BB60F9236
:100ED0002F933F934F935F936F937F938F939F9342
:100EE000AF93BF93EF93FF9380919A110E944F7439
:100EF00020919D1130919E112F5F3F4F30939E1195
:100F000020939D1190919C11953618F096E0909346
:100F1000991190919911943009F46EC0F8F49230BF
:100F200031F1933009F44CC090919B11992319F041
:100F3000811171C02F9AFF91EF91BF91AF919F9155
:100F40008F917F916F915F914F913F912F910F9072
:100F50000BBE0F900FBE0F901F901895953009F49F
:100F600057C0963009F791E0909369124FC08111F4
:100F7000DBCF20919D1130919E112436310528F44C
:100F800010929E1110929D11CFCF10926912109263
:100F90009C11E0919C1191E09E0F90939C11F0E0C8
:100FA00020919D1130919E11EE0FFF1FE156FE4ED4
:100FB0003183208310929E1110929D1193E019C0ED
:100FC000813009F0B1CFE0919C1191E09E0F909398
:100FD0009C11F0E020919D1130919E11EE0FFF1FAA
:100FE000E156FE4E3183208310929E1110929D1186
:100FF00094E09093991198CF882359F220919D11F4
:1010000030919E112536310508F48ECF95E0F1CF51
:1010100081118ACFB5CF2F988ECFCF93DF9391E0F8
:10102000909355118823B9F0C091B800D091BA00BF
:101030008091BC008A7B8093BC0060E084E10E94C8
:10104000877E60E085E10E94877E0E94B57ED09316
:10105000BA00C093B800DF91CF9108958F929F920C
:10106000AF92BF92CF92DF92EF92FF920F931F93B6
:10107000CF93DF93D091860CD13208F0D7C0182FD0
:10108000C091850C0E941B7F6B017C0180917D0CBF
:1010900081116BC082E080937D0C10937C0C8FEFEC
:1010A00080937B0C10927A0CD093790CABEFB4E167
:1010B000E9E5FCE080E0D81391C01092580C8091D3
:1010C000580CCC0FC82BC093580C8091570C813012
:1010D00009F088C01092570C0E941B7F6B017C01A5
:1010E0008091580C8093BB0080917F0C9091800C74
:1010F000A091810CB091820C892B8A2B8B2BA1F0B3
:101100000E941B7F00917F0C1091800C2091810C1C
:101110003091820C6C197D098E099F0906171707FB
:101120002807390708F442C08091BC0083FDD8CF5E
:1011300085EC8093BC000E941B7F6B017C01809139
:101140007D0C823009F450C080917B0C8F3F09F4F4
:101150006FC080917B0C803209F46CC080917B0C55
:10116000803309F469C084E026C080917F0C90919F
:10117000800CA091810CB091820C892B8A2B8B2B37
:1011800009F484CF0E941B7F80907F0C9090800C8C
:10119000A090810CB090820C6C197D098E099F097A
:1011A00086169706A806B90608F070CF80917E0CC7
:1011B0000E940D8885E01092840C1092860C10928B
:1011C000830CDF91CF911F910F91FF90EF90DF90F3
:1011D000CF90BF90AF909F908F9008959D919193E5
:1011E0008F5F69CF85EEA5CF80917F0C9091800CA9
:1011F000A091810CB091820C892B8A2B8B2B09F446
:101200009ECF0E941B7F00917F0C1091800C20913B
:10121000810C3091820C6C197D098E099F0906178B
:1012200017072807390708F08ACFC0CF81E0C3CF5E
:1012300080E0C1CF82E0BFCF83E0BDCFFC0124813D
:1012400031E03093830C2093850C1092840C109223
:10125000860C8385682B82EC9DE00E94F57481E00A
:101260000C942E880F931F93CF938C01C62F0E944E
:101270001E896C2F6460C8010E941E896C2F6B7FD1
:10128000C8010E941E8983EC90E00197F1F7CF918D
:101290001F910F910895CF93C82F682F607F8EE321
:1012A00091E10E94328980E1C89FB00111248EE350
:1012B00091E1CF910C943289CF93DF9300D000D08D
:1012C0001F921F92CDB7DEB798E0EBE2F3E0DE01AC
:1012D000119601900D929A95E1F79091471196170A
:1012E00008F46FEF70E0660F771F21E030E02C0FFD
:1012F0003D1F620F731FFB019081890F8068289644
:101300000FB6F894DEBF0FBECDBFDF91CF910C9426
:101310004B890F931F93CF938C01C62F607F616021
:101320000E94328980E1C89FB00111246160C80128
:101330000E94328981E090E0CF911F910F91089532
:1013400085ED8093BC0080917F0C9091800CA091E2
:10135000810CB091820C0796A11DB11D23E0B695BA
:10136000A795979587952A95D1F72091BC0024FDE4
:1013700003C010927D0C089540917F0C5091800C19
:101380006091810C7091820C452B462B472B69F3A1
:101390000097A105B10541F025E32A95F1F700007A
:1013A0000197A109B109E1CF80917E0C0C940D88C1
:1013B0001F920F920FB60F9211240BB60F922F931C
:1013C0003F934F935F936F937F938F939F93AF93CD
:1013D000BF93EF93FF938091B900887F803609F423
:1013E0004DC008F040C0883209F4A9C028F580310A
:1013F00009F49DC0C8F4882309F4FBC0883009F4BF
:1014000096C0FF91EF91BF91AF919F918F917F9186
:101410006F915F914F913F912F910F900BBE0F9065
:101420000FBE0F901F901895883109F488C0803244
:1014300041F780937B0C14C0803409F49DC040F4C4
:101440008033B9F38833E9F680937B0C85ECB0C028
:10145000803509F485C0883509F496C0883489F64A
:101460000E94A089CECF883909F48CC038F588371E
:1014700029F050F4883611F0803719F683E0809314
:101480007D0C1092981157C0883809F47BC08039C0
:1014900019F0803809F0B5CF80919811803208F0AA
:1014A00071C0E091981181E08E0F80939811809126
:1014B000BB00F0E0E858FE4E80833DC0803B39F031
:1014C000E0F4803A09F479C0883A09F09ACF84E0D0
:1014D00080937D0C1092771110927611E0918D120D
:1014E000F0918E1219958091761181110FC081E0D3
:1014F000809376111092561109C0803C09F4A6CF52
:10150000883C09F4A3CF883B09F07BCFE0917711A9
:1015100081E08E0F80937711F0E0EA5AFE4E8081D1
:101520008093BB00909177118091761129C08091B2
:10153000580C8093BB0085EC8093BC0062CF9091E7
:101540007A0C8091790C981758F5E0917A0C81E02B
:101550008E0F80937A0CF0E0E75AF34F8081E9CF49
:10156000E0917A0C81E08E0F80937A0C8091BB0021
:10157000F0E0E75AF34F808390917A0C8091790CD8
:101580009817C8F285E8D8CFE0917A0C81E08E0FE9
:1015900080937A0C8091BB00F0E0E75AF34F808390
:1015A00080917C0C81115CCF81E08093570C84EAA0
:1015B0008093BC0010927D0C24CF85EC8093BC00FE
:1015C00010927D0C80919811803230F4E091981146
:1015D000F0E0E858FE4E10826091981170E0E091C2
:1015E0008B12F0918C1288E791E119951092981165
:1015F00008CF10927B0C34CF4F925F926F927F9204
:101600008F929F92AF92BF92CF92DF92EF92FF9212
:101610000F931F93CF93DF93EC0142305105610587
:10162000710590F480E0DF91CF911F910F91FF90B1
:10163000EF90DF90CF90BF90AF909F908F907F9072
:101640006F905F904F90089589859A85AB85BC8592
:101650000196A11DB11D84179507A607B70710F3C2
:10166000CB88DC88ED88FE888F89803109F042C004
:10167000BB27A72F962F852F480159012A013B012F
:10168000C80ED91EEA1EFB1E809168029091690265
:10169000A0916A02B0916B02C816D906EA06FB0651
:1016A00099F58F898031C1F5B301A20155276627CD
:1016B0007727440F551F41575D4EFA019182808272
:1016C000809150118160809350118A89823080F01E
:1016D0008D819E81AF81B8858C0D9D1DAE1DBF1D76
:1016E0008093511190935211A0935311B0935411C0
:1016F00081E099CFDB01CA01E7E0B695A795979500
:101700008795EA95D1F7B8CF40E0C701B6010E94AE
:10171000E8758111C6CF86CFB301A2014F77552757
:1017200066277727440F551F440F551F41575D4EBD
:10173000FA0180829182A282B382C2CF8F929F925D
:10174000AF92BF92CF92DF92EF92FF920F931F93CF
:10175000CF93DF93FC0181859285A385B4850196A3
:10176000A11DB11D84179507A607B70770F480E087
:10177000DF91CF911F910F91FF90EF90DF90CF906D
:10178000BF90AF909F908F90089583889488A5888C
:10179000B6888789803189F5BB27A72F962F852F9B
:1017A000E9016A017B018F01BC01CD01680D791D42
:1017B0008A1D9B1D8090680290906902A0906A0229
:1017C000B0906B0286169706A806B90601F5F801D7
:1017D0008789803111F5DD24EE24FF24F601EE0F18
:1017E000FF1FE157FD4E80819181B0E0A0E088832A
:1017F0009983AA83BB8381E0BBCFDB01CA01C7E029
:10180000B695A79597958795CA95D1F7C9CF40E02A
:101810000E94E8758111DBCFAACFE894C7F8DD24D8
:10182000EE24FF24F601EE0FFF1FEE0FFF1FE1571E
:10183000FD4E80819181A281B381BF70D8CF4F923C
:101840005F926F927F92AF92BF92CF92DF92EF92B0
:10185000FF920F931F93CF93DF9300D01F92CDB7CA
:10186000DEB78C0149835A836B837C835901C12C79
:10187000D12C7601412C82E0582E612C712C4981AB
:101880005A816B817C819E012F5F3F4FC8010E946E
:101890009E8B882339F1F8018585A301920104C04C
:1018A000220F331F441F551F8A95D2F7DA01C90151
:1018B000C80ED91EEA1EFB1E49815A816B817C81AC
:1018C0008789803111F188EF9FEFAFEFBFE04817B4
:1018D00059076A077B0798F2F501C082D182E2823C
:1018E000F38281E00F900F900F900F90DF91CF91D6
:1018F0001F910F91FF90EF90DF90CF90BF90AF902E
:101900007F906F905F904F90089588EF9FEFA0E0D9
:10191000B0E0DDCFCF93DF93EC018D81882389F197
:101920008C8187FF2AC06E857F858889998941E0EF
:101930000E94E875882329F1EA8980E2E89FF00196
:101940001124E157FD4E3097E1F08D81823040F453
:101950008B899C89AD89BE89848F958FA68FB78F1F
:101960008F89988D938F828F8F89988DA98DBA8D4D
:10197000B58BA48B8C818F778C83DF91CF910C9466
:10198000AD7580E0DF91CF9108958F929F92AF92D5
:10199000BF92CF92DF92EF92FF920F931F93CF935C
:1019A000DF93EC018D8181110EC080E0DF91CF913A
:1019B0001F910F91FF90EF90DF90CF90BF90AF906D
:1019C0009F908F9008950B891C892D893E8904175B
:1019D00015072607370748F34A015B01823031F4C7
:1019E0008A869B86AC86BD8681E0E0CF8114910417
:1019F000A104B10449F41E821F82188619861A8632
:101A00001B861C861D86F0CF0A851B852C853D858F
:101A1000EB8DFC8D858590E00996B901A8014150B8
:101A2000510961097109082E04C07695679557958B
:101A300047950A94D2F775016401E1E0CE1AD10806
:101A4000E108F10804C0F694E794D794C7948A9506
:101A5000D2F7C416D506E606F70620F0012B022BB6
:101A6000032B11F58F89988DA98DBA8D8E839F8355
:101A7000A887B9878E010A5F1F4FC114D104E10402
:101A8000F10409F4ADCF4E815F81688579859801B5
:101A90008B8D9C8D0E949E8B91E0C91AD108E10824
:101AA000F1088111EACF81CFC41AD50AE60AF70AF4
:101AB000E1CF2F923F924F925F926F927F928F92DF
:101AC0009F92AF92BF92CF92DF92EF92FF920F93CD
:101AD0001F93CF93DF9300D01F92CDB7DEB78C0159
:101AE0005B011A01DC0115968C911597813009F084
:101AF000C8C014968C9181FFC4C082FDAEC0610144
:101B0000D8011A964D915D916D917C911D97C114EC
:101B1000D10409F429C15B968D919C915C97FC01DD
:101B200074802FEF270D2A013B0139E076946794EA
:101B3000579447943A95D1F7722E74207A01F1E0C8
:101B4000FF22711020C0E114F104E9F416964D91C2
:101B50005D916D917C911997411551056105710554
:101B600009F098C057968D919D910D90BC91A02D34
:101B70000097A105B10509F0AFC0C8010E949B0AFA
:101B8000882309F47EC080E092E08E199F09460107
:101B90008C159D0508F44C01D8015B964D915C9124
:101BA0005C9716968D919D910D90BC91A02D0297FA
:101BB000A109B109FA01258504C0880F991FAA1F40
:101BC000BB1F2A95D2F74685578560897189840F96
:101BD000951FA61FB71F9C01AD01270D311D411D8B
:101BE000511D29013A01811432E0930609F07AC0AF
:101BF0008091680290916902A0916A02B0916B0293
